:020000040800F2
:10000000D4B1001089010008CF0100088DB40008A8
:10001000D3010008D5010008D70100080000000046
:10002000000000000000000000000000D9010008EE
:10003000DB01000800000000199001080985010893
:10004000E1010008E3010008E50100088911010849
:10005000E9010008EB010008ED01000845A50008D2
:10006000E1BE0108F3010008F5010008F7010008EE
:10007000F9010008FB010008953B0108FF01000899
:1000800001020008413701080502000807020008C4
:10009000358B00080B0200080D0200081DBF010887
:1000A0004D0801086D090108BD0901083506010860
:1000B000D9080108DDBD01083D0701081F0200083D
:1000C0002102000823020008250200082702000878
:1000D000290200083137010871370108813701080A
:1000E0005D2E0108330200083502000837020008BF
:1000F000390200083B0200083D0200083F020008E8
:1001000041020008592E0108057500084702000841
:10011000C9370108113801084D0200084F020008D4
:10012000F91C000853020008550200085702000895
:1001300059020008CD3B0108D93B01085F020008C5
:1001400061020008630200086502000867020008F7
:100150006902000859380108013701088938010887
:100160007102000873020008750200087702000897
:10017000790200087B0200087D0200087F02000867
:0801800081020008830200085F
:100188003E48854618F012F94EF63470CEF200005B
:10019800016831F0404101604EF68850CEF200000F
:1001A800016851F47001016000BF00BF00BFF1EEAB
:1001B800100A50F04070E1EE100A314831490160F0
:1001C80000F062B87047FEE7FEE7FEE7FEE7FEE7ED
:1001D800FEE7FEE7FEE7FEE7FEE7FEE7FEE7FEE7EF
:1001E800FEE7FEE7FEE7FEE7FEE7FEE7FEE7FEE7DF
:1001F800FEE7FEE7FEE7FEE7FEE7FEE7FEE7FEE7CF
:10020800FEE7FEE7FEE7FEE7FEE7FEE7FEE7FEE7BE
:10021800FEE7FEE7FEE7FEE7FEE7FEE7FEE7FEE7AE
:10022800FEE7FEE7FEE7FEE7FEE7FEE7FEE7FEE79E
:10023800FEE7FEE7FEE7FEE7FEE7FEE7FEE7FEE78E
:10024800FEE7FEE7FEE7FEE7FEE7FEE7FEE7FEE77E
:10025800FEE7FEE7FEE7FEE7FEE7FEE7FEE7FEE76E
:10026800FEE7FEE7FEE7FEE7FEE7FEE7FEE7FEE75E
:10027800FEE7FEE7FEE7FEE7FEE7FEE700000220F6
:1002880008ED00E0000000082C49072291438D4644
:100298002B482C492C4A00F03EF82C482C492D4A72
:1002A80000F039F82C482D492D4A00F034F82D4833
:1002B8002D492E4A00F02FF82D482E492E4A00F0DD
:1002C8002AF82E482E492F4A00F025F82E482F49A3
:1002D800002200F02BF82E482E49002200F026F8C4
:1002E8002D482E49091A082903DB00220260043030
:1002F80001601D481D49884205D00268043003B4D6
:10030800904703BCF7E700208646EC460020002112
:10031800234A9047FEE7884207D0521A05D003784F
:1003280001300B700131013AF9D17047884202D08F
:1003380002700130FAE770471A487047D4B10010CC
:10034800F825020800000020BC070020B0030008C0
:10035800B003000838FD0108B42D02082047012029
:100368002047012038FD010838FD010838FD010843
:1003780038FD010838FD010838FD010838FD01087D
:1003880038FD0108F8250208BC070020202F0020AE
:1003980000000010D4AF0010202F002020470120BB
:0803A800D5B30008FFFFFFFFC1
:1003B00070B940F20000C1F2000040F2B1310268B1
:1003C0008388C0F6000153833C20012207F04CB81B
:1003D000012800D0704740F2000CC1F2000CDCF89C
:1003E0000010BCF804200A83704700BF70B940F2C7
:1003F0000000C1F2000040F2ED3102688388C0F6CF
:10040000000153830220012207F02EB8012800D0FA
:10041000704740F20003C1F2000340F2ED311A6868
:10042000B3F804C0C0F60001A2F818C03C200222B4
:1004300007F01AB810B5441C072C1ADC40F2000370
:10044000C1F2000393F81B1151FA04F010F00100FF
:100450000BD1FFF7ADFF40F23541C0F6000141205E
:100460002246BDE8104007F019B80020FFF7BEFF94
:10047000F1E710BD10B540F20004C1F20004012202
:100480002068B4F804C004F58871A0F818C084F896
:10049000142116F06BFEA06802688388138310BDD8
:1004A00010B540F20004C1F200040022206884F874
:1004B000142104F5887116F059FEA068026883883B
:1004C000538310BD08B503283DD8DFE800F02B1F8B
:1004D0000602BDE80840FFF7CDBF40F20003C1F2BD
:1004E000000340F2C5411A689888126910420CBF97
:1004F0004FF0000C4FF0010CC0F600011920032250
:1005000083F81AC1BDE8084006F0AEBFFFF7C8FF88
:1005100040F2C541C0F600010A200222BDE80840B1
:1005200006F0A2BF40F20000C1F2000040F2C54157
:1005300002688388C0F60001538302200122BDE8CF
:10054000084006F091BF08BD40F20003002810B536
:10055000C1F2000304461ADB93F81B0193F81A1149
:1005600011FA04F242EA0001C8B2062C83F81B011A
:1005700000DD10BD0020FFF7A5FF40F24951C0F695
:100580000001621C4120BDE8104006F087BF002238
:10059000104683F81B21EEE708B503283ED8DFE8B4
:1005A00000F02B1F0602BDE80840FFF763BF40F2D2
:1005B0000003C1F2000340F299511A689888126949
:1005C000104214BF4FF0000C4FF0010CC0F60001B8
:1005D0003C20032283F819C1BDE8084006F044BF5F
:1005E000FFF75EFF40F29951C0F600013C20022265
:1005F000BDE8084006F038BF40F20000C1F200003C
:1006000040F2995102688388C0F6000153834FF489
:10061000F5700122BDE8084006F026BF08BD00BF06
:1006200010B50346002854D0012848D040F20004F9
:10063000C1F2000494F81C2150B2002820DDD4F847
:100640000C3113F801CB013A4FF0FF3084F81BC195
:10065000C4F80C3184F81C21FFF7ECFE40F2216154
:100660000222C0F600014FF4167006F031FF94F933
:100670001C21002A22D104F10C01C4F80C1110BD78
:1006800094F81D21110616D4501EC2B2032B84F813
:100690001D2152D0130648D44FF0FF30FFF754FF0E
:1006A00040F22161C0F600014FF416700322BDE84C
:1006B000104006F00DBF032084F8180110BD40F271
:1006C0000002C1F2000292F81911C1B982F81801B2
:1006D00010BD40F20002C1F2000282F8193102237B
:1006E00082F81831FFF758FF40F22161C0F600018F
:1006F0004FF47A700122BDE8104006F0E9BE02F125
:100700000C03CC2182F81B11C2F80C314FF0FF30E2
:10071000FFF790FE40F22161C0F600014FF4167021
:100720000222BDE8104006F0D3BE40F2000CC1F238
:10073000000C03218CF8181110BDD4F80C3194F87A
:100740001B2103F8012B94F81D21C4F80C31A1E7FB
:1007500010B540F20004C1F200040346002084F802
:100760001C3184F81D11FFF75BFF94F81801022873
:10077000FBD094F8180110BDF8B540F20004C1F2A6
:1007800000044FF490720D460646002120461DF0ED
:10079000B7FD2946304608F0CFF9014604F58870C8
:1007A0000127A1602660A58016F09CFD022084F838
:1007B0001501C4F8105184F8147184F81771FFF70B
:1007C00059FE384619F0B6F8002384F81831F8BD00
:1007D000DFED147AC7EE807A08B59FED137A77EED5
:1007E000C77A17EE900A1BF087FC41EC100B1CF047
:1007F000BFFF51EC100B1BF09BFC07EE100A9FEDA6
:100800000B6ADFED0B7A67EE076A47EE067A26EE93
:10081000877ADFED086A47EE267A9FED070A37EE02
:10082000C00A08BD0022A1480050C347B9FCD5400A
:100830002A89274396210E3D00808843000000004E
:100840002DE9F04F2DED068BE14CE248E24D8FB0E3
:1008500002F04AF8D4F86001016882884B699FED84
:10086000D87B9FEDDE9A1A428DED087B8DED0C7BD7
:100870008DED0A7B4FF000060CBF4FF000084FF0E3
:1008800001080496CDF80880F0EE498AB0EE498A56
:1008900003960021607818F0F1F8D4F87461276CA1
:1008A0000196606CA16CE26C236DD4F854E0D4F82E
:1008B0005880D4F85CA0266ED4F880C00596666E89
:1008C000D4F888900696A66ED4F884B0079684442F
:1008D000D4F88C00E66FC4F880C0914403EB000CA0
:1008E000D4F89020D4F89430BF19E76708EB0306DA
:1008F0000EEB0207D4F89880059AD4F89CE0D4F85F
:10090000A0300AEB08008B44DDF81880C4F884B0EE
:1009100002EB0E01079AD4F8A4E0C4F8889008EB23
:10092000030A02EB0E03D4F8B490D4F8ACE0C4F898
:100930008CC0C4F89070D4F8B0C0E76EC4F894606E
:10094000C4F89C10D4F8A860216FC4F8A430626F7A
:10095000A36FC4F8980062447144206CC4F8A0A04E
:100960004B44BE19C4F8A860C4F8B020C4F8B43031
:10097000C4F8AC101BF0F2FA93A3D3E900231BF0E8
:1009800059FD00230022C3F6D0731BF053FD1BF06A
:10099000CFFB94ED557A09EE900AD5EDD67A79EE33
:1009A000879A48EE279AD5EDD97AD4F84480D4F8BE
:1009B00048A048EEA79AD5EDDC7A404649EE279A42
:1009C0001BF0CCFA80A3D3E900231BF033FD0023F6
:1009D0000022C3F6D0731BF02DFD1BF0A9FB94ED94
:1009E000567A0AEE100AD5EDD77A3AEE07AA08EE43
:1009F00027AAD5EDDA7A08EEA7AAD5EDDD7A50461A
:100A000009EE27AA1BF0AAFA6FA3D3E900231BF073
:100A100011FD00230022C3F6D0731BF00BFD1BF069
:100A200087FBD4ED577A06EE900A95EDD87A76EEEC
:100A3000A77A48EE077A95EDDB7A48EE877AD5ED0E
:100A4000DE6A95EDE27AB1EE4A6AF0EE692A46EE88
:100A5000072A49EE267A95EDE35AD5EDE45AF1EEF0
:100A6000676AB0EE627A06EE857A19EEA5AAD5ED30
:100A7000E55A95EDDF5A06EEA5AA87EE055AD4F899
:100A8000183141F21010C1F2000095EDE07A8AEEC3
:100A900007AAD0ED024A07EE103A04EE857AD0EDAF
:100AA000015A05EECA7AD5EDE73A95EDE64AF6EE3B
:100AB000006A26EE236A09EE846A27EE267A95ED0F
:100AC000E14A84ED467AD4F81C3176EE677A07EE77
:100AD000103AC7EE847A0AEE247A05EE257A27EEDC
:100AE000267A84ED477AD4F8203107EE103A77EE73
:100AF000277A67EEA66AC4ED486A09F02BFE049EC9
:100B00008EB1E66CD4F88870216DD4F88C00D4F8DE
:100B10009020636DBF1B411AD21AC4F88870C4F8C4
:100B20008C10C4F89020DDF804A01AF0010640F003
:100B30000B84E06F1BF012FA23A3D3E900231BF010
:100B400079FC00224FF07F531BF074FC1BF0F0FA8D
:100B50000346D4F88000C4F8B8301BF0FFF91AA39C
:100B6000D3E900231BF066FC00224FF07F531BF0FB
:100B700061FC1BF0DDFA0346D4F88400C4F8BC30F5
:100B80001BF0ECF910A3D3E900231BF053FC002267
:100B90004FF07F531BF04EFC1BF0CAFA0346D4F80B
:100BA0008800C4F8C0301BF0D9F907A3D3E90023AB
:100BB0001BF040FC0023002212E000BFAFF30080D6
:100BC00000000000000000004BD4AE44D99AD43E8F
:100BD0002001001038FD0108AC02001000000000E8
:100BE000C3F6D0731BF026FC1BF0A2FA0346D4F820
:100BF0008C00C4F8C4301BF0B1F90FF2D053D3E924
:100C000000231BF017FC00230022C3F6D0731BF057
:100C100011FC1BF08DFA0346D4F89000C4F8C830DC
:100C20001BF09CF90FF2A453D3E900231BF002FC44
:100C300000230022C3F6D0731BF0FCFB1BF078FAF4
:100C40000346D4F89400C4F8CC301BF087F90FF2B7
:100C50007C53D3E900231BF0EDFB00230022C3F6F5
:100C6000E0731BF0E7FB1BF063FAC4F8D000D4F884
:100C700098001BF073F90FF25453D3E900231BF0D3
:100C8000D9FB00230022C3F6E0731BF0D3FB1BF05B
:100C90004FFA0346D4F89C00C4F8D4301BF05EF938
:100CA0000FF22853D3E900231BF0C4FB00224FF0BE
:100CB0007F531BF0BFFB1BF03BFA0346D4F8A000A8
:100CC000C4F8D8301BF04AF90FF20053D3E90023DF
:100CD0001BF0B0FB00224FF07F531BF0ABFB1BF06F
:100CE00027FA0346D4F8A400C4F8DC301BF036F928
:100CF0000FF2D843D3E900231BF09CFB00224FF0F6
:100D00007F531BF097FB1BF013FA0346D4F8A8009F
:100D1000C4F8E0301BF022F90FF2B043D3E900230E
:100D20001BF088FB00224FF07F531BF083FB1BF06E
:100D3000FFF90346D4F8AC00C4F8E4301BF00EF918
:100D40000FF28843D3E900231BF074FB00224FF01D
:100D50007F531BF06FFB1BF0EBF90346D4F8B00098
:100D6000C4F8E8301BF0FAF80FF26043D3E900232F
:100D70001BF060FB00230022C3F6E0731BF05AFB5C
:100D80001BF0D6F9C4F8EC00D4F8B4001BF0E6F878
:100D90000FF23843D3E900231BF04CFB0023002261
:100DA000C3F6E0731BF046FB1BF0C2F9C4F8F00079
:100DB000D4F8D010D4F8EC20D4F8F030E66707EE81
:100DC000101A06EE102AF7EE047A37EE677ADFED96
:100DD000F86A36EE676AF3EE097AF0EE672A47EEB4
:100DE000262A46EE267ADFEDF3AADFEDF39A32EEFD
:100DF000AA7A77EEAA7A9FEDF1AA94ED3D6AD4ED36
:100E00003E6A27EE297A67EEA97A06EE0A7A46EE5E
:100E10008A7A00EE103A94ED3F8A84ED3D7AC4ED73
:100E20003E7AC4F88060C4F88460C4F88860C4F86E
:100E30008C60C4F89060C4F89460C4F89860C4F8FA
:100E40009C60C4F8A060C4F8A460C4F8A860C4F8AA
:100E5000AC60C4F8B060C4F8B460FFF7B9FC28EE29
:100E60000A8A30EE2A0AB0EE486A00EE296AD4F8FF
:100E7000B820D4F8BC10D4F8C03094ED567A04EE03
:100E8000902A06EE901AD4ED557AB3EE048A36EE27
:100E9000488A95EDD75AD5EDD65A76EE876A74EE24
:100EA000A77A48EE056A48EE257A68EE088A04EECD
:100EB000103AD5EDDA4AD5EDD95A94ED577A95ED39
:100EC000D85A34EE077A48EEA46A48EEA57A28EE9E
:100ED000889AD5EDDD4AD5EDDC5A08EE057A95ED18
:100EE000DB5A49EE257A49EE246A08EE857AD5ED7B
:100EF000DE5A95EDE25A09EE257AB0EE674AF1EE38
:100F0000665A05EE854AD5EDE44A57EEA46AD5ED5A
:100F1000E33AB0EE445A95EDE54AF1EE474A04EE65
:100F2000A35A95EDE73A44EE846AD5EDE63AD5ED5D
:100F3000E04A95EDDF4A65EE835A47EEA35A85EE07
:100F4000044A41F21010C1F20000C6EEA46AD5EDC9
:100F5000E17A35EEC77AD0ED014A87EE277A90ED37
:100F6000025A64EEA65A64EE247A55EE045A46EE0E
:100F7000857AC4ED495AC4ED4A7A84ED4B7AD4F8A7
:100F8000D430DFED8F7A07EE103A27EE277AD4EDD2
:100F9000417A67EE299A47EE8A9A84ED3F6A84ED9A
:100FA000406AC4ED419AD4F8D810D4F8DC20D4F8C3
:100FB000E030D5ED977A05EE901A95ED9A4AD5ED89
:100FC000986A06EE102A95ED9B7A75EEA75A48EEC0
:100FD000045AD5ED997A04EE103A36EE266A08EEF8
:100FE000076AD5ED9C6AD5ED9D3A95ED9E7A74EE33
:100FF000277A48EE267AD5ED9F2A95EDA04A48EE4D
:10100000A35A08EE876A29EE044A95EDA63AD5ED73
:10101000A73A48EEA27AD5EDA36A95EDA47A75EECB
:10102000845A34EE066A48EE036A08EE237AD5ED58
:10103000AF0A95EDB11A95EDA92AD5EDAA2A74EE5D
:10104000273AB1EE653AB0EE464AD5EDA81A56EE0B
:10105000205AD5EDA57A03EE014A48EE826A08EEE1
:10106000A27A95EDAD2AD5EDB09A95EDB20AD5EDFF
:10107000AC0AF1EE632A48EE217A42EEA95A95EDC8
:10108000B41AD5EDAB1A02EE804A09EE027A49EEA7
:10109000206A95EDB32A26EE016A48EEA17AD5EDD5
:1010A000AE2A03EE026AC5EEA66A84EE077A49EE1E
:1010B000227A76EE633A24EE876AC3EEA77A64EE6C
:1010C000A64A15EE266A45EE074A84ED4C6AC4ED41
:1010D0004D4AC4ED4E7AD4F8E420D4F8E8309FEDC0
:1010E000396A05EE902A05EE103ADFED376A94ED85
:1010F000437AD4ED447A75EE865A35EE066A05EEEB
:10110000A67A46EE267A95EDEA6AF6EE006A27EEB2
:10111000267A67EEA67AB4EE6A6AF1EE10FA84EDEA
:10112000437AC4ED447A40F0BA8184ED457AD4F82C
:10113000C430029905EE903A94ED525AD4F8C83072
:10114000D4F8CC20D4ED547A002900F0788102EE56
:10115000902A95EDB72A32EEE77AD5EDBA1A72EEFB
:10116000476A48EE216A95EDBD1A48EE816AD5EDD1
:10117000C00A49EE206ABFEE006AD5EDB57A95ED5A
:10118000B80AD5EDBB0A95EDBE1AD4ED534A95EDDC
:10119000B67A95EDB92AD5EDBC2A95EDBF3A01EEA8
:1011A000903AB0EE464AF1EE663AFF2314E000BFF3
:1011B000FFFF794300000000A323393C711B7D3FF2
:1011C000EA4EEB401283A03E098603474BD4AE445F
:1011D000D99AD43EFB01863535EEC5AA71EEE49A64
:1011E0004AEE047A09EE867A40EE087A02EE087A30
:1011F00040EEA87A02EEA87A41EE097A03EE097A67
:10120000D5EDC42A95EDC52A95EDC1AAD5EDC29AB2
:1012100095EDCD4AD5EDCF4AB0EE471A08EE22AA99
:1012200048EE029AF0EE671A47EE041AD5EDC70AA7
:1012300095EDC80A07EEA41A95EDC65A08EEA0AAC5
:1012400048EE809AD5EDC30A95EDCB3AD5EDCE5A4E
:10125000D5EDD0AA95EDCA6AB0EE614AF0EE414AEA
:1012600048EE050A03EEA54A43EEAA4A49EE039A60
:10127000D5EDD22A95EDC92A09EE06AAD5EDD11AE7
:1012800027EE221A48EE820A07EEA11AD5EDCC7A93
:1012900084EE0A5A41F2101BC1F2000B039984F844
:1012A0008831481C0390C4EEA95A49EE270A71EE12
:1012B000666A9BED010A86EEA06ADBED02AA20EECB
:1012C00025AA65EE009A1AEE85AA45EEAA9A84ED43
:1012D0004FAAC4ED509A84ED516AD4F8C4001AF0B4
:1012E0000BFF02460B46DDE90A011AF05FFFCDE96C
:1012F0000A01D4F8C8001AF0FFFE02460B46DDE9E9
:101300000C011AF053FFCDE90C01D4F8CC001AF00F
:10131000F3FE02460B46DDE908011AF047FFCDE96E
:101320000801D4F88071D4F87C617A0004EE902A28
:101330005FED583AB8EE644AC4F8786124EE233A77
:1013400084ED613A09F010FAD4F86031029E1A680F
:101350009B88506903420CBF00270127BE426AD018
:101360005269134060D003981AF0E0FD8846814628
:1013700043464A46DDE90A011BF012F91AF0D8FE8D
:1013800009EE900A43464A46DDE90C01C4ED529A43
:101390001BF006F91AF0CCFE0AEE100A43464A4644
:1013A000DDE9080184ED53AA1BF0FAF81AF0C0FE3B
:1013B000DDF80C80C4F85001B8F1640F0AEE900A11
:1013C00077DD79EEA96A012716EE900A02971AF0E6
:1013D00093FE02460B46DDE90A011AF0E5FE7AEEBD
:1013E0000A3AA8F1020CCDE90A0113EE900ACDF8F1
:1013F0000CC01AF081FE02460B46DDE90C011AF022
:10140000D3FE3AEEAA7ACDE90C0117EE100A049742
:101410001AF072FE02460B46DDE908011AF0C4FE1E
:10142000CDE90801FFF735BA4FF00109CDF810906A
:101430000293FFF72EBA00270497FFF72ABA00EEAF
:10144000902A95EDB70A70EEE7AA95EDBA6A7AEEA2
:10145000806A48EE066A95EDBD3A48EE836AD5ED9E
:10146000C07A49EE276AB7EE006A01EE903AD5EDF0
:10147000B57A95EDB80AD5EDBB0A95EDBE1AD4ED57
:10148000534A95EDB67A95EDB92AD5EDBC2A95ED7E
:10149000BF3AF1EE663AB0EE464A01239CE6F7EE1B
:1014A000005AB4EE656AF1EE10FA07D1C4ED457A40
:1014B0003DE6012602960496FFF7EBB9B0EE000A6E
:1014C000B4EE406AF1EE10FA7FF431AE77EE277A8F
:1014D00067EEA66AC4ED456A29E600BFAFF3008057
:1014E0002DE9F04F2DED048B642083B009F06EFAE6
:1014F000192009F06FF89FED8A7B40F22015C1F2A8
:1015000000055BEC17AB8DED007BD5F87841D0463C
:10151000D9461926D5F87831A342FBD0D5F87841C1
:10152000D5F8B8001AF0E8FD02460B464046494699
:101530001AF03CFE8046D5F8BC0089461AF0DCFD66
:1015400002460B46504659461AF030FE8246D5F800
:10155000C0008B461AF0D0FD02460B46DDE90001C3
:101560001AF024FE013ECDE90001D3D1D5ED400AA9
:1015700040F2AC240023C1F200040022C4F239037B
:1015800040464946B3EE048A30EEC88A1BF008F89C
:10159000D4EDD68A28EE280A064610EE100A0F4629
:1015A0001AF0AAFD02460B46304639461AF0FEFDF7
:1015B00068EE088A94EDD99A28EE897A064617EEE5
:1015C000100A0F461AF098FD02460B46304639467F
:1015D0001AF0ECFD28EE289AD4EDDC7A69EE276A41
:1015E000064616EE900A0F461AF086FD02460B4696
:1015F000304639461AF0DAFD1AF09AFD06EE100A66
:101600000023F1EE465A0022C4F2390350465946EF
:10161000C5ED555A1AF0C4FF94EDD75A68EE054A45
:10162000064614EE900A0F461AF066FD02460B4677
:10163000304639461AF0BAFD94EDDA4A68EE843A3B
:10164000064613EE900A0F461AF056FD02460B4668
:10165000304639461AF0AAFD94EDDD3A69EE032AC8
:10166000064612EE900A0F461AF046FD02460B4659
:10167000304639461AF09AFD1AF05AFD02EE100A69
:101680000023F1EE421A0022C4F23903DDE9000121
:10169000C5ED561A1AF084FF94EDD81A28EE018A87
:1016A000064618EE100A0F461AF026FD02460B46B3
:1016B000304639461AF07AFDD4EDDB0A68EEA08A8E
:1016C000064618EE900A0F461AF016FD02460B4623
:1016D000304639461AF06AFD94EDDE0A29EE009A8A
:1016E000064619EE100A0F461AF006FD0B46024692
:1016F000394630461AF05AFD1AF01AFD07EE100A64
:101700000023F1EE477AC5ED577AC5F82431C5F8C4
:101710002831C5F82C3103B0BDEC048BBDE8F08F47
:1017200000000000000000002DE9F04F4FF64C5083
:1017300040F220189DB0C1F20008C0F601004FF43D
:10174000805A01F0D1F8C4F2020A4FF4C6720021A7
:1017500040461CF0D5FD4FF48061504607F0ECF98F
:1017600004688588C8F860014FF48071258350466D
:1017700007F0E2F90768C8F8640180884FF48051E7
:101780007883504607F0D8F94FF4006B02688688DA
:10179000C8F86801C4F2020B56834FF40041584662
:1017A00007F0CAF903688488C8F86C015C8319A83B
:1017B00015F098FD002000244FF0030AFD25C4F227
:1017C000020019A919958DF868A08DF86B4015F0E5
:1017D000CDFC4FF48060C4F2020019A93F27CDF878
:1017E00064A046F2104915F0C1FC584619A9C4F28C
:1017F0000209199715F0BAFC01214FF4E06015F0C9
:1018000047FEA3214846C8F8701142F2083615F089
:10181000BFF940F2BC726023C4F20106C2F20002BA
:101820004FF0040B48466946029201964FF48072CD
:1018300004934FF480654FF440334FF400674FF446
:1018400000560A9306950797089609920094039408
:101850000594CDF82CB0CDF830A00D940E9415F071
:1018600099FA01224846182115F050FB4FF23D012C
:101870004846C9F2000115F061FB0121484615F008
:10188000E7FA4FF0010938251BA88DF86C508DF848
:101890006D408DF86E408DF86F9015F071F815A8B9
:1018A00015F0FEF816274FF4804115A84FF40055A7
:1018B000C4F2010517911597169415F0D7F80FA8E3
:1018C00015F0CAF810260FA928468DF850600F941D
:1018D0008DF840908DF841901194139415F090F884
:1018E0000721022328464A4615F0EAF8022207217A
:1018F0001346284615F0E4F80721022328465246ED
:1019000015F0DEF80721022328465A4615F0D8F8CC
:101910000E2105220223284615F0D2F80E210622B8
:101920000223284615F0CCF80E2107220223284670
:1019300015F0C6F80E2108220223284615F0C0F83B
:1019400028460F210922022315F0BAF80F210A2296
:101950000223284615F0B4F80F210B220223284653
:1019600015F0AEF80F210C220223284615F0A8F836
:1019700008210D220223284615F0A2F808210E2284
:101980000223284615F09CF808210F22022328463E
:1019900015F096F8022310220821284615F090F839
:1019A0004FF4045749462846C4F2010715F0D8F809
:1019B0000FA815F051F8102238460FA98DF85020C5
:1019C0000F948DF840908DF841901194139415F078
:1019D00017F80921384602234A4615F071F8022209
:1019E00038460921134615F06BF8384609210223C1
:1019F000524615F065F83846022309215A4615F07B
:101A00005FF8384605220223594615F059F8384642
:101A100006220223594615F053F8384607220223BE
:101A2000594615F04DF8384608220223594615F05C
:101A300047F8384605210922022315F041F83846B7
:101A4000052102230A2215F03BF8384605210B2216
:101A5000022315F035F8384605210C22022315F033
:101A60002FF8384606210D22022315F029F83846B2
:101A700006210E22022315F023F8384606210F22F4
:101A8000022315F01DF84FF40856102202230621F8
:101A90003846C4F2010615F013F80FA814F0DCFF65
:101AA000102330460FA98DF850300F948DF84090D8
:101AB0008DF841901194139414F0A2FF3046022344
:101AC00051464A4614F0FCFF022330461A4651465E
:101AD00014F0F6FF304602235146524614F0F0FF50
:101AE000304651465A46022314F0EAFF30460A2196
:101AF0000522022314F0E4FF30460B2106220223C4
:101B000014F0DEFF0221304607220B4614F0D8FF06
:101B10000221304608220B4614F0D2FF0221304643
:101B200009220B4614F0CCFF022130460A220B4654
:101B300014F0C6FF30460D210B22022314F0C0FF23
:101B40000C2230460223114614F0BAFF30460D2213
:101B50000223214614F0B4FF304621460E22022310
:101B600014F0AEFF304602230F22214614F0A8FFE6
:101B7000102202233046214614F0A2FF484614F0FA
:101B8000F9FF2846494614F091FF3846494614F0BB
:101B90008DFF3046494614F089FF2146484616F02D
:101BA000E7FE4FF658510646C0F60101582088F866
:101BB000016008F097FE40F67C06C2F20006074678
:101BC00040F6410007F5AE73214645F60A02C0F61D
:101BD0000000376017F08AFD8446284688F800C068
:101BE00014F0B8FF642017F0A5FED8F8D010D8F88C
:101BF000EC20D8F8F00003EE901A02EE902AB7EE2F
:101C0000043A33EEC30ADFED386A32EEC36AF3EE0C
:101C1000091AF0EE615A40EE265A46EE261A00EEF8
:101C2000100AC8ED3D5AC8ED3E1AFEF7D1FDD8F8AE
:101C3000D430DFED2E0A01EE103A61EE207A88ED05
:101C40003F0AC8ED417AFFF74BFCD8ED417AB2EE7E
:101C5000017AF4EEC77AF1EE10FA22D49FED244A0D
:101C6000F4EEC47AF1EE10FA31D4F3EE014AF4EE58
:101C7000E47AF1EE10FA1FD49FED1E5AF4EEC57A05
:101C8000F1EE10FA0AD54FF698500021C4F2A001E7
:101C9000C0F60100C8F8081100F026FE1DB0BDE82E
:101CA000F08F4FF65C504FF08041C0F60100C8F84D
:101CB000081100F019FEF1E74FF684504FF0814211
:101CC000C0F60100C8F8082100F00EFEE6E7002388
:101CD0004FF67050C4F24003C0F60100C8F8083156
:101CE00000F002FEDAE700BFFFFF7943EA4EEB4067
:101CF000CDCC4C416666AA4110B54FF4C84CC4F235
:101D0000020CDCF800104FF23D02C9F20002CCF8E0
:101D1000082048F22000C1F2000001EA000323B9C4
:101D200040F2BC73C2F2000300E0864B40F2201286
:101D3000C1F20002B3F848C0B3F84E108C44B3F8B7
:101D400054008444B3F85A10614450680818506035
:101D5000B3F802C019898C44D8898444998A6144B3
:101D6000906808189060B3F804C059898C44188AA8
:101D70008444D98A6144D0680818D060B3F800C0A0
:101D8000D9888C4498898444598A61441069081818
:101D90001061B3F818C0D98B8C44988C8444598D49
:101DA0006144506908185061B3F830C0D98E8C4432
:101DB000988F8444B3F84210614490690818906188
:101DC000B3F81CC0D1690CEB0100D061B3F840C07E
:101DD000116A0CEB01001062B3F81AC0198C8C4424
:101DE000D88C8444998D6144506A08185062B3F8C5
:101DF00032C0198F8C44D88F8444B3F844106144A6
:101E0000906A08189062B3F84AC0B3F850108C4436
:101E1000B3F856008444B3F85C106144D06A0818E3
:101E2000D062B3F828C0D98D8C44988E8444598FE1
:101E30006144106B08181063B3F84CC0B3F852102B
:101E40008C44B3F858008444B3F85E106144506B7E
:101E500008185063B3F822C0916B0CEB010090633B
:101E6000B3F846C0D36B0CEB0301D163D2F8700119
:101E700000F10103C2F87031A42B62D14FF440602D
:101E8000C4F20000416A96464FF00003C2F8703178
:101E9000D2F8742102F10104CEF8744114F0010F5C
:101EA0000BD040F2201CC1F2000CDCF860311A6843
:101EB00054699B88234242D0538340F22014C1F2DC
:101EC0000004636823644FF000036360A0686064EB
:101ED000A360E268A264E3602069E0642361626950
:101EE00022656361A0696065A361E269A265E3613F
:101EF000206AE0652362626A22666362A06A6066A5
:101F0000A362E26AA266E362206BE0662363626B0F
:101F100022676363A06B6067A363E26BA267E363FE
:101F2000D4F87C010A1AC4F88021C4F87C1116F098
:101F30001BFB607816F0DEFE16F01CFB10BD138351
:101F4000BBE710BD1C0800202DE9F04101FB02F4A5
:101F5000A3B28846064604211846174608F0A0FC9E
:101F60001FFA88F105460346BAB2304617F090FDD5
:101F70009FED030A28462146BDE8F04117F03CBD1D
:101F8000000000002DE9F04F2DED028B8BB0B2F870
:101F900000A00692B2F802B044880588069E099017
:101FA0009FED8C8A0BFB0AF30891A542B4BFAA46A9
:101FB000A2467068CDF810A0B0EE480A194617F096
:101FC0001BFD5246002A00F06682099B5A68029265
:101FD000DDF80880029E4FEA840B611C08EB0B0AB7
:101FE0004FF000088800043E444505900096079095
:101FF000CDF80CA0F0EE485A40F3E3800098D0ED05
:10200000017AF0EE486A47EEA76A6FEA080C08F119
:1020100001030CEB0409021D9C4209F00101F0EEE2
:10202000667A15DD41B10432D2ED000A01339C42DB
:10203000164640EEA07A0BDD92ED010A40EE007AE2
:1020400092ED027A023308329C4247EE077AF3DCC3
:10205000B1EEE76A0299D1ED000AF4EEC80AF1EE9A
:1020600010FAC8BFB1EE466AB4EE486AF1EE10FA53
:10207000894600F0A980069B5A885E6802FB088AA0
:1020800006EB8A0E8EED006AD1ED001A08F101060A
:1020900031EEC61AB542019681ED001A7ADD039839
:1020A000009FB446C246464654456EDD6FEA0603BD
:1020B0001A19D0ED001A97ED012A731C02F00108DD
:1020C000F0EE657A3A1D9C42014641EEC27A1EDD71
:1020D000B8F1000F0AD0043290ED010A92ED007AB7
:1020E0000133011D9C4240EE477A10DD91ED013A2B
:1020F000D2ED013A43EE637A91ED022AD2ED022A43
:102100000233083108329C4242EE627AEEDCD9EDAD
:10211000006A26EE265A90ED004AC7EE857AF14312
:10212000721C01EB04080346944208F0010107F118
:102130000408D7ED014A07EEE44AA3EC014A24DD86
:1021400061B108F1040893ED005AD8ED006A07EE7A
:10215000E65A01329442A3EC015A16DDD3ED000A8F
:1021600098ED011A47EEC10A9E46EEEC010A98ED81
:10217000020A93ED017A07EEC07A02327346944266
:10218000A3EC017A08F10808E8DC0CF1010C6545C4
:10219000584489DCDDF808A00598039E009B079948
:1021A0000AEB000C1A18DDF810A0CDF808C0701862
:1021B000019E0092564503900ED0B04644453FF72D
:1021C0001DAFF0EE487A43E700200BB0BDEC028B68
:1021D000BDE8F08F00000000049A02F1FF3B002AE6
:1021E00048D002FB04B76FEA0403B800DDF824A06E
:1021F000069F009411464FEA8309A2008D4201F127
:10220000FF3C33DDB7F80280DAF804407B680CFB52
:1022100008162418013E03EB8606D4F800806FEA06
:10222000010C4B1C0CEB050EC6F8048004369D42D5
:102230000EF0010C144419DDBCF1000F07D0D4F8E6
:1022400000C001339D4246F804CF14440EDDD4F89B
:1022500000C004EB020EC6F804C0DEF800400233F2
:10226000B46008369D420EEB0204F0DC01394844AC
:10227000C4D1009C089B002B00F00B81089D1A889C
:102280006988686801FB02F11FED2E0A17F0B4FBA4
:10229000049E631E9E4225DC621C686802FB03FCF0
:1022A00000EB8C0EC2EB82719D1BA31E89004FF0C8
:1022B0007E509E42CEF8000005F001050EEB0102B3
:1022C00010DC2DB1049D1060013B9D420A4409DCE5
:1022D000DDF810A010605518023B9A45286005EB08
:1022E0000102F5DDBBF1FF3F00F0D380089E099AA3
:1022F00075685268631C03FB0BF081006D18C3EB1B
:10230000837301959B00E6431FED4E5A01380493F9
:10231000019B5118B50002EB8006F0EE455A009182
:10232000059502960393A200019800994FF07E55FF
:10233000056091ED006AB4EE456AF1EE10FA884648
:1023400000F090805C4540F38D800699039D4E8897
:102350004B6806FB0BB703EB8709029FDC465E4622
:10236000D7ED017A95ED003AF0EE652A43EE672A43
:102370006FEA06031919731C381D9C4201F0010A0B
:10238000F0EE627A05EB020121DDBAF1000F0AD00E
:10239000043091ED004AD0ED004A01339C4244EEF6
:1023A000647A114413DDD1ED003A90ED014A01EB5E
:1023B000020A43EEC47A90ED023ADAED002A0233C3
:1023C00008309C4242EEC37A0AEB0201EBDC99ED45
:1023D000000A26EE007AD7ED016AC7EE877AF0434D
:1023E000711C00EB040E8C420EF0010007F1040A90
:1023F00005EB0203D5ED004A47EEE64AC5ED004A7B
:1024000028DD70B10AF1040A93ED006ADAED003AB2
:1024100007EEE36A01318C4283ED006AD64613442D
:1024200018DD9AED012AD3ED001A47EEC21A03EB2C
:10243000020EC3ED001A9AED021ADEED000A47EE15
:10244000C10A02318C42CEED000A0AF1080A0EEBF5
:102450000203E6DC0CF1010C0435644502DD98ED65
:10246000006A7DE704990098019DDDF80CC04618CC
:102470006B180096029D059E01930BF1FF3BAD1971
:102480000CEB060ABBF1FF3F0295CDF80CA07FF4E0
:102490004BAF012099E64FF0FF3BEBE62DE9F04F03
:1024A00016888BB01E80B2F800A0149CA3F802A07E
:1024B000A4F800A01D46DDF854A00B88B2F802E095
:1024C000AAF80030B2F800C0A4F802E00E4609886D
:1024D000AAF802C005915488079029461046149A1C
:1024E000FFF750FD30462946159A17F089FB059BEA
:1024F000002B00F09480621C04F1FF3CA000C2EBB2
:102500008271CDF810C00690002004FB04F3039004
:10251000880004990190013B4FEA8C0A02FB01F20A
:102520009800CDF808A008920990049A01326CD066
:10253000DDF850B0DDF85490DBF80400099E029FEE
:10254000D9F80450DDF81C800899D8F804903A1D99
:102550006FEA040300EB060C049E00EB8108AD1843
:102560004FEA830B731C9C425CDD09EB070292ED82
:10257000017A55ED017ADCED016A46EEC77A6FEA21
:10258000030E01330EEB040104329C4201F0010AF8
:1025900045ED017A28460CF1040125DDBAF1000F62
:1025A0000DD004310432D1ED002A92ED003A42EE12
:1025B000C37A01339C428E4645ED017A14DD91EDDC
:1025C000011AD2ED011A41EE617A023340ED017A2F
:1025D00091ED020AD2ED020A40EE607A083108322B
:1025E0009C4240ED017AEADC98ED002AC7EE827A3F
:1025F000013EDDF804A009EB0700043D043F731C15
:10260000D044DC44C0ED007AACD10299069B03981B
:10261000CA18059B029201308342039085DC0BB0FF
:10262000BDE8F08F55ED017ADEE700BF08B50EF08A
:10263000D5FC04F0B9FE0FF0C7FD07F005F913F063
:10264000D5F805F093FD04F053FD09F011FE07F0F5
:1026500097FC08F063F80CF073FF0EF071FA06F0C7
:1026600037F907F0BFFE0BF00FFB13F06DFF08F01A
:1026700093FE0EF091FF08F0E3F913F077F84FF6B0
:10268000AC50C0F6010000F02FF940F22C73C2F2FA
:1026900000034CF6FF12C3F69A321A60BDE80840F8
:1026A00017F0CAB840F68403C2F20003586D10F068
:1026B000D1BF00BF2DE9F047D743154687EA07127F
:1026C000D4B240F674122609C2F2000286F0FF0866
:1026D00048EA042C96798CEAC40989EA060484EA5B
:1026E00004175FFA87FC4FEA192440F6A81E84EA13
:1026F0001C17C2F2000E87EA0C2888EACC049EF868
:1027000000709EF801E01FFA84FC8CEA070989EA50
:1027100009185FFA88F94FEA1C2484EA191444EA7C
:10272000092888EAC90989EA0E0C8CEA0C14E4B27B
:102730004FEA192888EA141C8CEA042989EAC4089B
:102740001FFA88F484EA000C8CEA0C1982B05FFA54
:1027500089FC240A84EA1C1444EA0C288DF80260DF
:102760000C460136FE218DF801508DF800108DF8D1
:1027700003708DF804E08DF80500967188EACC0CA2
:10278000002D52D094F800E08EEA0C0888EA081276
:10279000D1B24FEA1C2C621C6E1E52FA86F6E04340
:1027A0008CEA1119301849EA012EB24200F00100FA
:1027B0008EEAC10C39D098B112F8018B88EA0C0965
:1027C00089EA091E5FFA8EF84FEA1C2080EA181188
:1027D00081EA082080EAC801B2421FFA81FC24D0B5
:1027E000104692F8019010F8011B81EA0C0282EA6F
:1027F0000211C9B24FEA1C2787EA111C8CEA012298
:1028000082EAC1011FFA81FC89EA0C0E8EEA0E18D9
:102810005FFA88F14FEA1C2282EA111242EA01298A
:10282000421CB24289EAC10CDAD183EA0C0181EA86
:1028300001124FEA1C20D1B280EA111383EA01226F
:1028400082EAC10083B2FE2100205FFA83F84FEADA
:102850001329FFF727FF9DF801100020FFF722FF43
:102860009DF802100020FFF71DFF9DF803100020C7
:10287000FFF718FF9DF804100020FFF713FF9DF8E5
:1028800005100020FFF70EFF15B3002705F1FF33F9
:102890000126E15D384603EA060AFFF703FFB54269
:1028A00016D9BAF1000F06D0A15D38460226FFF70F
:1028B000F9FEB5420CD9A15D01363846FFF7F2FEAC
:1028C000A15D38460136FFF7EDFEB0B28542F2D881
:1028D00000204146FFF7E6FE0020494602B0BDE871
:1028E000F047FFF7DFBE00BF40F68403C2F20003EB
:1028F0000146D87816F054BCF0B540F67413C2F215
:10290000000340F6A81793F806C08CF0950686EAF7
:102910000614E6B23209C2F2000782F02C0197F8E1
:1029200000E07F7841EA062585EAC60181EA0E04C7
:1029300084EA0412D2B20D0A85EA121686EA02244B
:1029400084EAC2018CB284EA070585EA0516220AE8
:10295000F5B282EA151141EA052686EAC5052E265A
:1029600085EA060484EA0412D2B2290A81EA121422
:1029700084EA022585EAC20189B281EA000484EA78
:1029800004150246EDB2080A80EA151444EA05214E
:1029900081EAC50585EA122080EA0014E4B2290A1A
:1029A00081EA141080EA042585EAC4018CB284F01F
:1029B0000B0085B080EA0015EDB2210A81EA1510FE
:1029C0008DF806C00CF1010C83F806C040EA05241E
:1029D000FE210020ADF80C2002228DF805208DF894
:1029E00007E08DF808708DF80960FFF75BFE9DF831
:1029F00005100020FFF756FE9DF806100020FFF797
:102A000051FE9DF807100020FFF74CFE9DF80810BE
:102A10000020FFF747FE9DF809100020FFF742FE57
:102A20009DF80C100020FFF73DFE84EAC5049DF8D8
:102A30000D100020FFF736FEE1B20020FFF732FE56
:102A4000210A002005B0BDE8F040FFF72BBE00BF13
:102A5000F0B540F67413C2F2000340F6A81793F8DD
:102A600006C08CF0950686EA0614E6B23209C2F278
:102A7000000782F02C0197F800E07F7841EA0625F4
:102A800085EAC60181EA0E0484EA0412D2B20D0A74
:102A900085EA121686EA022484EAC2018CB284EA2C
:102AA000070585EA0516220AF5B282EA151141EA00
:102AB000052686EAC5052A2685EA060484EA041264
:102AC000D2B2290A81EA121484EA022585EAC201F7
:102AD00089B281EA000484EA04150246EDB2080ACC
:102AE00080EA151444EA052181EAC50585EA122029
:102AF00080EA0014E4B2290A81EA141080EA04256D
:102B000085EAC4018CB284F01C0085B080EA00150F
:102B1000EDB2210A81EA15108DF806C00CF1010C06
:102B200083F806C040EA0524FE210020ADF80C2001
:102B300002228DF805208DF807E08DF808708DF8D9
:102B40000960FFF7AFFD9DF805100020FFF7AAFD13
:102B50009DF806100020FFF7A5FD9DF80710002046
:102B6000FFF7A0FD9DF808100020FFF79BFD9DF8E2
:102B700009100020FFF796FD9DF80C100020FFF7CC
:102B800091FD84EAC5049DF80D100020FFF78AFD31
:102B9000E1B20020FFF786FD210A002005B0BDE864
:102BA000F040FFF77FBD00BF2DE9F04F4FF44062CA
:102BB00040F6B010C4F20002C2F20000546A03688A
:102BC0009C42DDB0C0F0E58140F68405C2F200050C
:102BD00012F0EEFDA87816F0EBF84AF6144CC1F2AC
:102BE000000C03269CF8BC3185F8D660402113F018
:102BF000480F85F8D41000F08481052385F8D6307D
:102C00004AF2A82EC1F2000E9EF838556A1E032A19
:102C10000FD8DFE812F0B301A80104009D0140F6CF
:102C20008403C2F2000393F8D40040F0180683F83E
:102C3000D4604AF6144CC1F2000C9CF8BC219307F6
:102C400009D540F6840EC2F2000E9EF8D41061F051
:102C50007F058EF8D45040F68406C2F20006B36DAC
:102C60009C4200F2A381736E002B00F0518140F66C
:102C7000840EC2F2000EDEF89C108C4200F24484F6
:102C8000002B00F0498140F6840CC2F2000CDCF805
:102C9000B000844201F20682002B00F0468140F62B
:102CA0008405C2F20005D5F8A400844201F2338401
:102CB000002B00F0438140F68405C2F20005D5F8F0
:102CC000A8108C4200F20A8740F6840EC2F2000E71
:102CD0005BA903319EF8030016F036FA9DF86F31B8
:102CE0000146002B40F0DD808DF834300DF13500C9
:102CF0003222002901F0E1871BF0E4FA40F6741C4F
:102D0000C2F2000C40F6A8169CF8060080F09F0363
:102D100083EA0315EBB21F09C2F2000687F00C012B
:102D200041EA0322377876788DF8620182EAC3059A
:102D300085EA070E8EEA0E185FFA88F3290A81EAFF
:102D4000131A8AEA032989EAC30295B285EA060EB4
:102D50008EEA0E185FFA88F3290A81EA131545EA0C
:102D6000032A8AEAC303FD2583EA050989EA0912D1
:102D70005FFA82FE190A81EA1E1282EA0E28FE23F9
:102D800033210DF13409013088EACE0A8DF8603123
:102D90008DF864618DF861118DF863718DF865515E
:102DA0008CF806001FFA8AF209EB01064B46994699
:102DB000170A19F8010B93F8018099F8019080EA3D
:102DC000020C8CEA0C1E5FFA8EF187EA111545EAB7
:102DD000012787EAC10088EA000A8AEA0A12D2B209
:102DE000050A85EA121747EA022181EAC20789EA41
:102DF000070080EA0015E8B2390A81EA101C0333A3
:102E00004CEA0022B34282EAC002D0D182F05306DB
:102E100086EA0610C1B2170A87EA111585EA01226F
:102E200082EAC1030020FE219EB2FFF73BFC9DF821
:102E300061110020FFF736FC9DF862110020FFF7BA
:102E400031FC9DF863110020FFF72CFC9DF8641104
:102E50000020FFF727FC9DF865110020FFF722FCFA
:102E60005FFA86FA4FEA16290DF133050DF166086F
:102E7000002669783046FFF715FCA9783046FFF741
:102E800011FC6F1C15F8031F3046FFF70BFC45457E
:102E9000EFD100205146FFF705FC00204946FFF71F
:102EA00001FC40F68403C2F200031A6ED3F8CC0092
:102EB000824203D2DB6D9C4201F2228240F68405FD
:102EC000C2F2000595F8DA1095F8D930994204D28B
:102ED000D5F8DC20944201F20E86994201F011806F
:102EE00012F06EFC40F68401C2F20001887815F001
:102EF000D9FF40F6B013C2F200031C605DB0BDE81C
:102F0000F08F5A077FF57CAE042085F8D60077E66F
:102F1000B26E002A7FF4ABAE40F6840EC2F2000E11
:102F2000DEF87C1000297FF4AEAE40F6840EC2F2CB
:102F3000000EDEF87020002A7FF4B1AE40F6840E59
:102F4000C2F2000EDEF8740000283FF4BDAEB2E617
:102F500040F6840EC2F2000E9EF8D41041F0140523
:102F60008EF8D45065E640F6840CC2F2000C9CF852
:102F7000D42042F011008CF8D4005AE640F68406C2
:102F8000C2F2000696F8D43043F0100186F8D4104F
:102F90004FE640F68405C2F20005002105F19800D5
:102FA000A965E96534221BF0ABF90DE640F674180B
:102FB000C2F2000840F6A81798F8063096F8D550E7
:102FC00096F8D410559583F0460B8BEA0B1C5FFAEC
:102FD0008CF2C2F20007100980F0920E97F8009070
:102FE00097F801B0CDF80C904EEA022080EAC20EAC
:102FF0008EEA090282EA02195FFA89F94FEA1E2075
:1030000080EA191282EA092080EAC90290B280EAB5
:103010000B09CDF810B089EA091B5FFA8BF24FEA71
:10302000102E8EEA121040EA022989EAC20E8EEAB8
:103030000E1B5FFA8BF24FEA1E2080EA121080EA24
:10304000022080EAC2091FFA89F0454085EA051B83
:103050005FFA8BF94FEA102E8EEA191242EA09251F
:1030600085EAC90080EA001B5FFA8BFE050A85EA43
:103070001E1242EA0E2080EACE0585EA05195FFAA3
:1030800089FB280A80EA1B1242EA0B2E8EEACB0546
:1030900085EA05195FFA89FB280A80EA1B1297F86E
:1030A00002C08DF85A1142EA0B2585EACB0080EA6E
:1030B0000C0E8EEA0E195FFA89FB050A85EA1B10D1
:1030C00080EA0B2282EACB0E1FFA8EF04FF0050E3B
:1030D00080EA0E0989EA0915EDB2020A82EA1510A2
:1030E00040EA052B8BEAC50585EA010989EA091240
:1030F000D2B2280A80EA121585EA022196F8D6A0F3
:103100008DF859E181EAC20B1FFA8BF585EA0A09AD
:1031100089EA09105FFA80FB290A81EA1B1242EA58
:103120000B2080EACB094FF0030B89EA0B0585EAF7
:103130000511CDB24FEA192080EA151282EA052165
:1031400081EAC50085B285F0320282EA02195FFA8F
:1031500089F24FEA1521581C81EA1211059041EAC3
:103160000229DDF814E08DF85CB189EAC209092270
:103170000025DDF810B08DF86121039A88F806E08B
:103180002846FE218DF85BA16FF0010A8DF858C129
:103190008DF862318DF863218DF860A18DF864B1EE
:1031A0008DF86551FFF77EFA28469DF86111FFF70B
:1031B00079FA28469DF86211FFF774FA28469DF8BF
:1031C0006311FFF76FFA28469DF86411FFF76AFA5A
:1031D00028469DF86511FFF765FA28469DF85411B9
:1031E000FFF760FA28469DF85511FFF75BFA28466D
:1031F0009DF85611FFF756FA28469DF85711FFF72C
:1032000051FA28469DF85811FFF74CFA28469DF8C8
:103210005911FFF747FA28469DF85A11FFF742FA6D
:1032200028469DF85B11FFF73DFA28469DF85C1192
:10323000FFF738FA5FFA89F12846FFF733FA4FEAC9
:1032400019212846FFF72EFA42F20C2CC2F2000C8C
:10325000DFEDA87ADCF8001098F8062097F801E076
:1032600097F800C0B6F8D070D6F8E0B0049700EE3A
:10327000101AF8EE406A82F0F10326EEA77A83EA8C
:10328000031AC7EE275A5FFA8AF341F6B0501909BC
:10329000C2F2000040F22C77C2F2000781F0E70989
:1032A0000068D7F800A0C6F8E00049EA032181EAE7
:1032B000C30140F22013CBEB0009C1F2000393EDF0
:1032C000412A0AFB09F304EE903A81EA0C07DFED8C
:1032D0008C1AF8EE643A87EA071B9FED874A5FFA7B
:1032E0008BFA0B0A63EEA12A83EA1A1732EE445ACC
:1032F0009FED823A87EA0A2182EEA51A81EACA0383
:103300009FB287EA0E0989EA091B5FFA8BF3390A33
:1033100081EA131747EA032A8AEAC30B01278BEADB
:10332000070989EA09115FFA81FA85EE036A4FEA13
:103330001B2383EA1A1181EA0A2383EACA011FFACE
:1033400081F940F6A411C2F2000189EA0913DBB247
:1033500008604FEA192B8BEA131949EA0329FCEE9E
:10336000C16A62EE210A26EE210ABCEEE07A16EE70
:1033700090AAFDEEC07A16EE901ACAF57A7B17EE87
:10338000100AA6F8D210ADF898B00499ADF89A00DA
:103390004FF6FF7617EE90BA02EB070AADF89C6085
:1033A0006FF001001F26239524952595ADF89E50BA
:1033B000ADF8A010ADF8A250ADF8A450ADF8A650ED
:1033C000ADF8A8508DF86221CDED036A8DED057A38
:1033D000CDED067A8DF8AAB08DF860018DF86161A7
:1033E0000DF1AB058DF863C10DF18D028DF864E12F
:1033F0008DF8657188F806A089EAC30110460E0AA7
:1034000010F8017B92F80180794081EA011C5FFA93
:103410008CF386EA131E4EEA032989EAC30288EA7E
:10342000020787EA0716110AF7B281EA1713421C4E
:1034300043EA0726AA4286EAC701DFD181F07C056C
:1034400085EA0517FAB2090A81EA121686EA02230A
:1034500083EAC20085B2FE210020FFF723F99DF820
:1034600061110020FFF71EF99DF862110020FFF79F
:1034700019F99DF863110020FFF714F95FFA85F937
:103480009DF8641100204FEA15285CADFFF70AF99A
:1034900000269DF865110020FFF704F915F8E41DDA
:1034A00030460DF1AA07FFF7FDF869783046FFF7BF
:1034B000F9F8A97830460235FFF7F4F8BD42F4D1A7
:1034C00000204946FFF7EEF800204146FFF7EAF8F2
:1034D00002EE104ADFED071AB8EE426A40F6840C9D
:1034E00036EE211AC2F2000CFCEEC10ACCED160A2F
:1034F000FFF7EABB00247449CDCC1C419A9949419D
:1035000000007A440AD7233C40F67412C2F200024B
:1035100040F6A8159179399481F0300787EA0713AE
:10352000D8B20609C2F2000586F07A0E4EEA002BE8
:103530002E786D788DF862118BEAC00787EA060A4B
:103540008AEA0A195FFA89F8380A80EA181787EABE
:10355000082383EAC80087B287EA050C40F22013EB
:10356000C1F200038CEA0C1E5FFA8EF04FEA1727B7
:10357000D3F830A1D3F83491D3F83881D3F824C1EB
:10358000D3F828E187EA101BD3F82C710597D3F8FC
:103590003C710397D3F840710497D3F844318DF808
:1035A00063615FED297A4BEA002704EE90AADDED16
:1035B000036A87EAC0079DED047A1A269DED050A85
:1035C00064EEA73A04EE109A00EE908A05EE10CA57
:1035D00005EE90EA87EA060C03EE103A66EEA76A5B
:1035E0008CEA0C1E20EE270A27EE277A5FFA8EF36C
:1035F00024EE272A25EE271A4FEA1720FDEEE32AAC
:1036000060EEA71A23EE273A65EEA70ABDEEE65A4A
:1036100080EA131BFDEEC75AFDEEC03A12EE90AAE7
:1036200015EE100AFDEEC32A8BEA032BBDEEC26A2B
:10363000FDEEE17AFDEEC14ABDEEE04A13EE907A6E
:103640008BEAC30B15EE903AADF8F40016EE109A23
:1036500017EE908A14EE90CA14EE10EA12EE900A59
:103660000131ADF8F270ADF8F630FE271623CDED3E
:10367000035ACDED042AADF8E8A0ADF8EA90ADF814
:10368000EC80ADF8EEC0ADF8F0E0ADF8F8008DF8E4
:1036900060718DF8613191718DF864518DF86561BB
:1036A0001FFA8BF10DF1FA0539AA10460E0A10F82F
:1036B000013B92F801C083EA010989EA09175FFA20
:1036C00087F886EA181343EA082282EAC8078CEAD8
:1036D000070686EA0611CEB23B0A83EA161242EAD0
:1036E0000621421CAA4281EAC601DED1CDB285F094
:1036F000AA0383EA03175FFA87FA0E0A86EA1A1208
:1037000082EA0A2181EACA0085B2FE210020FEF782
:10371000C9FF9DF861110020FEF7C4FF9DF86211FA
:103720000020FEF7BFFF9DF863110020FEF7BAFFEF
:103730009DF864110020FEF7B5FF9DF8651100208B
:10374000FEF7B0FF5FFA85F94FEA15280DF1E40B9B
:103750000DF1E3050DF1F907002669783046FEF713
:10376000A1FFA97830460235FEF79CFFBD42F4D197
:1037700000204946FEF796FF00204146FEF792FFE3
:1037800040F67413C2F2000340F6A81C93F80680BA
:10379000519488F0F90585EA0512D6B23009C2F2D3
:1037A000000C80F0E60141EA062A9CF800009CF833
:1037B00001E08DF863018AEAC60585EA000989EA15
:1037C00009175FFA87FC290A81EA1C1686EA0C228F
:1037D00082EACC0A1FFA8AF181EA0E0787EA071506
:1037E0005FFA85F90E0A86EA191242EA092787EA82
:1037F000C9051D2785EA070C8CEA0C1A5FFA8AF9BD
:10380000290A81EA191686EA092282EAC90C1FFAF6
:103810008CF181EA040A8AEA0A155FFA85F90E0A30
:1038200086EA191242EA092585EAC90585EA1421C2
:1038300081EA0116F6B22A0A82EA161141EA062C3A
:103840008CEAC60585EA144A8AEA0A195FFA89F100
:103850002A0A82EA111640F22012C1F20002D2EDC9
:10386000457A5FEDD83A46EA012585EAC10967EE57
:10387000A32A89EA146C8CEA0C1ACDED522A5FFA5D
:103880008AF14FEA192686EA111545EA012A9DF8C0
:1038900048919DF849C19DF84A619DF84B518DF8BA
:1038A00062818AEAC10080EA090181EA0111C9B294
:1038B000000A80EA111040EA012080EAC10080EA93
:1038C0000C0181EA011C5FFA8CFC000A80EA1C11E1
:1038D00041EA0C2080EACC0080EA060181EA011C62
:1038E0005FFA8CF1060A86EA111040EA012686EAA0
:1038F000C10080EA050C8CEA0C15E9B2060A86EADA
:10390000111040EA012585EAC10686EA061C5FFA25
:103910008CF1300A80EA111545EA012686EAC100D9
:1039200080EA001C5FFA8CF1050A85EA111646EA66
:10393000012080EAC10585EA051C5FFA8CF12E0A98
:1039400092ED402A9FED636A86EA111040EA012C4D
:1039500062EE061A8CEAC10686EA0615BDEEE11A89
:10396000E9B2320A82EA111040EA012511EE102A6A
:1039700085EAC10080EA020C8CEA0C16F6B2050A50
:1039800085EA161181EA062080EAC605A8B280EA17
:10399000122181EA011C5FFA8CF1060A86EA1115F0
:1039A00045EA012080EAC10585F0730686EA061C17
:1039B0005FFA8CF6290A81EA16104FF0FE0C40EAF5
:1039C000062508F10108614683F80680002085EA93
:1039D000C605ADF8502100260E228DF860C18DF885
:1039E00061218DF864E153968DF86571FEF75AFEFA
:1039F00000209DF86111FEF755FE00209DF8621130
:103A0000FEF750FE9DF863110020FEF74BFE0020EC
:103A10009DF86411FEF746FE00209DF86511FEF743
:103A200041FE00209DF84411FEF73CFE00209DF869
:103A30004511FEF737FE00209DF84611FEF732FED5
:103A400000209DF84711FEF72DFE00209DF848113B
:103A5000FEF728FE00209DF84911FEF723FE002006
:103A60009DF84A11FEF71EFE00209DF84B11FEF74F
:103A700019FE00209DF84C11FEF714FE00209DF861
:103A80004D11FEF70FFE00209DF84E11FEF70AFEC5
:103A900000209DF84F11FEF705FE00209DF8501103
:103AA000FEF700FE00209DF85111FEF7FBFDE9B284
:103AB0000020FEF7F7FD290A0020FEF7F3FD40F68F
:103AC000840CC2F2000CDCF868100819CCF89C00D9
:103AD000FFF7FAB80000C84235FA8E3C40F6741A77
:103AE000C2F2000A40F6A8119AF806002B9480F062
:103AF0006A0585EA0513DAB21709C2F2000187F0F8
:103B0000D50686EAC2080F7849788DF8620188EAFE
:103B1000022686EA070B8BEA0B15EDB2320A82EA1F
:103B2000151E8EEAC50383EA0526B2B282EA010CAD
:103B300041F6B85E40F22018C1F200088CEA0C1978
:103B4000C2F2000E5FFA89F6130AD8F824B1D8F849
:103B500028C1D8F82C218DF8637183EA1615DEF898
:103B60003C348DF8641185EAC60585EA062601EE27
:103B7000102A1E2703EE10BAD3ED096A01EE90CA8F
:103B800093ED0A7AD3ED0B4A86EA07050EF58068B5
:103B90000EF581695FED302A85EA0513D8ED030A39
:103BA00071EEC73A31EE644A99ED000A98ED016A68
:103BB00073EE667A5FFA83FB320A82EA1B1620EE06
:103BC000A25A60EE225A26EE222A67EEE21A23EE6D
:103BD000A21A64EE220A86EA0B2585EACB06FE23AA
:103BE0001C2201308DED2C5ACDED2D5A8DED2E2A53
:103BF000CDED2F1A8DED301ACDED310A8DF86031F3
:103C00008DF861218DF865718AF80600B2B232AD87
:103C10002BAB1946160A11F8010B93F8019080EAB4
:103C2000020B8BEA0B12D7B286EA171E4EEA072C5C
:103C30008CEAC70789EA070080EA00135FFA83FA73
:103C40003E0A86EA1A124B1C42EA0A20AB4280EA7C
:103C5000CA02DED182F0270585EA0510160A5FFA4E
:103C600080F886EA181787EA082383EAC8018DB22C
:103C70000020FE21FEF716FD9DF861110020FEF7E1
:103C800011FD9DF862110020FEF70CFD9DF86311F7
:103C90000020FEF707FD9DF864110020FEF702FDED
:103CA0009DF865110020FEF7FDFC5FFA85F94FEAEB
:103CB00015280DF1C7070DF1AB05002669783046D0
:103CC000FEF7F0FCA97830460235FEF7EBFCBD426A
:103CD000F4D149460020FEF7E5FC41460020FEF7FE
:103CE000E1FC40F67412C2F2000240F6A816907988
:103CF0004B9480F0AB0585EA0513D9B20F09C2F2E7
:103D0000000687F0480989EAC108377876788DF887
:103D1000620188EA012585EA070C8CEA0C1B5FFA30
:103D20008BF9290A81EA191A8AEAC90383EA092860
:103D30001FFA88F181EA060C8CEA0C155FFA85FB04
:103D40000B0A83EA1B1585EACB014AF2F013C1F294
:103D5000000381EA0B29242589EA050AB3F842E029
:103D6000B3F846C0B3F83CB0CDF814E08AEA0A11C3
:103D7000C9B24FEA192888EA111AB3F83E90B3F88D
:103D80004080B3F844E0CDF80CC0B3F848C0B3F8B5
:103D90004A30ADF830B18AEA012B8BEAC10BADF89D
:103DA0003291FE21DDF81490DDF80CA0ADF83E3123
:103DB000002301308DF840318DF86011152350A992
:103DC0008DF861318DF865519071ADF83481ADF8A1
:103DD0003691ADF838E1ADF83AA1ADF83CC18DF8B7
:103DE00063718DF864611FFA8BF24D1C4BAB9A46E0
:103DF000170A1AF8010B93F801909AF801B080EABB
:103E0000020686EA06115FFA81FE87EA1E1242EA7E
:103E10000E2080EACE0789EA070888EA08165FFACA
:103E200086FC390A81EA1C1242EA0C2080EACC079F
:103E30008BEA070A8AEA0A16F2B2390A81EA121EE6
:103E400003334EEA0220AB4280EAC202CFD15FFACE
:103E500082F888F0DE0C8CEA0C1B5FFA8BF7100AF4
:103E600080EA171686EA072181EAC7020020FE21B0
:103E700095B2FEF717FC9DF861110020FEF712FCC9
:103E80009DF862110020FEF70DFC9DF863110020E3
:103E9000FEF708FC9DF864110020FEF703FC9DF876
:103EA00065110020FEF7FEFB4AAB5FFA85FA4FEA88
:103EB00015290DF5967BDD1C0DF5A0780026697897
:103EC0003046FEF7EFFBA9783046FEF7EBFB6F1CA0
:103ED00015F8031F3046FEF7E5FB4545EFD10020FE
:103EE0005146FEF7DFFB00204946FEF7DBFB40F6BC
:103EF0008403C2F200035A6F1519C3F8A850FEF7E5
:103F0000E3BE40F67413C2F2000340F6A81C93F817
:103F100006A08AF01C0686EA0612D7B23809C2F259
:103F2000000C80F03D0141EA07299CF800009CF854
:103F300001C08DF86B0189EAC70686EA000E8EEA99
:103F40000E155FFA85F8310A81EA181787EA082208
:103F500082EAC8091FFA89F181EA0C0585EA05168B
:103F60005FFA86FE0F0A87EA1E1242EA0E2585EAEC
:103F7000CE064FF02F0E86EA0E0888EA08195FFA7F
:103F800089F2310A40F68406C2F2000681EA12176D
:103F900087EA022585EAC20896F8D79096F8D87085
:103FA0008DF86AA11FFA88F089EA000181EA0115FB
:103FB000EDB2020A82EA151141EA052080EAC50144
:103FC00081EA070282EA02185FFA88F20D0A85EA9E
:103FD000121080EA022181EAC2081FFA88F080EA02
:103FE0000015EDB2010A81EA151242EA052080EAC5
:103FF000C505E9B281F0990282EA02185FFA88F2F7
:104000004FEA152080EA1211002541EA02280AF140
:10401000010A83F806A088EAC20828460322FE2186
:104020008DF869218DF86CC18DF86DE18DF86171A5
:104030008DF86251FEF736FB9DF869112846FEF7B0
:1040400031FB9DF86A112846FEF72CFB9DF86B1199
:104050002846FEF727FB9DF86C112846FEF722FB49
:104060009DF86D112846FEF71DFB28464946FEF7D0
:1040700019FB28463946FEF715FB28462946FEF768
:1040800011FB5FFA88F12846FEF70CFB4FEA182176
:104090002846FEF707FB96F8DA20531C86F8DA303C
:1040A000FEF71EBF41F26805C1F2000591A3D3E9F6
:1040B0000023D5E90E0118F0BDF917F0BBFF4AF255
:1040C000A826C1F200068BA3D3E9002396F83B751E
:1040D0000646D5E9100118F0ADF917F0ABFF40F630
:1040E0007412C2F2000240F6A81392F806E01D9086
:1040F0008EF0780181EA0111C9B2C2F200034FEAE1
:10410000111C8CF0F60C93F8018093F800901C962B
:104110004CEA012383EAC10181EA090383EA03131C
:10412000DBB2090A81EA131181EA032181EAC303A0
:1041300099B281EA080383EA0313DBB2090A81EA30
:10414000131141EA0321D5ED125A4FF0180C81EA00
:10415000C303DFED677A95ED1D6A83EA0C01D5EDA7
:104160001E6A95ED187A65EEA75A81EA0111D5ED20
:10417000197AC9B21B0ABCEEC66A83EA1115FCEEB5
:10418000E66ABCEEC77AFCEEE77A1AAB85EA01254F
:104190004FF0000B16EE100A85EAC101CDF86CB0A5
:1041A0001D4616EE906AFE23FDEEE55A17EE10AAA4
:1041B00017EE90BA8DF862E1ADF87C008DF86031B1
:1041C0000EF1010E1E23FF20ADF87E608DF86131E7
:1041D0008DED036ACDED046A8DED057ACDED067A9D
:1041E0001A94CDED1E5AADF880A0ADF882B08DF8CE
:1041F00084708DF885000DF186068DF863912B464D
:1042000082F806E08DF864818DF865C18AB219469E
:1042100093F8019011F8010B80EA0203170A83EA70
:104220000312D0B287EA101C4CEA002E8EEAC003BB
:1042300089EA030888EA0817FFB2180A80EA171308
:1042400043EA07224B1CB34282EAC702DFD182F065
:10425000180686EA0610130A5FFA80F983EA191233
:1042600082EA092787EAC9018EB20020FE21FEF703
:1042700019FA9DF861110020FEF714FA9DF86211F9
:104280000020FEF70FFA9DF863110020FEF70AFAEE
:104290009DF864110020FEF705FA9DF865110020D5
:1042A000FEF700FA5FFA86F94FEA16281D350DF180
:1042B0006706002771783846FEF7F4F9B17838467A
:1042C0000236FEF7EFF9AE42F4D100204946FEF780
:1042D000E9F941460020FEF7E5F940F6840CC2F208
:1042E000000CDCF87C100D19CCF8B050FEF7ECBCDB
:1042F00000007A4400000000D012634100409C4658
:1043000040F2AC2940F2000EC1F2000909EB820C28
:10431000C2F2000EDCF800805EF82210ADF8CE206C
:104320000922ADF8CC008DF8E020CDF8C88034A883
:104330001022002900F0C58419F0C4FF40F6741360
:10434000C2F2000340F6A816987980F0C70E8EEAF4
:104350000E15E9B20A09C2F2000682F0820796F849
:1043600000E076788DF8620147EA012C8CEAC105FD
:1043700085EA0E0888EA08195FFA89F22F0A87EAA7
:10438000121181EA022585EAC20C1FFA8CF787EA2E
:10439000060888EA08195FFA89F2390A81EA1215D3
:1043A00045EA022787EAC201162581EA050C8CEA54
:1043B0000C185FFA88F20F0A87EA12115CAF81EAE3
:1043C000022989EAC20C17F8A88D8DF863E11FFA5B
:1043D0008CF288EA020181EA01195FFA89F1120A76
:1043E00082EA111C01304CEA01224FF0FE0E4FF020
:1043F00019088DF8655198718DF860E18DF861812B
:104400008DF864610DF1E1050DF1C90382EAC10285
:10441000194693F8019011F8010B80EA0203160A7D
:1044200083EA03125FFA82F886EA181E4EEA082C25
:104430008CEAC80389EA030080EA0016F6B21A0A79
:1044400082EA161343EA06204B1CAB4280EAC602FE
:10445000DED1D1B281F0DC0585EA0510130A5FFADE
:1044600080F983EA191282EA092686EAC9018DB227
:104470000020FE21FEF716F99DF861110020FEF7DD
:1044800011F99DF862110020FEF70CF99DF86311F7
:104490000020FEF707F95FFA85F99DF86411002006
:1044A0004FEA15285CADFEF7FDF800269DF8651172
:1044B0000020FEF7F7F815F8A81D30461837FEF76C
:1044C000F1F869783046FEF7EDF8A9783046023504
:1044D000FEF7E8F8BD42F4D100204946FEF7E2F8C5
:1044E00000204146FEF7DEF804EE104A40F6840C48
:1044F000F8EE442A1FED7F5AC2F2000C72EE855A84
:10450000DCF86000BCEEE52A431CCCF860308CED92
:10451000172AFEF7E5BC40F67413C2F2000340F21E
:10452000AC2099793F94C1F2000081F0300E8EEA00
:104530000E12D0ED061AD7B2D0ED080A3D09BDEE35
:10454000E14A85F07A06D0ED037A46EA072614EEB2
:1045500010CAFDEEE05A86EAC7064AF6BC17C1F259
:10456000000790ED027AD0ED042A90ED056A90EDF7
:10457000071A90ED090AFDEEE73A15EE900A0CF1E4
:10458000080C083037F81CC0039013EE90AAFDEE1B
:10459000C06A40F6A812C2F20002BDEEC73AADF8FA
:1045A00014C0BDEEE22ADDF80CC0157837F81CC047
:1045B0008DF86211FDEEC64ABDEEC15A0AF1080A35
:1045C00016EE900A37F81AA0ADF80CC013EE10BA28
:1045D000083012EE109A14EE908A15EE10EA04904C
:1045E00097ED0E7A86EA0500DDF810C00AF5806ABC
:1045F0000BF1080B09F1080908F108080EF1080E83
:10460000CDF820A080EA0010BDF80CA037F81CC03F
:1046100037F81BB037F8199037F8188037F81EE0D4
:10462000ADF818C0C0B2370ABCEEC73A87EA101618
:104630000AF580670796BDF814C08DED043A03971C
:10464000BDF81860DDF81CA08DF8635106F5806791
:10465000ADF80E7100270BF5806B8DF8107113EE1D
:10466000107AADF800B1DDF80CB08DF811718AEA5E
:10467000002608F58068FE27DDF820A0ADF8068149
:10468000ADF80CB186EAC00892F801B08DF86071FF
:1046900016278DF861711FFA88F70EF5806EADF858
:1046A00002A187EA0B0AADF80AE18AEA0A1E5FFA5C
:1046B0008EF53E0A86EA151040EA052787EAC50509
:1046C000232085EA00020CF5806CADF808C182EA6F
:1046D000021C5FFA8CFA09F580692E0AADF8049184
:1046E00086EA1A1989EA0A28013188EACA07997103
:1046F0008DF864B18DF86501BAB20DF589753FABDF
:104700001946100A11F8016B93F8019086EA020E1F
:104710008EEA0E12D7B280EA171B4BEA072A8AEA02
:10472000C70689EA060888EA081C5FFA8CF7300A8F
:1047300080EA171343EA07264B1CAB4286EAC702FE
:10474000DED1D5B285F0F40181EA0116120AF7B282
:1047500082EA171C8CEA072080EAC703FE210020AA
:104760009DB2FDF79FFF9DF861110020FDF79AFFB4
:104770009DF862110020FDF795FF9DF86311002060
:10478000FDF790FF9DF864110020FDF78BFF9DF869
:1047900065110020FDF786FF3FA95FFA85F94FEA12
:1047A000152801F115070DF1FB0500266978304643
:1047B000FDF778FFA97830460235FDF773FFBD425B
:1047C000F4D149460020FDF76DFF41460020FDF77A
:1047D00069FF40F67412C2F2000240F2AC219079F7
:1047E0004594C1F2000180F0300791ED020A87EA9A
:1047F000071391ED037AD1ED047AD1ED052A91EDFD
:10480000066A91ED072AD1ED081A91ED091A40F6D2
:10481000A811DDB2C2F200014FEA151991F800B0FB
:104820008DF86201FDEEE73AFDEEC15A89F07A0992
:10483000FDEEC06A49EA0529BDEEC73ACDF810B0D1
:1048400013EE90CA89EAC50B15EE909A16EE906A9F
:1048500013EE108AFDEEE24ABDEEC64ABDEEC25A24
:10486000FDEEE10ACDF80CB04AF6BC130CF1080BD2
:1048700009F1080CC1F20003CDF814C0DDF8109066
:10488000DDF80CC006F1080A08F1080814EE90EAF9
:1048900014EE107A15EE106A10EE905A33F81AA042
:1048A0008CEA090C0EF1080E33F8189033F81B80CF
:1048B000DDF814B0CDF818C00837083605F1080542
:1048C00033F81EC033F817E033F8167033F815606C
:1048D00033F81B50DDF818B093ED0E0A0AEB4A03CB
:1048E0000AEB830A039B1B0A029309EB4903039318
:1048F00008EB480305930CEB4C0306930EEB4E03B9
:104900000793AAF5185A07EB47030893AAF1160A6A
:1049100006EB46030993CDF804A005EB4503DDF84B
:104920000CA00A938BEA0B1B029B5FFA8BFB09EB33
:104930008A09DDF818A0ADF81A9183EA1B130293D7
:104940000CEB8A0C059BDDF820A0DDF81090ADF88B
:104950001EC108EB830807EB8A07079BDDF828A038
:10496000ADF82271FCEEC06A0EEB830E05EB8A05F2
:10497000099BDDF808A0ADF8265116EE905A06EB1B
:10498000830600278AEA0B238DF828718DF82951B8
:10499000162783EACB058DF8639191F80190ADF865
:1049A00024618DF86171FE26AFB28DF8606187EAEF
:1049B000090686EA0611CEB23B0A83EA1615ADF85F
:1049C00020E145EA062E8EEAC6072225ADF81C81B5
:1049D00087EA050888EA081C5FFA8CFE390A81EA32
:1049E0001E16DDF804A08DF8649186EA0E2383EA92
:1049F000CE08471CCDED0B6AADF818A145AB8DF87C
:104A0000655197710DF595751FFA88F2194693F85F
:104A1000018011F8010B80EA020787EA0713D8B278
:104A2000160A86EA101242EA002989EAC00788EAD3
:104A3000070C8CEA0C1E5FFA8EF23B0A83EA121610
:104A40004B1C46EA0220AB4280EAC202DED1D6B25B
:104A500086F0ED0585EA05115FFA81FE100A80EA0D
:104A60001E1787EA0E2383EACE06B2B20020FE218B
:104A70005FFA82F94FEA1228FDF714FE9DF86111E2
:104A80000020FDF70FFE9DF862110020FDF70AFEE1
:104A90009DF863110020FDF705FE9DF864110020CC
:104AA000FDF700FE9DF865110020FDF7FBFD44AD0C
:104AB00045A9033501F11507002669783046FDF751
:104AC000F1FDA97830460235FDF7ECFDBD42F4D189
:104AD00000204946FDF7E6FD00204146FDF7E2FDD6
:104AE00040F6840CC2F2000CDCF870301A19CCF8D5
:104AF000A420FEF7E9B840F67413C2F2000340F6B2
:104B0000A81C9A79ADF8681182F0A30E8EEA0E18EF
:104B10005FFA88F74FEA1710C2F2000C80F04906DE
:104B20009CF800809CF801C095F8D7A095F8D89023
:104B30008DF86AA146EA072080EAC70787EA080ECF
:104B40008EEA0E16F6B23F0A87EA161080EA0627AA
:104B500087EAC60087B287EA0C0E8EEA0E16F6B216
:104B6000380A80EA161747EA062E8EEAC6074FF083
:104B7000280E87EA0E0080EA0016F6B23F0A87EA9E
:104B8000161080EA062787EAC60080B280EA01078D
:104B900087EA0716F6B2010A81EA161747EA0620E5
:104BA00080EAC60787EA0711C9B23E0A86EA1110F1
:104BB00040EA012787EAC10080EA0A0686EA061A67
:104BC0005FFA8AF6070A87EA161181EA062080EA68
:104BD000C607BEB286EA090181EA011A5FFA8AF1C4
:104BE000300A80EA111747EA012686EAC106F0B2C8
:104BF00080F0E60787EA071A5FFA8AF7310A81EA46
:104C0000171002F1010A40EA072683F806A00020E7
:104C1000FE2186EAC70604278DF862218DF864C15B
:104C20008DF865E18DF86B918DF861718DF8638178
:104C3000FDF738FD00209DF86111FDF733FD0020E0
:104C40009DF86211FDF72EFD00209DF86311FDF720
:104C500029FD00209DF86411FDF724FD00209DF83A
:104C60006511FDF71FFD00209DF86811FDF71AFD85
:104C700000209DF86911FDF715FD00209DF86A11CF
:104C8000FDF710FD00209DF86B11FDF70BFDF1B253
:104C90000020FDF707FD310A0020FDF703FD00EEBF
:104CA000904A9FED0A6AB8EE600A70EE067AFCEE52
:104CB000E73AC5ED373AFEF713B919F021FBFEF7D5
:104CC0001DB819F01DFBFFF739BB00BF0024744964
:104CD0002DE9F041858C042D84B000F0F080F52D95
:104CE00000F0BF80042440F67413C2F2000340F6C3
:104CF000A81E9A79ADF80C5082F01C0888EA081CAE
:104D00005FFA8CF00709C2F2000E87F03D069EF8AC
:104D100000C09EF801E08DF8062046EA002181EAF5
:104D2000C00686EA0C0888EA0817FFB2300A80EA53
:104D3000171686EA072181EAC70087B287EA0E06BE
:104D400086EA0611CEB2380A80EA161848EA062723
:104D500087EAC6004D2780EA070181EA0116F6B20C
:104D6000000A80EA161888EA062181EAC60086B29F
:104D700086EA050181EA01185FFA88F1300A80EAC3
:104D8000111646EA012080EAC10080EA152888EA67
:104D90000816F6B2010A81EA161545EA062080EAED
:104DA000C60585EA040181EA01185FFA88F1280A3C
:104DB00080EA111646EA012585EAC105E8B280F0CD
:104DC0008F0686EA06185FFA88F6290A81EA161025
:104DD00002F1010840EA062583F8068085EAC60547
:104DE0000020FE2103268DF807C08DF808E08DF81D
:104DF0000E408DF805608DF80970FDF753FC9DF8A5
:104E000005100020FDF74EFC9DF806100020FDF770
:104E100049FC9DF807100020FDF744FC9DF80810A0
:104E20000020FDF73FFC9DF809100020FDF73AFC3B
:104E30009DF80C100020FDF735FC9DF80D100020AA
:104E4000FDF730FC00202146FDF72CFCE9B20020E4
:104E5000FDF728FC290A002004B0BDE8F041FDF769
:104E600021BC4AF61441C1F2000191F8BC3113F0A3
:104E7000040330D1D0ED027AF5EE407AF1EE10FA6B
:104E80002BD0B7EE007AF4EE477AF1EE10FA30D07C
:104E9000B0EE000AF4EE407AF1EE10FA21D0F0EE16
:104EA000080AF4EE607AF1EE10FA7FF41BAF1846B0
:104EB00003F0C0F90028ACBF0124042413E740F636
:104EC000FC54C2F20004204605F0A0FD2046FDF788
:104ED0000BFD012407E7022405E703F081F8012414
:104EE00001E7184603F098F80028ACBF0124042419
:104EF000F9E603F083F80124F5E600BF2DE9F04F51
:104F00002DED048B40F68403F1B0C2F200034FF69E
:104F1000D050C0F6010060AF0DF5CC789FEDBE9A81
:104F2000DFEDBE8A5D6DFDF7DFFC0397CDF80880ED
:104F3000052014F0FFFC4AF61444C1F20004284690
:104F40000EF0A0FB0028F3D028460EF0A9FB40F697
:104F50007412C2F200020026D1781670C3B2092979
:104F60002CD8DFE811F018011801F6003001B80064
:104F7000D7000A008F005D003E0040F6B818C2F26C
:104F80000008B8F8000088F8073083EA000B8BEAC5
:104F90000B12D3B2070A87EA131141EA032A98F8E1
:104FA00003608AEAC30940F67413A8F80090C2F2BD
:104FB0000003002E40F026810826DE7040F67418AB
:104FC000C2F20008002298F8026088F8022040F639
:104FD0008403C2F20003B3F8D070F619A3F8D060CE
:104FE000ADE740F6B816C2F200063188B3EB112FD8
:104FF00000F0168140F67412C2F20002012092F80D
:105000000280D07008EB0007FE2B9770D6D10221EA
:1050100000234FF6FF79D170F370A6F80090CDE72A
:1050200040F6B812C2F200024FF6086BD179108830
:10503000C0F6010B1BF801A08AEA000989EA0916EB
:10504000F7B2000A80EA171848EA072E8EEAC7016D
:10505000CEB21180B34240F67411C2F2000100F0EA
:10506000D48091F802C001200CEB0007FE2BC87021
:105070008F70A3D1022700264FF6FF73CF70D67032
:1050800013809BE740F67411C2F2000140F6B81E8F
:105090000F79C2F2000E0EEB070C01378CF80830C6
:1050A000BEF800009EF803C083EA000B8BEA0B1ADF
:1050B0005FFA8AF9060A86EA1912F8B242EA092367
:1050C00083EAC90884450871AEF800807FF476AFA2
:1050D0000823CB7072E740F6B81CC2F2000C40F611
:1050E000741BBCF800208CF8043083EA020989EABA
:1050F00009185FFA88F6100A80EA161E4EEA06279B
:10510000C2F2000B87EAC6010323ACF800108BF84B
:10511000033053E740F6B81AC2F2000A40F6741999
:10512000BAF800208AF8063083EA020E8EEA0E1CD6
:105130005FFA8CF6100A80EA161B4BEA0627C2F2C9
:10514000000987EAC6010623AAF8001089F803308F
:1051500034E740F6B81CC2F2000C40F6741BBCF8F1
:1051600000208CF8033083EA020A8AEA0A195FFAFF
:1051700089F7100A80EA1718C2F2000B48EA072ED6
:105180008EEAC701002604238BF80460ACF80010F7
:105190008BF8033012E7FE2B7FF410AF40F6741A41
:1051A00040F6B819C2F20009C2F2000A0222002732
:1051B0004FF6FF708AF8032089F8037089F80230EF
:1051C000A9F80000FAE640F6B81BC2F2000B40F660
:1051D000741ABBF800208BF8053083EA020888EACD
:1051E000081E5FFA8EF6100A80EA161C4CEA0627A3
:1051F000C2F2000A87EAC6010523ABF800108AF85C
:105200000330DBE60721D970D8E691F804E0724458
:105210000920C8701372D1E60024744900007A4452
:1052200040F67417C2F200074FF0010B3A7987F885
:1052300000B006EB020A0AA88AF8093031464FF49A
:10524000887287F803B019F03DF83B78012B41F0E4
:10525000968536793A897E7102B97A8140F6741C56
:10526000C2F2000C501C00279CF80260ACF8080049
:105270008CF8027040F6840EC2F2000E9EF8020016
:1052800013F096FD9DF82F20531F472B74D8DFE8AD
:1052900013F0AC08730073007300730073005204C2
:1052A0007300730073007300730073007300730066
:1052B000E80635037300F80773007300730073008A
:1052C0007300730073007300730073007300730046
:1052D00073007300730053037F05180373001F02EC
:1052E0009200770173007300730073007300730002
:1052F0007300730073007300730073007300730016
:105300007300730073007300730073004800730030
:1053100073007300730073007300730073007300F5
:105320007C0040F6A818C2F200089DF8321098F8E8
:1053300000708F4220D1BDF830309DF834205F1EC0
:10534000B8B2C62801F26B810C2A01F268819DF87F
:105350003510002901F0638104EE903AB8EEE44A7A
:1053600040F68409C9EE043AC2F2000909EB820A48
:10537000BCEEE33A8AED193A40F6840BC2F2000B18
:105380009BF8020013F08EFD21E640F6A818C2F249
:1053900000089DF84E0098F800708742ECD140F666
:1053A000840BC2F2000B0AA8FFF792FC9BF80200E4
:1053B00013F078FD0BE640F6A819C2F200099DF83B
:1053C000320099F80070B842D6D19DF830A0BAF1F9
:1053D000190F41F238814FF0010840F67413C2F200
:1053E000000340F6A8199A798DF8BC7182F01C0C64
:1053F0008CEA0C1A5FFA8AFB4FEA1B1080F03D0121
:1054000041EA0B2080EACB0080EA070E8EEA0E1CF0
:105410005FFA8CF14FEA1020C2F2000980EA111AFB
:1054200099F801908DF8AE214AEA012B8BEAC10070
:1054300080EA090E8EEA0E1C5FFA8CF1000A80EAFF
:10544000111A4AEA012B8BEAC1004FF02F0B80EAB8
:105450000B0E8EEA0E1C5FFA8CF1000A80EA111A1C
:105460008AEA012080EAC10E1FFA8EF087EA000C5A
:105470008CEA0C1A5FFA8AF1000A80EA111040EAFD
:10548000012E8EEAC10080EA090C8CEA0C1A5FFA40
:105490008AFC000A80EA1C1E8EEA0C2181EACC00FC
:1054A00080B280EA080A8AEA0A115FFA81FA000AE1
:1054B00080EA1A1E4EEA0A2C8CEACA00C1B281F0B8
:1054C000990181EA01115FFA81FE010A81EA1E1148
:1054D000501C4FF0FE0A059041EA0E2C8CEACE0ECD
:1054E00051468DF8ACA1059A8DF8BE814FF0030AA4
:1054F0000020CDF810E08DF8BD918DF8ADA18DF8AC
:10550000AF718DF8B0918DF8B1B19A71FDF7CAF80D
:105510009DF8AD110020FDF7C5F89DF8AE110020F3
:10552000FDF7C0F89DF8AF110020FDF7BBF89DF81E
:10553000B0110020FDF7B6F89DF8B1110020FDF77D
:10554000B1F839460020FDF7ADF849460020FDF7D7
:10555000A9F841460020FDF7A5F8049F0020F9B204
:10556000FDF7A0F840F6840B049BC2F2000B00206C
:10557000190AFDF797F89BF8020013F093FC26E553
:1055800040F6A819C2F200099DF8307099F8003071
:105590009F427FF4F1AE08F063FC40F67413C2F250
:1055A000000380469A7999F801C099F800B0CDF8C7
:1055B00014C082F01C0181EA011A5FFA8AF108091D
:1055C00080F03D0989EAC10080EA012080EA0B0AE7
:1055D0008AEA0A195FFA89FA000A80EA1A1181EA4E
:1055E000CA0080EA0A2188B280EA0C0A8AEA0A1C08
:1055F0005FFA8CF1000A80EA111080EAC10989EA99
:10560000012080F02F0A8AEA0A1C5FFA8CF9000A4E
:1056100080EA191181EA092080EAC90188B287EA83
:10562000000A8AEA0A1C5FFA8CF1000A80EA111962
:1056300089EAC10080EA01204FF0BE0980EA090A28
:105640008AEA0A1C5FFA8CFA000A80EA1A1181EAD7
:10565000CA0080EA0A2188B280EA080C8CEA0C1A97
:105660005FFA8AFA010A81EA1A1040EA0A2C8CEAE7
:10567000CA00C1B281F0990181EA01115FFA81FE8D
:10568000010A81EA1E11501C8DF8AE21059A069080
:105690004FF0FE0A41EA0E2C8CEACE0C51468DF8F2
:1056A000ACA18DF8B0214FF0030A4FF02F028DF816
:1056B000B1218DF8BC710020CDF810C08DF8BD91DE
:1056C0008DF8BE818DF8ADA18DF8AFB1069A1CE7BB
:1056D00040F6A818C2F200089DF8302098F800B0F3
:1056E00093457FF449AE9DF82D709DF82EB008F0DB
:1056F0009DFB40F67413C2F2000398F800C09A793B
:1057000098F801A0ADF8AC0182F0A30181EA01197B
:105710005FFA89F14FEA111888F0490E4EEA012923
:1057200089EAC10E8EEA0C0888EA0811C9B24FEA6C
:105730001E2989EA111888EA012E8EEAC1091FFA8A
:1057400089FE8EEA0A0888EA0811C9B24FEA1E29C2
:1057500089EA111848EA012E8EEAC10E8EF02C0952
:1057600089EA09185FFA88F94FEA1E2181EA1911BE
:1057700081EA092181EAC9011FFA81F989EA000851
:1057800088EA081E5FFA8EF84FEA192181EA18119B
:1057900041EA082E8EEAC80989EA102080EA001141
:1057A000C9B24FEA192888EA111E8EEA012080EA60
:1057B000C1091FFA89F080EA070888EA081E5FFA23
:1057C0008EF1000A80EA111040EA012989EAC1003D
:1057D00080EA0B0888EA081E5FFA8EF8000A80EA61
:1057E000181989EA082181EAC80080B2C1B281F0A3
:1057F000DD0181EA01115FFA81FE010A501C04906B
:105800008DF8AE7104278DF8B571049F8DF8B6211F
:1058100081EA1E114FF0FE0841EA0E292C229F71E9
:105820004146002089EACE098DF8B7C18DF8B9212B
:105830008DF8AFB18DF8B4818DF8B8A1FCF732FFC7
:105840009DF8B5110020FCF72DFF9DF8B611002042
:10585000FCF728FF9DF8B7110020FCF723FF9DF807
:10586000B8110020FCF71EFF9DF8B9110020FCF7CD
:1058700019FF9DF8AC110020FCF714FF9DF8AD1145
:105880000020FCF70FFF9DF8AE110020FCF70AFF87
:1058900040F6840B9DF8AF110020FCF703FFC2F225
:1058A000000B5FFA89F10020FCF7FCFE00204FEAB4
:1058B0001921FCF7F7FE9BF8020013F0F3FAFFF74B
:1058C00086BB40F6A81BC2F2000B9DF832209BF865
:1058D000008090457FF450ADBDF83030182B3FF676
:1058E0004BAD40F6840BC2F2000BD8B207F02AFA97
:1058F0009BF8020013F0D6FAFFF769BB40F6A81830
:10590000C2F200089DF8302098F8009091457FF48D
:1059100033AD40F6840BC2F2000B0027CBF8607069
:10592000CBF85C7040F6840BC2F2000B9BF80200CF
:1059300013F0B8FAFFF74BBB40F6A818C2F2000804
:105940009DF8502098F80070BA427FF415ADBDF86C
:105950004CB09DF85280BBF1180F07D8B8F1000F7A
:1059600000F01E86B8F1030F00F01A864FF0010810
:1059700040F6741AC2F2000ACDF814A09AF806A0F4
:105980008AF01C0E8EEA0E10C2B2130983F03D019C
:1059900041EA022080EAC20383EA070C8CEA0C1E6B
:1059A00040F6A8195FFA8EF2190AC2F2000981EADC
:1059B000121099F8019040EA022383EAC20181EAB9
:1059C000090C8CEA0C1E5FFA8EF2080A80EA1213A8
:1059D00043EA022181EAC20080F02F0C8CEA0C1EFF
:1059E0005FFA8EF2030A83EA121181EA022080EA4A
:1059F000C20C1FFA8CF187EA010E8EEA0E135FFAD1
:105A000083FC080A80EA1C1242EA0C2383EACC03D6
:105A100083EA090181EA0110C0B21A0A82EA101170
:105A200081EA002E8EEAC00399B281EA080282EA76
:105A3000021C5FFA8CF3080A80EA131E4EEA032167
:105A400081EAC301CAB240F6840CC2F2000C82F0B3
:105A500099004FF4406280EA0013C4F200020BF197
:105A600001005FFA83FE8CF8DA00080A536A8DF8A9
:105A7000BC7180EA1E1141EA0E22CCF8DC3082EAC9
:105A8000CE0CDDF814E0CDF810C00AF101034FF0A0
:105A9000FE0B03228EF80630594600208DF8AD210A
:105AA0004FF02F028DF8B1218DF8ACB18DF8AF71A8
:105AB0008DF8BD918DF8BE818DF8AEA18DF8B091B5
:105AC000FCF7F0FD9DF8AD110020FCF7EBFD9DF813
:105AD000AE110020FCF7E6FD9DF8AF110020FCF7A9
:105AE000E1FD9DF8B0110020FCF7DCFD9DF8B1113F
:105AF0000020FCF7D7FD39460020FCF7D3FD4946CE
:105B00000020FCF7CFFD41460020FCF7CBFD049FB1
:105B10000020F9B2FCF7C6FD40F6840B049BC2F2EC
:105B2000000B0020190AFCF7BDFD9BF8020013F0E2
:105B3000B9F9FFF74CBA40F6A813C2F200039DF87A
:105B40003420187882427FF417AC40F67411C2F208
:105B5000000193F801C08F799DF835908DF8B671EA
:105B600087F0F10E8EEA0E1A5FFA8AF34FEA1318E5
:105B700088F0E70B4BEA032E8EEAC30B40F22010AD
:105B80008BEA020AC1F20000D0ED411A8AEA0A1833
:105B9000DFED7D2A5FFA88F34FEA1B2080EA131EAF
:105BA00071EEE26A9FED792A4EEA032A8AEAC3007F
:105BB00086EE821A80EA0C0888EA081B5FFA8BFEE0
:105BC000030A83EA1E1080EA0E2383EACE0A1FFA34
:105BD0008AF04FF0010E80EA0E0888EA081B5FFA8F
:105BE0008BFA000A80EA1A1343EA0A2080EACA08FC
:105BF00040F68403C2F2000388EA0810C0B24FEAFC
:105C0000182B21EE280AB3F8D2A0B3F8D08083F87D
:105C1000D49061EEA80A8BEA101383EA002BBDEE44
:105C2000C07A8BEAC00BFCEEE07A4FF6FF700023DF
:105C3000ADF8700117EE100A17EE909A5893599329
:105C40005A93ADF87231ADF87631ADF87831ADF8E0
:105C50007A31ADF87C31FE237744CAF57A7A8DF833
:105C60007E018DF8B4311F205FAB8DF8B7218DED2B
:105C7000047A58AA8F71ADF86CA1DF1CADF86E9153
:105C8000ADF874818DF8B5018DF8B8C18DF8B9E122
:105C900001321FFA8BF3114692F801B011F8019B03
:105CA00089EA030C8CEA0C124FEA13205FFA82FA9D
:105CB00080EA1A1E4EEA0A2888EACA028BEA020023
:105CC00080EA00135FFA83FC100A80EA1C1242EAA1
:105CD0000C294A1CBA4289EACC03DCD183F07C004F
:105CE00080EA0011C8B21B0A83EA101787EA002273
:105CF00082EAC0018BB20020FE215FFA83FB4FEAEB
:105D0000132AFCF7CFFC9DF8B5110020FCF7CAFC64
:105D10009DF8B6110020FCF7C5FC9DF8B7110020D6
:105D2000FCF7C0FC9DF8B8110020FCF7BBFC4FF05D
:105D300000089DF8B9110020FCF7B4FC9DF8601133
:105D4000404658AF0DF5BF79FCF7ACFC797840467A
:105D5000FCF7A8FCB97840460237FCF7A3FC4F4596
:105D6000F4D1594640F6840B0020C2F2000BFCF738
:105D700099FC00205146FCF795FC9BF8020013F0BB
:105D800091F8FFF724B900BFCDCC1C419A99494145
:105D900040F6A818C2F200089DF8323098F800705A
:105DA0009F427FF4E9AABDF83070384608F074F8D5
:105DB00090F82C2090F82D90012A0CBF4FF0030B87
:105DC0004FF0000BB9F1010F824600F07385B9F175
:105DD000030F01F06D80B9F1020F01F02480B9F1D9
:105DE000040F00F0D487B9F1050F00F08F869DF8FD
:105DF0002D30816904934AF2A822C1F2000244F6D0
:105E0000D35392F83A25C1F26203A3FB01E39B0945
:105E1000C7EB020EDEF1000207EE103AD0E90001F6
:105E200042EB0E020892B8EE478A16F081F906900E
:105E3000DAE9020116F07CF940F67413C2F20003AD
:105E400098F80090997998F801C08DF8AE1181F01A
:105E5000280282EA0212D2B24FEA121E8EF0790EA6
:105E60004EEA022E8EEAC20E8EEA090282EA02127F
:105E7000D2B24FEA1E2E8EEA121E8EEA022E8EEA51
:105E8000C20E1FFA8EFE8EEA0C0282EA0212D2B213
:105E90004FEA1E2E8EEA121848EA02284FF0270E0B
:105EA00088EAC20888EA0E024FEA1828CDF8248052
:105EB000DAF82480CDF81480DAF81080DAF814A02B
:105EC000CDF81C80CDF838A182EA0212DDF824A0BA
:105ED0005390D2B28AEA121801F1010A88EA02212B
:105EE0004FF000080798CDF84081DDF814805490F9
:105EF000CDF84481ADF85471DDF81880049FCDF8D9
:105F000048811020ADF85601BE208DF8590181EA74
:105F1000C2028DED4F8A8DF858718DF85AB183F811
:105F200006A09DF83831DDF820808DF8AF9192B24F
:105F30005340012083EA0313DBB2120A8DF85C019F
:105F4000FE2082EA13118DF8AC0125208DF8AD01F9
:105F500041EA032157A84EAA8DF85B818DF8B0C1A4
:105F60008DF8B1E10130013281EAC303114692F8A4
:105F700001B011F801CB8CEA030E8EEA0E125FFA23
:105F800082F94FEA132787EA191343EA092787EAB8
:105F9000C9028BEA020888EA081A5FFA8AFC170A23
:105FA00087EA1C1242EA0C234A1C824283EACC0391
:105FB000DCD15FFA83FA8AF0FE0787EA0711CFB2D5
:105FC0001B0A83EA171080EA072282EAC7018BB214
:105FD0000020FE215FFA83FA4FEA1329FCF762FBE7
:105FE0009DF8AD110020FCF75DFB9DF8AE1100207F
:105FF000FCF758FB9DF8AF110020FCF753FB9DF810
:10600000B0110020FCF74EFB9DF8B1110020FCF709
:1060100049FB4FF000084EA807469DF8381140464E
:106020000DF5AE7BFCF73EFB79784046FCF73AFB7A
:10603000B97840460237FCF735FB5F45F4D10020C4
:106040005146FCF72FFB00204946FCF72BFB40F69E
:10605000840BC2F2000B9BF8020012F023FFFEF744
:10606000B6BF40F6A818C2F200089DF8322098F892
:10607000007097427FF480A940F6840BC2F2000BB7
:10608000BDF83030DBF8CC008342BFF675A940F292
:10609000AC2E40F2000CC1F2000E0EEB8301C2F2F6
:1060A000000CD1F800905CF82310ADF8863109237C
:1060B000CDF88091ADF884018DF89831002900F079
:1060C0002D8762A8102218F0FDF840F6741BC2F26A
:1060D000000B40F6A8119BF8060080F0C70888EA7C
:1060E0000817FAB21309C2F2000183F0820991F88D
:1060F000008049788DF8AE0149EA022A8AEAC2078F
:1061000087EA080E8EEA0E1C5FFA8CFA3A0A82EAD7
:106110001A1989EA0A2383EACA07BFB287EA010289
:1061200082EA02135FFA83FC3A0A82EA1C1747EA02
:106130000C2E8EEACC03162783EA070989EA091A8E
:106140005FFA8AFE1B0A83EA1E1260AB82EA0E2CFB
:106150008CEACE0213F8019B8DF8AF811FFA82FC06
:1061600089EA0C0A8AEA0A1E5FFA8EFA4FEA1C22B2
:10617000013082EA1A1242EA0A224FF0FE094FF079
:1061800019088BF8060066A88DF8AC918DF8AD81E2
:106190008DF8B0118DF8B171013082EACA0219464A
:1061A00093F801A011F8017B87EA02034FEA122B52
:1061B00083EA0312D7B28BEA171848EA072989EA5B
:1061C000C7038AEA030E8EEA0E1C5FFA8CFB1F0AD5
:1061D00087EA1B1343EA0B224B1C834282EACB0261
:1061E000DDD15FFA82FA8AF0DC0E8EEA0E115FFAD8
:1061F00081FC100A80EA1C1787EA0C2383EACC0191
:106200008AB20020FE215FFA82FA4FEA1229FCF7D7
:1062100049FA9DF8AD110020FCF744FA9DF8AE1143
:106220000020FCF73FFA9DF8AF110020FCF73AFA86
:106230009DF8B0110020FCF735FA9DF8B11100204F
:10624000FCF730FA4FF0000860A807469DF880116F
:1062500040460DF5CC7BFCF725FA79784046FCF7F3
:1062600021FAB97840460237FCF71CFA5F45F4D1B1
:1062700000205146FCF716FA00204946FCF712FAB6
:10628000E5E640F6A813C2F200039DF834C0187882
:1062900060457FF471A80DF13601102267A818F04F
:1062A00011F840F68401C2F20001D1F8CCE0BEF151
:1062B000000F7FF761A840F20000C2F20000002743
:1062C00050F8042B9DF89C31117899427CD100291B
:1062D00000F0C4819DF89D315178994274D1002914
:1062E00000F0BC819DF89E31917899426CD10029D3
:1062F00000F0B4819DF89F31D178994264D1002992
:1063000000F0AC819DF8A031117999425CD100294F
:1063100000F0A4819DF8A1315179994254D100290E
:1063200000F09C819DF8A231917999424CD10029CD
:1063300000F094819DF8A331D179994244D100298C
:1063400000F08C819DF8A431117A99423CD100294A
:1063500000F084819DF8A531517A994234D1002909
:1063600000F07C819DF8A631917A99422CD10029C8
:1063700000F074819DF8A731D17A994224D1002987
:1063800000F06C819DF8A831117B99421CD1002945
:1063900000F064819DF8A931517B994214D1002904
:1063A00000F05C819DF8AA31917B99420CD10029C3
:1063B00000F054819DF8AB31D17B994204D1002B80
:1063C00000F04C819DF8AC31002B00F04781013783
:1063D00077457FF475AF40F6840BC2F2000B9BF853
:1063E000020012F05FFDFEF7F2BD40F6A811C2F206
:1063F00000019DF8303091F800904B457EF4BCAF21
:1064000040F67412C2F20002497892F806E0049154
:106410008EF01C0989EA0917F9B2080980F03D0BD2
:106420004BEA012787EAC10080EA030181EA011CE7
:106430005FFA8CF7000A80EA171949EA072B0499DA
:106440009DF82D809DF831A08DF8AF318BEAC70003
:1064500080EA010C8CEA0C175FFA87FB010A81EADB
:106460001B1080EA0B2989EACB07B8B280F006013D
:1064700081EA011C5FFA8CF7000A80EA171949EAE1
:10648000072B8BEAC70788EA070181EA011C5FFA3C
:106490008CFB380A80EA1B1949EA0B2787EACB00F4
:1064A00080EA0A0181EA011C5FFA8CF7000A80EA9F
:1064B000171989EA072B8BEAC70188B280EA001C0A
:1064C0005FFA8CF7000A80EA171949EA072B8BEA72
:1064D000C70787F06801049B8DF8AEE181EA0110DF
:1064E0005FFA80FC0EF1010005908DF8B0314FF09D
:1064F0000603390A8DF8B131059B8DF8B481002768
:1065000081EA1C114FF0FE0B41EA0C2993713846C9
:1065100059468DF8ACB14FF0030B89EACC098DF8E0
:10652000ADB18DF8B5A18DF8B671FCF7BBF89DF84B
:10653000AD113846FCF7B6F89DF8AE113846FCF7B9
:10654000B1F89DF8AF113846FCF7ACF89DF8B011E2
:106550003846FCF7A7F89DF8B1113846FCF7A2F8C9
:1065600038464146FCF79EF838465146FCF79AF803
:1065700040F6840B38463946FCF794F8C2F2000B1B
:106580005FFA89F13846FCF78DF838464FEA192151
:10659000FCF788F89BF8020012F084FCFEF717BDA8
:1065A0009DF84E30142B00F02E85102B00F01D8529
:1065B000B32B00F06E81162B00F0B684012B00F097
:1065C000E484152B7FF4D2A9584607F065FC0746F2
:1065D000A8F10300D0F1000848EB0008052310984B
:1065E00087F82C8087F82D3015F086FD02460B4683
:1065F0001198C7E9002315F07FFD129BDDF834E008
:106600003B610F9B0E9ABB62A94BC7F820E0C7E91C
:106610000201FA614FF000081F78FFF7A9B940F6B0
:10662000840EC2F2000E183240F6840B0EEB820C80
:10663000C2F2000B0020CCF804009BF8020012F01C
:1066400031FCFEF7C4BC07F00BFC012800F0798395
:1066500099F800704FF00108FEF7BFBEBE457EF707
:106660008BAE9DED0C8AB0EE480A16F023F9002897
:1066700000F0F98440F68408C2F2000840F2AC2C25
:10668000B8F8CC90ADF88671C1F2000C0CEB870025
:10669000ADF8849140F674190368C2F2000967A945
:1066A0001022092762A860938DF8987117F00AFEEE
:1066B00099F8060080F0C70A8AEA0A11CAB240F6C1
:1066C000A81B1309C2F2000B83F082079BF800A0FD
:1066D0009BF801B08DF8AFA147EA022E8EEAC20105
:1066E00081EA0A0C8CEA0C185FFA88FE0A0A82EA30
:1066F0001E1787EA0E2383EACE0C1FFA8CF787EA6F
:106700000B0181EA01125FFA82F83B0A83EA181151
:1067100041EA082282EAC807162187EA010E8EEABA
:106720000E1C5FFA8CF83B0A83EA181260AB82EA0F
:10673000082787EAC80213F801EB8DF8AE0197B27B
:106740008EEA070C8CEA0C185FFA88FA4FEA1727D2
:1067500087EA1A124FF0FE078DF8AC714FF0190757
:10676000013042EA0A228DF8AD7166AF89F8060061
:106770008DF8B0B18DF8B111781C82EACA021946C1
:1067800093F8018011F8017B87EA020383EA031B77
:106790005FFA8BF74FEA122E8EEA171242EA072CA5
:1067A0008CEAC70388EA030989EA091A5FFA8AF2C0
:1067B0001F0A87EA121B4B1C4BEA022E83428EEA09
:1067C000C202DCD15FFA82FB8BF0DC0E8EEA0E1C7B
:1067D0005FFA8CF0120A82EA101989EA002A8AEA22
:1067E000C0018FB20020FE21FBF75CFF00209DF866
:1067F000AD11FBF757FF00209DF8AE11FBF752FFDC
:1068000000209DF8AF11FBF74DFF00209DF8B0115F
:10681000FBF748FF0DF5BE7800209DF8B111FBF79E
:1068200041FF08F103034FF000086FEA03024046FE
:106830009DF8801102F0010BFBF734FF02985FFA1C
:1068400087F94FEA172A60AF874218D0BBF1000FD3
:1068500009D060AB40469DF881115F1CFBF722FF19
:10686000029887420BD079784046FBF71BFFB97836
:106870004046FBF717FF029B02379F42F3D10020EF
:106880004946FBF70FFF00205146FBF70BFFFEF7D1
:1068900073BD9DF85380B8F1000F00F0FD83044FE5
:1068A00006F0B4F94FF000083F78FFF761B800BF79
:1068B000A809002007F0FAFA9DF82D3081690493A9
:1068C0004AF2A822C1F2000244F6D35392F83A25C4
:1068D000C1F26203A3FB01E39B09C7EB020BDBF1EF
:1068E000000207EE103A42EB0B028246D0E90001AB
:1068F0000892B8EE478A15F01BFC0690DAE902010F
:1069000015F016FC40F67413C2F2000398F800B0BC
:10691000997998F801C08DF8AE1181F0280282EAC9
:106920000212D2B24FEA121E8EF0790E4EEA022EF9
:106930008EEAC20E8EEA0B0282EA0212D2B24FEA4D
:106940001E2E8EEA121E8EEA022E8EEAC20E1FFA4A
:106950008EFE8EEA0C0282EA0212D2B24FEA1E2E9C
:106960008EEA121848EA02284FF0270E88EAC20879
:1069700088EA0E024FEA1828CDF82480DAF824803D
:10698000CDF81480DAF81080DAF814A0CDF81C8065
:10699000CDF838A182EA0212DDF824A05390D2B2D9
:1069A0008AEA12180798ADF8547101F1010A88EAD1
:1069B00002214FF00008CDF84081DDF8148054909A
:1069C0001420CDF84481ADF85601DDF81880049FFD
:1069D000CDF84881BE208DF85901002081EAC2021D
:1069E0008DED4F8A8DF858718DF85A0183F806A005
:1069F0009DF83831DDF820808DF85C9192B25340DB
:106A000083EA0313DBB2FE20120A82EA13118DF827
:106A1000AC0125208DF8AD0141EA032157A84EAA0B
:106A20008DF85B818DF8AFB18DF8B0C18DF8B1E113
:106A30000130013281EAC303114692F801A011F836
:106A400001EB8EEA030B8BEA0B124FEA1327D3B24A
:106A500087EA131848EA032787EAC3028AEA020989
:106A600089EA091C5FFA8CF8170A87EA181E4A1C83
:106A70004EEA082B82428BEAC803DDD15FFA83FC21
:106A80008CF0FE0787EA0711CFB21B0A83EA1710C2
:106A900080EA072282EAC7018BB20020FE215FFA5A
:106AA00083FA4FEA1329FBF7FDFD9DF8AD11002095
:106AB000FBF7F8FD9DF8AE110020FBF7F3FD9DF804
:106AC000AF110020FBF7EEFD9DF8B0110020FBF7A1
:106AD000E9FD9DF8B1110020FBF7E4FD4FF000083F
:106AE0004EA807469DF8381140460DF5AE7BFBF7E2
:106AF000D9FD79784046FBF7D5FDB9784046023795
:106B0000FBF7D0FD5F45F4D1FFF799BA4AF2A8230D
:106B1000C1F200039DF82D2093F83A350492C7EB9B
:106B2000030CDCF1000343EB0C03D0E900010993F3
:106B300015F0FEFA0890DAE9020115F0F9FA40F6CC
:106B40007413C2F2000398F80090997998F801C084
:106B50008DF8AE1181F0280282EA0212D2B24FEA19
:106B6000121E8EF0790E4EEA022E8EEAC20E8EEAC8
:106B7000090282EA0212D2B24FEA1E2E8EEA121ED9
:106B80008EEA022E8EEAC20E1FFA8EFE8EEA0C02EA
:106B900082EA0212D2B24FEA1E2E8EEA121848EA98
:106BA00002284FF0270E88EAC20888EA0E0282EA1D
:106BB0000212D2B24FEA182888EA121888EA02288C
:106BC00088EAC2081FFA88F888EA08124FEA1828EB
:106BD000CDF80080DAF82080CDF81480DAF81C8037
:106BE000CDF81880DAF82880DAF810A0CDF81C80EB
:106BF000CDF850A1DDF800A0ADF85471D2B28AEA08
:106C0000121801F1010A00214E910599049F4F913C
:106C100006995390509107995191089952911521D5
:106C2000ADF85611BE218DF858718DF8591101211A
:106C3000099F8DF85C11FE2148EA02288DF8AC11FD
:106C400083F806A0252157A84EAB8DF85AB18DF8D0
:106C50005B718DF8AD118DF8AF918DF8B0C18DF8E5
:106C6000B1E10130013388EAC202194693F801907C
:106C700011F8017B87EA020383EA03185FFA88F7B9
:106C80004FEA122A8AEA171242EA072C8CEAC70353
:106C900089EA030E8EEA0E1B5FFA8BF91F0A87EA58
:106CA00019184B1C48EA092A83428AEAC902DCD136
:106CB0005FFA82F989F0FE0E8EEA0E115FFA81FB0F
:106CC000100A80EA1B1787EA0B2383EACB018AB2FA
:106CD0000020FE215FFA82FA4FEA1229FBF7E2FC5C
:106CE0009DF8AD110020FBF7DDFC9DF8AE110020F2
:106CF000FBF7D8FC9DF8AF110020FBF7D3FC9DF803
:106D0000B0110020FBF7CEFC9DF8B1110020FBF77D
:106D1000C9FC4FF000084EA807469DF838114046C0
:106D20000DF5AE7BFBF7BEFC79784046FBF7BAFC6D
:106D3000B97840460237FBF7B5FC5F45F4D1FFF761
:106D40007EB940F6840EC2F2000E9DF82D709DF8BB
:106D50002E308EF8D7704FF4406C4FF00008C4F21C
:106D6000000C8EF8D8308EF8D9A08EF8DA80DCF8D6
:106D7000241099F80070CEF8DC10FEF72EBB00212D
:106D8000BE78B970002B7EF475AAFEF720B9BF4B10
:106D9000D0F818E093F83A359DF82D804FF47A72C8
:106DA000BEFBF2F2C7EB0309D9F1000307EE102A8C
:106DB000D0E9000143EB0903B8EE478A019315F0CF
:106DC000B7F98146DAE9020115F0B2F9DAF81010E4
:106DD000DAF81CC0DAF824E0019BDAF814A0549128
:106DE0000122BE218DED4F8ACDF838A1CDF840C1EA
:106DF000CDF844E1CDF848915390ADF85471ADF819
:106E000056218DF858818DF859118DF85AB18DF8A9
:106E10005B318DF85C2127204EA92522FE23FBF74C
:106E200049FCFEF7A9BA994BD0F818E093F83A3527
:106E30009DF82D804FF47A72BEFBF2F2C7EB030E81
:106E4000DEF1000307EE902AD0E9000143EB0E03C8
:106E5000B8EE678A019315F06BF98146DAE9020111
:106E600015F066F9DAF81020DAF824E0DAF82010E4
:106E7000DAF814C054928DED4F8ACDF838C1CDF8B0
:106E800040E15191CDF848915390ADF854711622DC
:106E90000198ADF85621BE2301228DF858818DF856
:106EA00059318DF85AB18DF85B018DF85C21B2E74C
:106EB000764BD0F818E093F83A359DF82D804FF4D2
:106EC0007A72BEFBF2F2C7EB030CDCF1000307EEB3
:106ED000102AD0E9000143EB0C03B8EE478A019376
:106EE00015F026F98146DAE9020115F021F9DAF800
:106EF0001020DAF81CE0DAF82410DAF814C0549202
:106F0000CDF838C18DED4F8ACDF840E15191CDF8E3
:106F100048915390ADF854711022B9E762A810223D
:106F200017F0EEF9FFF7D1B8584606F0B5FFA8F113
:106F3000030C0746DCF1000848EB0C08022310980C
:106F400087F82C8087F82D3015F0D6F802460B46CE
:106F50001198C7E9002315F0CFF8129A0C9B3A61FB
:106F6000DDED0D7A7B610F9B0E9A3B6267EEA87A8E
:106F7000474B7A62FCEEE77AC7E90201C7ED067A71
:106F80004FF000081F78FEF7F3BC584606F084FF68
:106F90000746A8F10300414241EB0002109887F830
:106FA0002C20042387F82D3015F0A6F802460B4656
:106FB0001198C7E9002315F09FF8DDED0D7A129ABC
:106FC0000C9B3A6167EEA87A7B610F9B0E9A7B62FD
:106FD000FCEEE77AC7E90201C7ED067A2C4BFA61AD
:106FE0001F784FF00008FEF7C3BC584606F054FF68
:106FF000A8F103030746584240EB030187F82C1021
:1070000010980323CEE7584606F046FF012380F888
:107010002D3006F04BFF07460323109887F82D30DC
:1070200015F06AF802460B461198C7E9002315F0DF
:1070300063F8129A0C9B3A617B610F9BDDED0D7A30
:107040007B62144B67EEA87AD3F8FC31FCEEE77A4A
:10705000FB610F4BC7E90201C7ED067A4FF000084C
:107060001F78FEF785BCB0EE480A15F00FFC00282B
:107070007FF400AB94F8BC2151073FF5FBAA05480B
:1070800000EB870E8EED008AFFF7F4BAA8A200107D
:10709000A8090020AC02001006F008FF07460323F1
:1070A000109887F82D3015F027F802460B461198F6
:1070B000C7E9002315F020F8129A0C9B3A617B6116
:1070C0000F9BDDED0D7A7B62074B67EEA87AD3F854
:1070D000FC31FCEEE77AFB61044BC7E90201C7ED26
:1070E000067A1F78FEF744BCAC020010A809002005
:1070F0002DE9F04F40F68404C2F2000440F2AC2BBC
:1071000083B00021F022C1F2000B204617F0F8F8FE
:10711000DBED7D1AFCEEE17A00264FF4805017EE8D
:10712000901A33464FF44072C4F2010000960CF0FE
:107130007BF9606511F00EFE012203461421201D2B
:10714000A37011F0B1FF01464FF6F050C0F60100F8
:10715000E170FBF7C9FB4FF4B770C4F8CC002066B0
:1071600006F064FE4FF60061C5B26A1CC0F601016C
:107170004FF48C7084F8D95084F8DA2003F0B2FB15
:1071800040F6F85AC2F2000A074600F58A6341F653
:10719000280244F6FD603146C0F20102CAF80070D0
:1071A0000C33C0F6000012F0A1FA034630466370BB
:1071B00002F080FD44F6D351C1F26201A1FB00153B
:1071C00040F6A819C2F200092A09FA274FF44068CC
:1071D00007FB12030125C4F2000802220327BE2187
:1071E00089F8003089F8022089F8011084F8D570F8
:1071F00084F8D46084F8D650D8F8246002EE106A7F
:107200009FED473AF8EE422ADFED463A72EE837A76
:107210009FED454ADFED454A9FED455ADFED455A62
:107220009FED456A9FED451ADFED456ADFED450AA2
:107230009FED457A9FED450ADFED451A37EEA32A0B
:1072400077EE842A37EEA43A77EE853A37EEA54AF0
:1072500077EE864A37EE815A77EEA65A37EEA06A65
:1072600037EE871A77EE800A37EEA10ABCEEC22A03
:10727000FCEEE22ABCEEC33ABCEEC44AFCEEE44AA1
:10728000FCEEE55A44F24023FCEEE33ABCEEC55A6C
:10729000BCEEC66AFCEEC16ABCEEE07AFCEEC07AD7
:1072A00048F2A062C0F20F0365F31F4212EE10AA6B
:1072B00012EE909A13EE108A14EE107A14EE906A81
:1072C00015EE90BA84ED2F6AC4ED306A84ED317A00
:1072D000A36684ED272AE366C4ED282A236784ED9C
:1072E000293AC4ED2A3AA36784ED2B4AE367C4ED3B
:1072F0002C4AC4F8803084ED2D5AC4F88430C4ED93
:107300002E5AC4F88830C4F88C30C4F89030C4F8D1
:107310009430C4ED327A626703B0BDE8F08F00BFED
:107320008096984A00409C4500401C4600606A4692
:1073300000409C460050C3460060EA4600B808473B
:1073400000401C4700C82F470050434700D856470D
:1073500000606A474FF44060C4F20000B0F80CC00F
:107360002CF0020211040B0C0221838110F058BF93
:107370004FF44060C4F20000B0F80CC02CF00402DE
:1073800011040B0C0421838110F04ABF4FF44060BC
:10739000C4F20000B0F80CC02CF0080211040B0C71
:1073A0000821838110F03CBF70B58AB0002501260A
:1073B000322209A88DF824208DF825608DF82650FA
:1073C0008DF827600FF0DCFA0820314610F052F8F3
:1073D00042F20C2CC2F2000C4DF68360DCF808304F
:1073E000ADF8205013FA06F4C4F21B30A0FB0421C0
:1073F0004FF44064C4F20004880C4FF0FF32431E87
:1074000006A920460792ADF81830ADF81A5010F0D2
:1074100017FC2946204610F07DFCFFF79BFFFFF785
:10742000A7FFFFF7B3FF01A810F0AEFD2023204611
:1074300001A9ADF80430ADF80660ADF8105010F0B9
:107440007DFC2046294610F0A9FD204601A910F038
:10745000C1FC2046294610F0ABFD2046314610F015
:107460005FFC0AB070BD00BF10B44FF4406340F63B
:107470002C64C4F20003C2F200044FF6FD7CE2600B
:107480002160A3F810C0596A42185A63998988B2DA
:1074900040F002029A8110BC704700BF10B44FF454
:1074A000406340F62C64C4F20003C2F200044FF6BD
:1074B000FB7C22616160A3F810C0596A42189A638C
:1074C000998988B240F004029A8110BC704700BFCD
:1074D00010B44FF4406340F62C64C4F20003C2F2CF
:1074E00000044FF6F77C6261A160A3F810C0596AEE
:1074F0004218DA63998988B240F008029A8110BC78
:10750000704700BF70B54FF44064C4F200042046D9
:10751000022110F079FE20BB2046042110F074FEF9
:1075200058B92046082110F06FFE002841D12046AE
:10753000102110F069FE38BB70BD4FF6FB7CA4F83B
:1075400010C0A18940F62C6E21F00400C2F2000E9A
:107550000204130CDEF81000DEF80410A381884743
:1075600070BD4FF6FD722282A38940F62C6C23F089
:107570000200C2F2000C01040A0CDCF80C00DCF87A
:107580000030A281984770BD4AF60025C1F200057F
:1075900020466E6910F008FEB11C05EB810C013627
:1075A000CCF80400102120466E61BDE8704010F058
:1075B00037BE4FF6F7722282A38940F62C6E23F075
:1075C0000800C2F2000E01040A0CDEF81400DEF816
:1075D0000830A281984770BDDFED0F7AB4EEE70A5C
:1075E000F1EE10FA08D59FED0D7A30EE070AB4EEF1
:1075F000E70AF1EE10FAF8D4DFED087AB4EEE70A04
:10760000F1EE10FA06DB30EE670AB4EEE70AF1EEAF
:1076100010FAF8DA704700BF000000000000B44321
:1076200030EEC00ADFED107AB4EEE70AF1EE10FAA0
:1076300008DD9FED0E7A30EE470AB4EEE70AF1EE70
:1076400010FAF8DCDFED0A7AB4EEE70AF1EE10FA90
:1076500008D89FED067A30EE070AB4EEE70AF1EE9D
:1076600010FAF8D9704700BF000034430000B4435B
:10767000000034C340F2AC23C1F200032DE9F00F47
:107680004FF0000BC4F2CE2BC3F800B04FF0804B8C
:10769000C3F810B04FF0000BC4F2400BC3F814B0A5
:1076A0004FF0814BC3F818B04FF0000BC4F2A00BA1
:1076B000C3F81CB04FF0000BC4F2C00BC3F820B0ED
:1076C0004FF0000BC4F2E00BC3F824B04FF0824B34
:1076D000C3F828B04FF0000BC4F2101BC3F82CB055
:1076E0004FF0000BC4F2201BC3F830B04FF0000B7A
:1076F000C4F2301BC3F834B04FF0000BC4F2400B9F
:10770000C3F838B04FF4804BC4F2884BC3F83CB098
:107710004FF0000BC4F2BD4BC3F840B043F2333B13
:10772000C3F6337BC3F848B04BF2177BC3F6D11BCB
:10773000C3F854B04FF0000BC4F2202BC3F858B07C
:10774000C3F85CB04FF0000BC4F2963BC3F864B0D2
:107750004FF0000BC4F2343BC3F868B04FF4C04B99
:10776000C4F2E05BC3F874B04FF440404CF6CD4433
:1077700000254FF0000B00224FF07E51C4F27940FB
:10778000C4F2A015C3F64C544FF07A59C4F27A3BB8
:10779000D9601D66C3F87890D8675A609A605A64B9
:1077A000DC641C65DA661A67C3F88000C3F888B029
:1077B0004FF0000BC4F2963BC3F88CB049F69A1B0D
:1077C000C3F6196BC3F890B04FF0000A4FF0000BEE
:1077D000C4F2A02AC4F2482BC3F894B0C3F89CA00A
:1077E000C3F8A0A0C3F8A4A04FF0000B4FF0000A0C
:1077F000C4F2343BC4F2702AC3F8A8B0C3F8ACA0FA
:1078000041F26F2B4FF0000AC3F6032BC4F2DA4AA1
:10781000C3F89890C3F8B0B0C3F8B4A0C3F8B89058
:107820004FF0000B4FF000094CF2AC5AC4F296290D
:10783000C4F27A3BC3F2A77AC3F8C090C3F8C8B0C9
:10784000C3F8D0A04FF000094DF20A7B4FF0000AB8
:10785000C3F6A079C3F6235BC4F6610AC3F8DC90D3
:10786000C3F8E0B0C3F8E890C3F8ECA04FF000090B
:107870004FF4204B4FF4404AC4F24839C4F28C4BC9
:10788000C4F2734AC3F8F090C3F8F8B0C3F8FCA090
:107890004FF000084FF440494FF0000B4FF0000A42
:1078A000C4F21638C4F2F349C4F2FA3BC4F2E17AE6
:1078B000C3F88400C3F80091C3F804B1C3F8BC80D6
:1078C000C3F8C480C3F8CC40C3F8D420C3F8D82090
:1078D000C3F8E420C3F8F420C3F80821C3F80C214E
:1078E000C3F81021C3F81421C3F81821C3F81C21D0
:1078F000C3F82021C3F82421C3F82821C3F82C2180
:10790000C3F83021C3F83421C3F83821C3F83C212F
:10791000C3F84021C3F84421C3F84821C3F84C21DF
:10792000C3F85021C3F85421C3F85821C3F85C218F
:10793000C3F86021C3F86421C3F86821C3F86C213F
:10794000C3F87021C3F87421C3F87821C3F87C21EF
:10795000C3F88021C3F88421C3F88821C3F88C219F
:10796000C3F89021C3F8F4A14FF0000AC4F2E00A72
:10797000C3F8F851C3F808A2C3F81052C3F8145260
:107980004FF000094DF20A7A0025C3F6A33AC4F27B
:10799000A0094FF07F5BC4F2F015C3F8FC91C3F867
:1079A00000B2C3F80CA2C3F89421C3F89821C3F81D
:1079B0009C21C3F8A021C3F8A421C3F8A821C3F8CF
:1079C000AC21C3F8B021C3F8B421C3F8B821C3F87F
:1079D000BC21C3F8C021C3F8C421C3F8C821C3F82F
:1079E000CC21C3F8D021C3F8D421C3F8D821C3F8DF
:1079F000DC21C3F8E021C3F8E421C3F8E821C3F88F
:107A0000EC21C3F8F021C3F80422C3F81852C3F8DC
:107A10002402C3F82C020020C4F24830C3F830021C
:107A20000020C4F22F40C3F83C02C3F840020020FB
:107A3000C4F22000C3F84C02C3F8540243F2333CB2
:107A40004AF2E35748F65C7646F266694CF6CD4B4F
:107A50000020CBF6D37CC3F69B47C3F64266C4F244
:107A60003609C3F64C6BCCF282204FF07C55C3F83C
:107A70003492C3F844B2C3F85CC2C3F860C2C3F81E
:107A800064C2C3F81C52C3F82022C3F82822C3F8EA
:107A90003882C3F84822C3F85022C3F85822C3F8EA
:107AA0006822C3F86C22C3F87022C3F87422C3F8AA
:107AB0007822C3F87C22C3F88022C3F88422C3F85A
:107AC0008822C3F88C72C3F89072C3F89472C3F81A
:107AD0009822C3F89C2243F6715CC3F8A02247F6B3
:107AE000FA69C3F8A422C3F8A822C3F8AC22C3F8E9
:107AF000B022C3F8B422C3F8B822C3F8BC22C3F83A
:107B0000C022C3F8C422C3F8C822C3F8CC22C3F8E9
:107B1000D022C3F8D422C3F8D822C3F8DC22C3F899
:107B2000E022C3F8E422C3F8E822C3F8EC22C3F849
:107B3000F022C3F8F422C3F8F822C3F8FC22C3F8F9
:107B40000023C3F80463C3F80863C3F80C63C3F8E5
:107B50001023C3F81423C3F81823C3F81C23C3F855
:107B60002023C3F82423C3F82823C3F8A0034FF429
:107B70002040CBF6AA7CC3F6EA59C4F20C50C3F8F5
:107B80004CC3C3F850C3C3F854C3C3F87C93C3F8C1
:107B90008093C3F88493C3F82C23C3F83023C3F82D
:107BA0003423C3F83823C3F83C23C3F84023C3F875
:107BB0004423C3F84823C3F85823C3F85C23C3F80D
:107BC0006023C3F86423C3F86823C3F86C23C3F8A5
:107BD0007023C3F87423C3F87823C3F88823C3F849
:107BE0008C23C3F89023C3F89423C3F89823C3F8D5
:107BF0009C23C3F8A423C3F8A823C3F8AC23C3F879
:107C0000B023C3F8B4030020C4F24830C3F8C4035F
:107C10004FF4204C4FF400494FF48040C4F20C5C08
:107C2000C4F23B49C4F2B440C3F8BCC3C3F8C09328
:107C3000C3F8CC034FF4004B40F6413C40F6A16939
:107C40000020C4F23B4BC3F6344CC3F66A49C4F27D
:107C50006000C3F8B8B3C3F8D0C3C3F8D493C3F873
:107C6000E0034FF4604B43F2333045F6C04C41F231
:107C70005D69C4F2C44BC4F25300C4F2131CC4F2D5
:107C80006D19C3F8C8B3C3F8D8A3C3F8E403C3F8A5
:107C9000E8C3C3F8EC9349F6364A03F5806943F22A
:107CA000667B4DF2AE6042F6CD1CCCF26B2AC4F27C
:107CB000E92BCCF2D620C4F2172CC3F8F0A3C3F8FA
:107CC000F4B3C3F8F803C3F8FCC3C9F80020C9F83B
:107CD0000420C3F8DC23DFF804934FF4006046F679
:107CE000CD43C4F2BD50C4F28E53C9F80800C9F8A0
:107CF0000C304EF2C12B4AF6C57C46F6903045F664
:107D00001003C3F6106BC3F6752CC3F63F20C4F204
:107D10008223C9F804B0C9F810C0C9F81800C9F81E
:107D20001C304FF6DB4B4DF2D13C40F665204FF650
:107D30004F63C3F63F5BC3F2934CC3F67E00C3F6BA
:107D4000D503C9F814B0C9F820C0C9F82800C9F88B
:107D50002C304BF2600A41F61F1B4FF4064C4EF6D6
:107D600074504EF27803C3F69B5AC3F25E5BC3F2C3
:107D70008A3CC3F2B810C3F29643C9F800A0C9F810
:107D800024B0C9F830C04CF6303BC9F83800C9F807
:107D90003C304CF6A96C48F6C3504AF2A403C3F237
:107DA000EB3BC3F2937CC3F6A000C3F62103C9F8F2
:107DB00034B0C9F840C0C9F84800C9F84C304DF695
:107DC000525B47F2EE6C40F64A404CF2FC43C3F67D
:107DD000460BC3F63D5CC4F27200C3F68143C9F89A
:107DE00044B0C9F850C0C9F85800C9F85C3041F631
:107DF000EF4B4DF6556C43F63A304BF29573C3F6A4
:107E00004A4BC3F62E6CC3F69940C3F6C363C9F858
:107E100054B0C9F860C0C9F86800C9F86C3043F2C2
:107E2000FE5B09F1780349F2666C41F2A930C3F6B2
:107E30005040C3F6C80BC4F2005CC9F864B0C9F87E
:107E400070C0186358634FF4194B40F2DE5C002099
:107E5000CCF2CA7BC3F6CA4CCCF22010A9F1080AB6
:107E6000C9F874B0C9F8841009F1900BC9F88810EA
:107E7000C9F88C10C9F8B0C0C9F8B400C9F87820A6
:107E8000C9F87C20C9F88020C9F89420C9F8982046
:107E9000C9F89C20C9F8A020C9F8A420002309F142
:107EA000B8094EF68530CCF2C813C4F26910CBF88D
:107EB0000020C9F80030C9F80C00CBF83810CBF816
:107EC0003C1000234CF6CD4100204FF0814CCCF209
:107ED0002013C4F29411C4F27A40C9F818C0C9F84A
:107EE0002030C9F82410C9F8280009F1280109F147
:107EF00020004FF4404C4FF40053C4F2F34CC4F252
:107F0000CB53C9F80420CAF8C820CBF84440C9F8BC
:107F10002CC0C9F83820C9F84020C9F84420CAF854
:107F20000821C9F84C20CBF87820CBF87C20C9F880
:107F30005820CBF88420C9F86820C9F87020C9F807
:107F40007420CAF83821C9F87C20CBF8A820CBF8D7
:107F5000AC208B60CA604A618A63CA634A64C9F80C
:107F60008820CBF8B420C9F89820C9F8A020C9F817
:107F7000A420CAF86821C9F8AC20CBF8D820CBF8E7
:107F8000DC20C9F8B820CBF8E420C9F8C820C9F82B
:107F9000D020C9F8D420CAF89821C9F8DC20CBF841
:107FA0000821CBF80C21CBF814218A66CA664A67EF
:107FB000C1F89820C1F89C20C1F8A4200AF5CC7A19
:107FC00009F1D009C0F8C8200BF5847BC1F8C8209E
:107FD000C1F8CC20BDE8F00F704700BFB406001018
:107FE00008B501F063FE014640F2AC20C1F200008A
:107FF0004FF4B762BDE8084016F064B908B501F067
:1080000055FE40F2AC21C1F200014FF4B76201F01D
:1080100091FDC0B208BD00BF2DE9F04F89B0002826
:1080200000F0958001F03CFC002801900090C0F227
:10803000938001214FF4007002F000FC012183467F
:10804000802002F0FBFB40F2000440F2AC258046A9
:108050000027C2F20004C1F20005009859464FF013
:10806000FF324FF4007301F08DFC0028824653DD8F
:10807000002604E008F8073001375645EDD01BF81C
:10808000063001360A2B01D07F2FF3D14FF63C7119
:108090004FF00009C0F6010108F80790404603AA16
:1080A00007AB16F0CDF8022817D04FF65C71C0F67A
:1080B0000101404603AA07AB16F0C2F802280CD013
:1080C0004FF65471C0F60101404603AA07AB16F003
:1080D000B7F8022801D04F46CFE7002739591022C0
:1080E00003A816F0C1F8034607F1040903A81022FB
:1080F000EF190BB90799396059F8041016F0B4F864
:1081000018B905EB0900079A026009F10407B7F5F1
:10811000B76FE3D10027B0E7019801F057FCB8F141
:10812000000F04D040468021012202F0A9FBBBF1E0
:10813000000F05D058464FF40071012202F0A0FB59
:108140005FFA8AFA4FFA8AF009B0BDE8F08F4FF66D
:108150000870C0F6010065E74FF61470C0F6010024
:10816000FAF7C2FB4FF0FF0AECE700BF10B52DEDA8
:10817000028BFFF735FF0020FFF74EFF002842DBA0
:108180000DF026FB01F092FD90ED008AB0EE480A5A
:1081900014F090FBC8B9DFED257AB4EEE78AF1EE72
:1081A00010FA14D440F2AC23C1F20003D3ED007AEC
:1081B000B4EEE78AF1EE10FA2FDAB4EEE78AF1EEC8
:1081C00010FA1AD4BDEC028B10BD9FED198A40F253
:1081D000AC24C1F20004D4ED007A9FED147AF4EEE1
:1081E000C77AF1EE10FAE3D5FFF744FAD4ED007A3E
:1081F000B4EEE78AF1EE10FAE4D5BDEC028BBDE8EF
:108200001040FFF7FBBE40F2AC2000214FF4B762F4
:10821000C1F2000016F074F8B4E7FFF7E1FE40F297
:10822000AC20C1F20000D0ED007AC6E70000CE42DB
:10823000000000002DE9F04FA5B0002860D001F04B
:108240002FFB0028039080465FDB40F20004C2F25F
:10825000000404F5B6604FF68C76031D2F4D029393
:10826000043CC0F601064FF0FF391CE0586857681F
:1082700013F042FF3A4682468B4604A83146CDE9C8
:1082800000AB15F0C7FF07463B46404604A94A46E7
:1082900001F08AFB5FFA80FA4FFA8AF39F421FDCF3
:1082A000029A944224D06868676813F025FF3A4622
:1082B00082468B4604A83146CDE900AB15F0AAFFF3
:1082C000074604A94A463B46404601F06DFB41B2D1
:1082D000221D2B1D8F4202F1040403F10405C5DDAC
:1082E0004FF69C70C0F60100FAF7FEFA4FF0FF0A55
:1082F000039801F06BFB4FFA8AF025B0BDE8F08FD0
:108300004FF60870C0F6010099E74FF66470C0F6AA
:108310000100FAF7E9FA4FF0FF0AECE7A8020010B3
:108320002DE9F84341F2406040F6640441F6B85547
:108330002DED068BC0F60200C1F20004C2F200056A
:10834000FAF7D2FA04F1240705F58266ADE140F2AE
:10835000AC29C1F20009D9ED020ABDEEE00A4AF6E5
:10836000BC1810EE100AC1F200080830D9ED187AD6
:1083700038F9101006EE901AB8EEE67AB4EEE77A05
:10838000F1EE10FA08DC4AF2A82CC1F2000C9CF8BD
:108390003805002800F0558201200DF0F7F94AF267
:1083A000A823C1F2000393F83825002A40F0F18198
:1083B00040F2AC2EC1F2000E9EED024AFDEEC43A30
:1083C0004AF6BC1813EE902AC1F200080832DEED1E
:1083D000182A38F9120003EE100AB8EEC32ADEEDAF
:1083E000127A72EE621A21EEA70ADFEDF38A27EE07
:1083F000A86ABDEEC08AFDEEC65A18EE100A012129
:1084000015EE902A4AF2F01902F0E6FAC1F20009DC
:108410009FEDEA8AD9ED274A05EE100AF4EE484AA4
:10842000F1EE10FAB8EEC5AA00F0688140F2AC2374
:10843000C1F20003D3ED05AAFDEEEA9A4AF6BC129A
:1084400019EE901AC1F200020831D3ED167A32F912
:10845000110009EE100AB8EEC98AB4EEE78AF1EE0F
:1084600010FA40F3368178EE677AD3ED156A27EE7D
:10847000A68A4AF2A828C1F20008D8ED031A05F529
:10848000806CDCED010A38EE210AFFF7C9F815F01F
:10849000C5FC9FEDCB1AB4EEC10AF1EE10FA00F163
:1084A000D581D8ED030A40F2AC2894ED080AC1F258
:1084B0000008FFF7B5F8D8ED1A3A9FEDC24AF1EE81
:1084C000634AC4EE840A83EE841A02F08DFA94EDB6
:1084D000083A30EE030AFFF77FF84AF2A823C1F208
:1084E000000384ED080A93F83825032A00F0A181DF
:1084F00098ED040AD8ED037AFDEEC06ABDEEE77A86
:1085000016EE901A17EE103A4AF6BC19C1F200099D
:108510000831083339F911E039F913000AEE90EA0D
:1085200009EE900AB8EEEA6A98ED139AF8EEE98A35
:1085300098ED148A66EE095A28EE885A012AC4ED8D
:10854000025A84ED035A40F278814AF2A828C1F217
:108550000008D8F82810D8F82C002161606138464E
:1085600094ED020A02F016FB04F13C0084ED020ACD
:1085700094ED030A02F00EFB04F1540084ED030AAB
:1085800094ED040A02F006FB04F16C0084ED040A89
:1085900094ED050A02F0FEFAD4ED043A96ED014A94
:1085A00096ED003A20EE042A23EE841A13EE832A75
:1085B00000EE031A40F2AC2CC1F2000CD4ED022AFA
:1085C000D4ED031ADCED116A9FED7C8A72EE227AFB
:1085D00071EE810AF4EE486AF1EE10FA84ED050AB4
:1085E000C4ED067AC4ED070A00F0EE80F7EE004A0B
:1085F000F4EE646AF1EE10FA00F03B81B0EE489AB6
:1086000005F5806EDEED010A94ED080AD4F8988035
:10861000D4F88C90FFF704F84046F0EE400A9FED46
:10862000670A07F081F840F22010C1F2000040F222
:10863000AC28D0F82031484600EE903A07F074F8A4
:10864000C1F2000898ED191AF0EE409AF1EE410AD5
:10865000B0EE480A02F0C8F998ED191AF0EE40AAF7
:10866000F1EE410AB0EE490A02F0BEF998ED191A8E
:10867000B0EE408AF1EE410AB0EE690A02F0B4F9B8
:10868000F0EE480AF0EE401AB0EE6A1AB0EE4A0A6E
:1086900003F02EFA40F2201CC1F2000C6068DCF8F6
:1086A0007821411CC4F89C20616041F21012C1F293
:1086B00000020021107810F0E1F94AF61440C1F2EE
:1086C000000090F8BC319B073FF541AE03F052F932
:1086D000E0E7B1EE677AB4EEC78AF1EE10FA06D49D
:1086E0004AF2A829C1F20009D9ED030ADBE638EE07
:1086F000270AD3ED150A20EE208ABAE605F5806137
:108700004AF2A8284B68D4F888002362C1F2000816
:10871000B0EE480AC8F80C30F0EE480A07F0EAF864
:10872000D4F88400B0EE480AF0EE480A07F0E2F808
:10873000D4F88C00B0EE480AF0EE480A07F0DAF8F8
:10874000D4F89400B0EE480AF0EE480A07F0D2F8E8
:10875000D4F89000B0EE480AF0EE480A07F0CAF8E4
:10876000D4F89800B0EE480AF0EE480A07F0C2F8D4
:1087700098F838C5BCF1020F7FF458AE41F2680E8C
:10878000C1F2000E9EED0E0B9EED101B05F0E4FCF9
:108790004CE6D5F83C14986C91ED021A93ED0C0A56
:1087A000F1EE410A06F0C0FF40F2AC23C1F2000333
:1087B000D3ED127A19E600BF0000AF4400000000BC
:1087C000000034420000C84305F5816E40F22019D4
:1087D000DEED000AB0EE670AD4F89400C1F2000999
:1087E00006F0A2FFD9F81C31D4F8880000EE903AC8
:1087F000B0EE409AB0EE480A06F096FF05F58061AB
:10880000D1ED030AD4F8900030EE099A94ED070AEE
:1088100006F08AFFD9F81821D4F88400F0EE408AD7
:1088200000EE902AB0EE480A06F07EFF30EE288A6D
:10883000E6E60022A260E26087E60023236163612E
:108840008DE60CF0A3FF03F095F823E7D4ED082A9A
:1088500038EE220AFEF7C0FE98ED032A84ED080ADE
:1088600038EE020AFEF7B8FEF0EE400A88ED030A81
:1088700019E640F2201805F58161C1F20008D1ED3A
:10888000000AB0EE670AD4F89400D4F8889006F095
:108890004BFFD8F81C21484600EE902A06F044FF12
:1088A00005F5806CDCED030AD4F89000D4F88490D0
:1088B000B0EE409A94ED070A06F036FFD8F818019A
:1088C00000EE900A484606F02FFFB0EE408A97E689
:1088D0002DE9F04F2DED048B41F258608BB040F63E
:1088E0006404C1F200049FED8F8ADFED8F8AC0F629
:1088F00002009FED8E9A0994F9F7F6FF0021A0225D
:108900000998DFF82CB215F0FBFC04F12400B0EE5E
:10891000480AF0EE490AB0EE681A02F02BF904F1A9
:108920003C00B0EE480AF0EE490AB0EE681A02F0D8
:1089300021F904F15400B0EE480AF4EE000AB0EE5A
:10894000681A02F017F94FF0000AB0EE480AF4EE88
:10895000000AB0EE681A04F16C000BF104070BF189
:1089600008060BF10C05CDF820A002F003F9DDF8A4
:1089700020C00BF110040BF114080BF118090BF1D6
:108980001C0A394632462B4658468DE81007CDF86A
:1089900010C0CDF814C0CDF818C0CDF81CC006F03A
:1089A000A5FE3946099F8446C7F888C08DE81007A0
:1089B000DDF8209032462B465846CDF81090CDF881
:1089C0001490CDF81890CDF81C9006F08FFEDDF8CD
:1089D00024E0DDF820C004460BF12000CEF88440EE
:1089E00000F11004009400F11404019404340BF11C
:1089F00024010BF128020BF12C030294043403949C
:108A0000CDF810C0CDF814C0CDF818C0CDF81CC0FA
:108A100006F06CFE04F10801099CDDF820C00BF1A2
:108A2000400786460BF148050BF14C06C4F88CE074
:108A30000BF1500807F11C042A4633460BF1540988
:108A40000BF1580A3846CDF810C0CDF814C0CDF857
:108A500018C0CDF81CC08DE80007039406F046FE50
:108A60003346099E8646C6F894E08DE80007DDF897
:108A7000208003942A460BF144013846CDF810803B
:108A8000CDF81480CDF81880CDF81C8006F02EFEAD
:108A9000DDF82480DDF820E00646C8F890600BF190
:108AA000780C0BF168020BF164010BF16C030BF114
:108AB00070050BF174040BF160000BF17C07CDF82D
:108AC00008C0CDF810E0CDF814E0CDF818E0CDF8EE
:108AD0001CE000950194039706F008FE41F26861DE
:108AE0000346C0F60201C8F89830962001F0FAFE5D
:108AF00040F64864DDF820C0C2F20004054648F2A2
:108B00002130C0F6000005F51573614649F2056293
:108B1000256010F0EBFD88F800000BB0BDEC048B75
:108B2000BDE8F08F0AD7233B00000000CDCCCC3D40
:108B300018030010704700BF70B50E4682B005469E
:108B40000821012001F0ACFE0560868004466E839A
:108B500068460EF0C7FB022000238DF805000122B5
:108B60002846694600968DF806308DF804208DF869
:108B700007300EF0FBFA204602B070BD0368828811
:108B800059690A4214BF5A831A83704710B540F2DC
:108B90000004C1F2000482B0034604220621022030
:108BA00022736373F7F7D4FDA07BE17B227C637CA7
:108BB0008DF804008DF805108DF806208DF807302B
:108BC0009DED010A02B010BD10B542F2A8432DED93
:108BD000048BC0F60203D3ED008A0446FFF7D6FFEC
:108BE000F4EE408AF1EE10FAB0EE408A59D02046F9
:108BF000FFF7CCFFB4EE408AF1EE10FAB0EE409AE7
:108C000057D02046FFF7C2FFB4EE409AF1EE10FABB
:108C1000B0EE408A4AD02046FFF7B8FFB4EE408A53
:108C2000F1EE10FAB0EE409A43D02046FFF7AEFFC7
:108C3000B4EE409AF1EE10FAB0EE408A36D02046FB
:108C4000FFF7A4FFB4EE408AF1EE10FAB0EE409ABE
:108C50002FD02046FFF79AFFB4EE409AF1EE10FABB
:108C6000B0EE408A22D02046FFF790FFB4EE408A53
:108C7000F1EE10FAB0EE409A1BD02046FFF786FFC7
:108C8000B4EE409AF1EE10FAB0EE408A0ED02046D3
:108C9000FFF77CFFB4EE480AF1EE10FA08BFF0EEE1
:108CA000488AB0EE680ABDEC048B10BDF0EE498A2C
:108CB000F7E7F0EE488AF4E730B583B00DF1080C21
:108CC0002CED010A40F20003C1F200039DF80440BC
:108CD0009CF802109CF801509CF803209C730446F9
:108CE00005201873062019745C73DD735A740146ED
:108CF000F7F72EFD2046FFF767FF03B030BD00BF3A
:108D0000F8B540F2B855C2F2000506462C68204678
:108D100015F070FB21460246304615F0A5FA0024F6
:108D2000E0B101240EE06F68384615F063FB394668
:108D30000246304615F098FA0134043570B101341A
:108D40002B2C0ED06F68384615F054FB394602467E
:108D5000304615F089FA04350028E4D1E0B240B27B
:108D6000F8BDFF2040B2F8BD38B52DED028B0546A9
:108D7000B0EE408AFFF7C4FF002823DBC4B22046D0
:108D8000B0EE480AFFF798FFB4EE480AF1EE10FA89
:108D900004D1012040B2BDEC028B38BD2046B0EEBC
:108DA000480AFFF789FFB4EE480AF1EE10FAF0D056
:108DB0002046B0EE480AFFF77FFFB4EE480AF1EE16
:108DC00010FAE6D040F64C64C2F2000441F2706141
:108DD000C0F602012A46204615F01CFA2046F9F793
:108DE00083FDFF20D6E700BF10B540F20004C1F2BA
:108DF0000004022103460922084622736373F7F731
:108E0000A7FC0A2300220221012023736273F7F7D3
:108E10009FFC237B0A2B0CBF607BFF2010BD00BF93
:108E20002DE9F04F2DED028B8BB0002800F03D8135
:108E300000F036FD002802900190C0F25A81012115
:108E40004FF4007001F0FAFC01210746802001F088
:108E5000F5FC0646002F00F02D81002800F02D8142
:108E600000254FF63C7A9FEDAD8A0395A946C0F6E2
:108E7000010A019839464FF0FF324FF4007300F0B9
:108E800081FD0028804640F3CA8017F809306FEA58
:108E9000090B58440A2B00F0010B09F1010400F002
:108EA0008A807F2D00F08780735501354445E0D0DE
:108EB000BBF1000F09D03B5D01340A2B11D07F2D8F
:108EC0000FD0735501354445D3D03B5D01340A2B97
:108ED00024D07F2D22D073553B5D013501340A2B00
:108EE000EDD106F805903046514605AA09AB15F0BC
:108EF000A7F902282FD105A8FFF702FF00280BDBF6
:108F0000C5B22846FFF760FEDDED097AB4EE670AC8
:108F1000F1EE10FA40F099804D46D4E706F805903E
:108F20003046514605AA09AB15F08AF902282AD124
:108F300005A8FFF7E5FE00280BDBC5B22846FFF7C2
:108F400043FEDDED097AB4EE670AF1EE10FA40F067
:108F500090804D46AFE74FF65471C0F601013046A0
:108F600005AA09AB15F06CF90228C4D04FF65C7164
:108F7000C0F60101304605AA09AB15F061F90228D7
:108F8000B9D04D469FE74FF65471C0F60101304607
:108F900005AA09AB15F054F90228C9D04FF65C7147
:108FA000C0F60101304605AA09AB15F049F90228BF
:108FB000BED04D467FE706F805903046514605AADB
:108FC00009AB15F03DF9022811D105A8FFF798FE6D
:108FD00000280ADBC5B22846FFF7F6FDDDED097A69
:108FE000B4EE670AF1EE10FA71D14D465EE74FF626
:108FF0005471C0F60101304605AA09AB15F020F9FD
:109000000228E2D04FF65C71C0F60101304605AA95
:1090100009AB15F015F90228D7D04D4646E702985E
:1090200000F0D4FC30468021012201F029FC2FB150
:1090300038464FF40071012201F022FC039A50B22D
:109040000BB0BDEC028BBDE8F08F2846B0EE670A8E
:10905000FFF732FEB4EE480AF1EE10FA1DD041F2ED
:10906000C460C0F60200F9F73FFC01204D460390B2
:1090700029E72846B0EE670AFFF71EFEB4EE480A5D
:10908000F1EE10FA1BD041F2C460C0F60200F9F70D
:109090002BFC012103914D460DE741F2E860C0F63B
:1090A0000200F9F721FC4D460DE741F29460C0F64D
:1090B0000200BDE680BB0390C0E70390B8E741F231
:1090C000E860C0F60200F9F70FFC4D46F3E62846CB
:1090D000B0EE670AFFF7F0FDB4EE480AF1EE10FAC1
:1090E00010D141F2E860C0F60200F9F7FDFB4D46F1
:1090F000DCE641F2A060C0F60200F9F7F5FBFF23C1
:1091000003939BE741F2C460C0F60200F9F7ECFB61
:1091100001234D460393C9E6039783E7000000004F
:1091200070B540F200042DED028BC1F2000416462A
:10913000F7F722FB0322012010212273F7F708FB27
:1091400094F81831012B22D040F68C65C2F200054C
:1091500041F20871C0F6020104F10C02284615F034
:1091600059F82846F9F7C0FB0120FFF72DFD07EE5F
:10917000906AB8EE678AB4EE480AF1EE10FA28D188
:109180000020FFF74DFE60B9BDEC028B70BD41F2CF
:109190006870C0F60200BDEC028BBDE87040F9F7C4
:1091A000A3BB40F2000CC1F2000C072200210120F9
:1091B0008CF80C20F7F7CCFA41F24870C0F60200A8
:1091C000F9F792FB6420BDEC028BBDE8704010F013
:1091D000B1BB3046FFF708FEB04205D041F218702F
:1091E000C0F60200F9F780FB41F23470B0EE480A95
:1091F000C0F60200FFF7B8FDC2E700BF10B590F857
:10920000603282B00446ABB1D4F84C12002904DBC2
:1092100004F1240012F07AF9B8B9D4F84812D4F85D
:10922000502204F1240001AB11F08AFF68B90198C3
:1092300002B010BD00F12400611C0A2211F060FD93
:1092400048B9012084F86002DEE7002184F860124A
:109250004FF0FF30ECE74FF0FF30E9E710B590F842
:10926000603282B00446ABB1D4F84C12002904DB62
:1092700004F1240012F04AF9B8B9D4F84812D4F82D
:10928000502204F1240001AB11F06CFE68B9019882
:1092900002B010BD00F12400611C012211F030FD6C
:1092A00048B9012084F86002DEE7002184F86012EA
:1092B0004FF0FF30ECE74FF0FF30E9E710B590F8E2
:1092C000603204462BB100F1240012F057F818B9AF
:1092D00010BD4FF0FF30FBE7002084F860024FF034
:1092E000FF3010BD30B583B090F8603200220446E4
:1092F0000192DBB940F6AC60C2F2000000F5606597
:10930000043541F69811D0F8442EC0F60201631CD2
:10931000284614F07FFF04F1240029460A2211F0A8
:10932000EFFC00283DD1012184F86012D4F85822C6
:10933000D4F85C32D01A14F073FEB0F5007F2EDB47
:10934000D4F85852D4F85C028542CBBFD4F85852B6
:10935000D4F85C02D4F85C02D4F850522A1AB2F560
:10936000007F01D9510A4A02D4F85C32D4F848127D
:1093700004F12400C91801AB11F0E2FED4F85C52EC
:10938000019BD4F8502205EB030CBCFBF2F502FB69
:1093900015C2C4F85C2220B9184603B030BD019B49
:1093A000FAE74FF0FF30F8E710B5044690F8600296
:1093B00000B910BD04F1240012F0A0F84FF0000332
:1093C000002884F8603218BF4FF0FF3010BD00BF96
:1093D00010B590F86132032B044618D0012B1BD036
:1093E000022B1ED0042B21D0052B07D02078002182
:1093F00084F86112BDE810400FF03CBCFFF7D4FFC9
:10940000C4F8540294F86132032BEFD110BDFFF77A
:1094100069FFC4F85402F5E7FFF720FFC4F85402CF
:10942000F0E7FFF7EBFEC4F85402EBE7FFF746FF67
:10943000C4F85402E6E700BF38B5084C41F6A4155D
:10944000C0F602050B4602462946204614F0E2FE0D
:109450002046BDE83840F9F747BA00BFB01C0020ED
:10946000F0B540F6AC64C2F2000404F53C6041F68D
:10947000B4110430C0F6020183B012F005F90328DC
:10948000014600F08B80012800F0888080B141F611
:10949000B810C0F60200FFF7CFFF002001460246D9
:1094A00012F024F90146002840F08480C4F8440EEC
:1094B00040F6AC64C2F2000441F6FC1104F53E67CC
:1094C000C0F602013846012211F01AFC05460028B8
:1094D00046D040F6AC63C2F20003D3F8444E611CA0
:1094E000B1F57A7FC3F8441E36D240F6AC64C2F2BE
:1094F000000441F6FC1104F53E65C0F60201284661
:109500000A2211F0FDFB014600284AD104F56060F3
:10951000061D41F65441D4F8442EC0F602013046EF
:1095200014F078FE304614F065FF3146024601AB78
:10953000284611F005FE0646284611F0DFFF002EF2
:109540002CD141F62420C0F60200D4F8441EFFF7C7
:1095500073FF304603B0F0BD0025C3F8445EC4E796
:1095600004F560660436402201AB3846314611F0FE
:10957000F9FC019B012B0DD941F6544104F56462BD
:109580000432C0F60201304614F05AFE0028D8BF5B
:10959000C4F8445E0C4811F0B1FF9AE74FF0FF3079
:1095A000D8E741F60820C0F60200FFF745FF4FF06C
:1095B000FF30CFE741F6E010C0F60200FFF73CFFB6
:1095C0004FF0FF30C6E700BF8C1A002041F638206C
:1095D0002DE9F843C0F6020040F6AC64C2F2000484
:1095E000F9F782F904F5186704F53C6904F5986504
:1095F0000126143709F104090C3500200CF0BEF8DF
:1096000000214FF40972384614F07AFE48460021D2
:109610001C2214F075FE002E41D131464FF4097220
:1096200004F1280014F06CFE4FF0FF38207984F824
:109630006462C4F858820FF01DFB31464FF4097282
:1096400004F5237014F05CFE94F8680284F8C86492
:10965000C4F8BC840FF00EFB31464FF4097204F5D8
:109660009E6014F04DFE94F8CC0484F82C67C4F886
:1096700020870FF0FFFA04F5EA6031464FF40972D3
:10968000043014F03DFE94F8300784F89069C4F873
:1096900084890FF0EFFA4FF47A7010F04BF93946E5
:1096A000002011F019FB0146002840F0C28005217E
:1096B00060780FF0E3F9D4F8481E4B1CC4F8483E1C
:1096C000FFF7CEFE0028C0F2B28001200CF056F861
:1096D00017E094F8C964002E3AD194F82D67002E53
:1096E0005AD194F89169002E78D160780FF068FA19
:1096F000607805210FF0C2F9D4F8480E461CC4F872
:10970000486E94F86522002AE3D0261D3046FFF704
:109710005FFE94F865020328DBD1D4F858120029C3
:109720007FDBD4F8483E44F6D351581CC1F26201A5
:10973000A1FB001291094FF47A7C0CFB1103002B62
:10974000C7D13046FFF7BAFD94F8C964002EC4D0E3
:1097500004F51A763046FFF73BFE94F8C904032857
:10976000BBD1D4F8BC1400295BDBD4F8482E44F6F6
:10977000D35C531CC1F2620CACFB031081094FF4A3
:109780007A7E0EFB1132002AA7D13046FFF796FDF4
:1097900094F82D67002EA4D02846FFF719FE94F800
:1097A0002D37032B9DD1D4F82017002939DBD4F8AD
:1097B000480E44F6D3510130C1F26201A1FB0013FF
:1097C0009A094FF47A7606FB1201002989D12846BE
:1097D000FFF774FD94F89169002E86D004F5E666D3
:1097E0003046FFF7F5FD94F89129032A7FF47DAF09
:1097F000D4F88419002914DBD4F8483E44F6D35138
:10980000581CC1F26201A1FB001291094FF47A7E4B
:109810000EFB1103002B7FF468AF3046FFF74EFDBF
:1098200063E741F67020C0F60200FFF705FE002650
:10983000E3E641F64C20C0F60200FFF7FDFDBDE86F
:10984000F8430FF0F9BF00BF70B540F6AC64C2F248
:10985000000440F64C620021204614F051FD002126
:1098600008460FF085F841F690210346C0F6020144
:10987000A020637001F036F841F6F8450646C2F2C2
:10988000000549F2CD50C0F6000006F51F73002117
:109890004AF23E022E600FF029FF207070BD00BF1B
:1098A00070B540F6AC64C2F20004054694F86662F6
:1098B0003EB3601D294614F075FD00283CD094F895
:1098C000CA34EBB104F51A700130294614F06AFD70
:1098D000B0B194F82E1759B304F598600D302946AD
:1098E00014F060FD20B394F892291AB304F5E663EE
:1098F000581C294614F056FDE0B1FF2040B270BD5F
:10990000012640F6AC60C2F200004FF4197404FB6B
:1099100006040122294684F86622601D14F020FD09
:10992000002001460FF024F82071F0B240B270BD63
:109930000226E6E70326E4E70646E2E710B504461A
:1099400090F86202D8B140F6AC6CC2F2000CC4F8D8
:1099500048129DF808109CF8010084F86112C4F8C0
:109960004C22C4F850320FF085F920780FF028F916
:10997000207800210FF082F8D4F8540210BD4FF087
:10998000FF3010BD30B540F6AC64C2F200044FF4B5
:10999000197505FB004083B0012404300094FFF7E3
:1099A000CDFF03B030BD00BF30B540F6AC64C2F2AD
:1099B00000044FF4197505FB004083B00224043005
:1099C0000094FFF7BBFF03B030BD00BF38B540F6D1
:1099D000AC63C2F200034FF4197505FB00352C1D72
:1099E00094F86222DAB194F8600228B9002184F870
:1099F0006212D4F8540238BD5878052384F86132D5
:109A00000FF038F928790FF0DBF8002128790FF0F2
:109A100035F8002184F86212D4F8540238BD4FF0B2
:109A2000FF3038BD40F6AC61C2F200014FF419724C
:109A300002FB0013D3F85C02704700BF40F6AC6C29
:109A4000C2F2000C4FF4197202FB00C3C3F85C129F
:109A5000704700BF10B440F6AC6CC2F2000C4FF47B
:109A6000197404FB00C393F86602043348B1032061
:109A700083F86102C3F84812C3F85022012010BCD9
:109A800070474FF0FF30FAE700F1784243F6FF737A
:109A90009A420FD9A2F580429A4201D80820704715
:109AA0004FF4004CCFF2FF7C00EB0C01994203D83D
:109AB00010207047002070474FF48041CFF2FF71B3
:109AC00042189A4201D81820704700F1774303F5F5
:109AD0007F0CBCF5803F01D2202070474FF6FF720B
:109AE00003F57E01C0F20102914201D8282070479F
:109AF00003F57C0C944501D83020704703F57A01BA
:109B0000914201D83820704703F5780C944501D86C
:109B10004020704703F57603934201D848207047F0
:109B200000F1774202F57400B0F5003F2CBF5820D9
:109B3000502070472DE9F0470024C0F60E0400289D
:109B400014BF06462646904689460DF063FAF32078
:109B50000DF07CFA3046FFF797FF044606EB08004D
:109B6000FFF792FF031B02251B07074618D5BC42CF
:109B70002946204624D80DF0BDFA0246082A294677
:109B800020467FD00DF0B6FA08287BD0204602216F
:109B90000DF0B0FA00240DF04FFA2046BDE8F08732
:109BA00084420DD8204629460DF0A4FA082805D095
:109BB000204629460DF09EFA0828E7D10834D6E75A
:109BC000B8F1000F5CD04C46304654F8041B0DF041
:109BD00071FA08F1FF37082807F0010711D054F88F
:109BE000041C30460DF066FA08280AD054F8041C0C
:109BF000304600240DF05EFA0DF01EFA2046BDE856
:109C0000F087002501350436454539D08FB154F829
:109C1000041B30460DF04EFA082806D054F8041CF8
:109C200030460DF047FA0828E0D1013504364545A5
:109C300026D054F8041B30460DF03CFA01460829A2
:109C40003046A14605D054F8041C0DF033FA08281C
:109C5000CCD10436216830460DF02CFA034601358C
:109C6000082B3046374609F1040405D054F8041C8B
:109C70000DF020FA0828B9D101353E1D4545D8D14F
:109C8000012488E70834294620460DF033FA84463B
:109C9000BCF1080F29462046A24604D00DF02AFA4E
:109CA00008287FF473AF0AF1080460E70020C0F6CB
:109CB0000E00704747F61023C1F6FF7353F82000DB
:109CC000704700BF4EF63073CEF200035A6822F0A0
:109CD00000415960586820F080425A60704700BFC8
:109CE0002DE9F00F41F23C03C1F2000390B0197E60
:109CF0004A0700F1DC80DA7AB3F81480DF78B3F831
:109D000006A0DD79B3F8109093F804C01E7A1C7B8E
:109D1000D3F804B058880492DA7B0CF03F0C05921B
:109D2000DA7C4FEA4C1C4CEAD70CCBF38A1BC0F30D
:109D30000A00CAF34A07DDF810A00F92ADF808B088
:109D4000ADF80000E400D3F808B0588944EA5A148A
:109D500006F07F06D3F80CA0360146EA1516CBF3C1
:109D6000CA15C0F38A0BCAF30A20B3F80EA04FEA53
:109D7000C959CAF3CA0AADF818A04FEAD959DDF893
:109D800014A04FEA890949EA9A19D3F810A0CAF336
:109D90004A2AADF820A0B3F812A04FEA8852CAF3BD
:109DA0000A1AADF828A04FEA9258DDF83CA04FEA15
:109DB000480848EADA18D3F814A0CAF38A2AADF89A
:109DC00030A0BDF808A0CAF5D46ACDF808A0BDF847
:109DD00000A0AAF5806ACDF800A04AF6BC12ACF546
:109DE000806AC1F20002CDF810A0DDF808A0BDF82D
:109DF00018C0A2F810A0DDF800A0A7F58067A2F8AF
:109E000012A0DDF810A00597A2F814A0C6F5806690
:109E1000DDF814A00E96A2F816A0C5F58065DDF851
:109E200038A00F95BDF82070BDF82860BDF83050FF
:109E3000A2F818A0DDF83CA0C4F58064C0F58060ED
:109E4000CBF5806BCCF5806CC9F58069C7F5806770
:109E5000C6F58066C8F58068C5F580651084A2F8EF
:109E60001AA0A2F81CB0D483A2F822C0A2F82490B1
:109E7000D7841685A2F82A809585DC8A11F0010F17
:109E80004FF6E0430CBF18464FF44870C4F34A1431
:109E900011F0020F18BF4FF44873C4F58061D185EB
:109EA00010865386012010B0BDE8F00F70474FF0C8
:109EB000FF30F8E741F23C03C1F200031A78012AAF
:109EC00009D003D3022A12D0002070470F284FF088
:109ED000000013D070475A7899180132D2B2172A6D
:109EE00088705A70F0D1022018700020704700224C
:109EF0001A7008B110467047FFF7F2BE01221A70BF
:109F00005870704770B541F23C0000254FF49844FA
:109F100048F2A06686B0C4F2000429461922C0F2B5
:109F20000106C1F2000014F0EBF9202331462A4665
:109F30002046009509F078FA4AF6BC1CC1F2000CE4
:109F4000024602A8CCF804200EF0F2F94FF40051BA
:109F50004FF48060ADF80E10ADF8100004232046D9
:109F600002A90296ADF80C50ADF81450ADF81230BD
:109F70000EF05EF9204601210EF0E6F906B070BD44
:109F800041F2580000210C2270B5C1F2000014F01B
:109F9000B7F940F2AC23C1F2000393EDF17ADFEDA3
:109FA000507AB4EE677AF1EE10FA5ED09FED4D1A5A
:109FB000C1EE070ADFED4C6A20EEA60AD3EDEB6A8C
:109FC000BCEEC07AF4EE676A17EE105AF1EE10FAA2
:109FD000ADB268D1FF2640F2AC23C1F20003D3ED4D
:109FE000EC7AF5EE407AF1EE10FA3FD1FF2432061A
:109FF0001BD440F2AC20C1F20000D0EDF25ABCEE0E
:10A00000E55A294615EE102AF0B24FF0FF3306F05C
:10A010004BF941F25802C1F2000241F6F021C0F6BC
:10A02000020150600846F8F75FFC23061DD440F299
:10A03000AC2EC1F2000E9EEDF37ABCEEC76AE0B220
:10A0400016EE102A29464FF0FF3306F02DF941F2A3
:10A050005803C1F2000341F6103CC0F6020C9860B0
:10A060006046BDE87040F8F73FBC70BDB2EE0C3AF8
:10A07000F4EEC37AF1EE10FAB8D8F7EE004A37EEF4
:10A08000E44AFDEEC43A13EE904AE4B2204606F0EC
:10A0900003F90028ABD041F6C420C0F60200F8F75F
:10A0A00023FCFF24A3E7F2EE0C7AF4EEE76AF1EE6C
:10A0B00010FA8FD8F7EE002A36EEE22AFDEEC21A29
:10A0C00011EE906AF6B2304606F0E6F8002882D02B
:10A0D00041F69820C0F60200F8F706FCFF267AE762
:10A0E000000000000000484300409C4510B541F2CC
:10A0F0005803C1F200032DED028B5A68002A5CD090
:10A1000040F2AC22C1F2000292ED091AFDEEC10A42
:10A110004AF6BC1C10EE901AC1F2000C0831D2EDC8
:10A12000F46A3CF9110000EE100AB8EEC07A4AF267
:10A13000A82187EE267AC1F20001DFED5A7A91ED6F
:10A14000006A06EE277AD3ED007AF4EE477AF1EE54
:10A1500010FA07D037EEC72AD2EDF61A42EE617A2E
:10A16000C3ED007A5048DFED4F5A90ED005A40F2AF
:10A17000AC2E45EE657AC1F2000EDEEDF24A46EEF7
:10A18000A74ADEEDF03A9EEDEF3ABDEEE44AFDEE71
:10A19000E36AFDEEC32A14EE100A12EE902A16EEC0
:10A1A000901A00F019FC4FF4406CC4F2000C42F21B
:10A1B0001073DCF824209A4269D841F25801C1F2A8
:10A1C0000001886800283CD040F2AC24C1F20004B1
:10A1D00094EDF76AB5EE406AF1EE10FA334B33D1E5
:10A1E00093ED034ADFED2F4AD4EDF53A64EE646A4D
:10A1F000D4EDF37A46EEA37AD4EDEE6AD4EDED5ABF
:10A20000BDEEE77ABDEEE66ABDEEE55A17EE100A3E
:10A2100015EE102A16EE101A00F0DEFB4FF4406C1B
:10A22000C4F2000C42F21073DCF824209A4280B28F
:10A2300007D941F2580EC1F2000EDEF8082011686D
:10A240000860BDEC028B10BD93ED038ABDEEC83AE9
:10A2500013EE100A13F0E4FE94EDF72ADFED142A52
:10A26000C2EE820A01EE900AB8EEE11A9FED0D0AE5
:10A27000C1EE207A94EDF57A28EE678AD4EDF37A70
:10A2800028EE008AD4EDEE6A48EE077AB6E741F28E
:10A29000580CC1F2000C81B2DCF804301A6811606D
:10A2A0008BE700BF00007A44C0210020B8210020C5
:10A2B0000000C84238B540F2201441F26803C1F2F0
:10A2C0000004C1F20003D4F87841D3F8A05049F259
:10A2D0008062611BC0F298029142054637D993F81B
:10A2E0002440621C5FFA82FC4FFA8CF1881C83F8D0
:10A2F00024C053F820205AB341F26804C1F200048C
:10A3000041F63030C0F60200F8F7EEFA94F9242056
:10A31000911C284654F8211009F0EEF90BF05AFC74
:10A3200040F2AC2CC1F2000C9CED3B0AFCEEC07A72
:10A33000284617EE901A09F0DFF90BF003FC40F203
:10A340002010C1F20000D0F87831C4F8A03038BD38
:10A3500083F82420D0E700BF70B5204D20486C68FA
:10A36000F8F7C2FA0BF024FC0A200FF0E3FA2046BB
:10A37000FFF7A0FFAB6A1A689B8851690B420CBFBC
:10A380000026012606B91383204609F07BF9024610
:10A390002046A2B109F084F9C0B20BF081FD01287A
:10A3A00014D0022816D00328EED12046FFF782FFF2
:10A3B000204609F067F902462046002AEAD1002E1D
:10A3C000D2D1A96A08688E884683CDE7A8780EF0B6
:10A3D00051FCD9E768780EF04DFCD5E76810001005
:10A3E0004C1B0208F0B541F6643041F2680489B0B4
:10A3F000C1F20004C0F6020040F2AC27F8F774FA8C
:10A40000C1F20007A8220021204613F079FF97ED42
:10A410003B1A4FF416524FF48056FCEEC10AC4F2B8
:10A420000206E2604FF461334FF4E132002501216E
:10A430003046236162614FF496434FF41642C4EDF7
:10A44000020AA361E261256284F82450FEF774FBDE
:10A4500097ED3B0AB0F804C0D0F800E0A062FCEE33
:10A46000C07A4FF400774FF49040AEF81AC017EE60
:10A47000901A2A463B46C4F20000009708F0D4FF29
:10A4800029460746284667600EF072FA29460346B9
:10A49000284663700EF06CFA41F670310246C0F641
:10A4A00002016820A27000F01DFA41F6FC47C2F2DA
:10A4B000000786464AF259300EF5CE73C7F800E021
:10A4C00046F623022946C0F600000FF00FF90346B6
:10A4D00003A8237002270CF005FF304603A9039759
:10A4E0008DF810508DF813500CF040FE012104201F
:10A4F0000DF09AFA0126082205A88DF81920059773
:10A500008DF818508DF81A600CF03AFD072107A855
:10A510008DF81C108DF81D508DF81E508DF81F60A1
:10A520000CF02EFA4FF410534FF47842C4F6741323
:10A53000C7F64222A3662365E364C4F8A42009B0E9
:10A54000F0BD00BF10B44FF4406141F26803C4F2A3
:10A550000001C1F20003496AD3F8944048F20F1C8D
:10A560000C1BCFF6F17C48F29E6004EB0C02C0F2AB
:10A570000100824207D8D3F8A420A2EBC424A2EBA6
:10A580006410C3F8A40041F26803C1F20003D3F8D9
:10A590009000C3F89410C3F88C00022010BC0CF09B
:10A5A00033BD00BF4FF48660704700BF00B541F671
:10A5B000943083B041F6A031C0F6020101AAC0F682
:10A5C000020013F03DFE42F62D30C0F2331003B00E
:10A5D00000BD00BF2DE9F04F2DED028B840089B046
:10A5E0000E34064600AF24F00700ADEB000DC7F8AF
:10A5F0000CD040F22014ADEB000DC7F808D04FF09E
:10A600000008ADEB000DC1F200049FED328A3E6000
:10A61000C7F804D04546A146D4F87821D4F878315B
:10A620009342FBD0D9F83011D9F83401D9F8382148
:10A630009346FA684FEA880302EB030C8A467A686D
:10A64000B968CCF800A008F10108C918D318B542C0
:10A6500098FBF6F20860C3F800B006FB128826DA11
:10A66000D4ED610AB7EE007A87EE200A0135FDEEDF
:10A67000C07A17EE90CA0CEB8C00854210DAAE421D
:10A68000CADAD7ED062A97ED053A97ED072A73EE59
:10A69000221A31EE821AB4EEC81AF1EE10FABBDCBF
:10A6A00007F12407BD46BDEC028BBDE8F08FF868CA
:10A6B000396807F114020FF055FC3968B86807F1E2
:10A6C00018020FF04FFC7868396807F11C020FF090
:10A6D00049FCC5E7CDCC4C3D10B540F2AC23C1F2EE
:10A6E00000032DED028BDFED0C7A93ED968A28EEB8
:10A6F000278A41F21014B0EE480A13F045FBC1F26C
:10A70000000484ED010AB0EE480A12F0A5FF84EDC2
:10A71000020ABDEC028B10BD35FA8E3C10B541F239
:10A720001014C1F2000414220021204613F0E8FDA9
:10A73000002101200EF01CF90021034601202370A6
:10A740000EF016F96070FFF7C7FFBDE81040F6F78E
:10A75000EBBF00BF41F21013C1F200031969187872
:10A760004A1C1A610EF086BA41F21013C1F20003BE
:10A77000D96858784A1CDA600EF07CBA2DE9F047A7
:10A7800041F6A859C2F20009D9F80030002B3DDD8E
:10A7900041F2241AC1F2000A0024AAF102070AF1C8
:10A7A0002006254637F8020F002843D00AF1800121
:10A7B00061580A78FF2A3FD1002310F0010F0A46A2
:10A7C00013D10123834213DA91F801C0BCF1FF0FCA
:10A7D00001EB030209D00BE012F8011FFF2907D19A
:10A7E00012F8011F0133FF2902D101338342F3DB49
:10A7F00036F8022B9A42C8BF26F8023C0F2B07DD21
:10A80000D9F8003001350434AB42CBDCBDE8F08729
:10A810000AF1400041F60458C2F2000841F6B03196
:10A820002258C0F60201404613F0F4FC4046F8F707
:10A830005BF8E5E70346DBE70023D9E770B50C4694
:10A84000054613F083FC41F60053C2F2000341F6C3
:10A85000AC52C2F2000206461868116805FB0404F7
:10A860008C421C6088BF14600EB1304670BD41F64A
:10A87000D030C0F60200F8F737F8304670BD00BFA0
:10A8800038B50C46154648B113F070FC41F600533C
:10A89000C2F200031A6804FB15241C6038BD00BF17
:10A8A00038B541F64454C2F2000401FB00F1CD1C5E
:10A8B0002068AD082818B0F5105F05D8084B206057
:10A8C000421B03EB820038BD41F6E830C0F60200BF
:10A8D000F8F70AF82068024B421B03EB820038BDF0
:10A8E000E4110010F8B58700BDB20E4601202946DC
:10A8F000FFF7D6FFFF213A46044613F001FD41F66B
:10A90000A852C2F2000241F224131168C1F20003FE
:10A9100003EB810003EB410C4F1CC0F88040066440
:10A9200023F81150ACF8205017602046F8BD00BF46
:10A930004FF44063C4F20003596A5A6A40189042C7
:10A9400042D900BF00BF00BF00BF00BF00BF00BFB3
:10A9500000BF00BF00BF00BF00BF00BF00BF00BFFF
:10A9600000BF00BF00BF00BF00BF00BF00BF00BFEF
:10A9700000BF00BF00BF00BF00BF00BF00BF00BFDF
:10A9800000BF00BF00BF00BF00BF00BF00BF00BFCF
:10A9900000BF00BF00BF00BF00BF00BF00BF00BFBF
:10A9A00000BF00BF00BF00BF00BF00BF00BF00BFAF
:10A9B00000BF00BF00BF00BF00BF00BF00BF00BF9F
:10A9C00000BF5A6A9042BCD8704700BF4FF47A73F8
:10A9D00003FB00F0FFF7ACBF884203DB8242B4BF49
:10A9E0001146014608467047B4EEE00AF1EE10FA4F
:10A9F00008D4B4EEC10AF1EE10FAD4BFF0EE400A6A
:10AA0000F0EE410AB0EE600A704700BF30B583B087
:10AA10000546FFF7CBFD0446FFF7C4FD022341F6D0
:10AA2000FC3141F6204200900193C0F60201C0F6CD
:10AA300002022846234613F0EDFB03B030BD00BFF1
:10AA4000F0B5642083B00EF075FF0220FFF732F9F5
:10AA500006460120FFF72EF907460020FFF72AF9E6
:10AA600041F64854C2F2000441F62C413B463246BE
:10AA7000C0F6020105462046009513F0CBFB2046A8
:10AA8000F7F732FF64200EF055FF0020FFF712F9B0
:10AA900044F6D351C1F26201A1FB0012FA2312095C
:10AAA00041F6444103FB1202C0F60201204613F0B6
:10AAB000B1FB2046F7F718FF64200EF03BFF42F28F
:10AAC0000C2CC2F2000C4DF68360DCF80030C4F2AE
:10AAD0001B30A0FB031241F65841920CC0F6020154
:10AAE000204613F097FB2046F7F7FEFE64200EF099
:10AAF00021FF41F60051C2F2000141F6AC50C2F212
:10AB000000000A68036841F66C41C0F60201204665
:10AB100013F080FB2046F7F7E7FE64200EF00AFFF3
:10AB200041F64453C2F2000341F688411A68C0F668
:10AB3000020192004FF41043204613F06BFB2046B5
:10AB4000F7F7D2FE64200EF0F5FE2046FFF75EFF19
:10AB50002046F7F7C9FE642003B0BDE8F0400EF0D0
:10AB6000E9BE00BFC0EE200A80ED011AC0ED000A68
:10AB7000704700BFC0EE200A80ED011AC0ED000A48
:10AB8000C0ED020A80ED031AC0ED040A80ED051A3B
:10AB9000704700BFD0ED057A90ED042A30EE670AC9
:10ABA000D0ED030A40EE027AD0ED021A37EEE01A39
:10ABB00090ED010A41EE210AD0ED006A30EEC06A44
:10ABC000C0ED057A06EE260AC0ED030A80ED010A03
:10ABD000704700BFD0ED017A90ED007A30EE670A41
:10ABE00040EE077AB0EE670AC0ED017A704700BF09
:10ABF0000A6802604B684360082070470B68036076
:10AC0000042070470B880380022070470B78037084
:10AC100001207047F8B54AF2E414C1F2000494F937
:10AC20000B00FEF7FFFE2268412317181354054658
:10AC3000712148207970B870A67A40F26461FE7084
:10AC4000381DC2F20001C82213F03CFB2268002626
:10AC5000EB1CD218374633463146581C12F806E032
:10AC600012F800C071449C1CCEB206EB0C00145DBF
:10AC70005FFA80FE06EB070C0EEB04015EFA8CF621
:10AC80000333C9B251FA86F4C92BE7B21E46E4D1A8
:10AC90004AF2E41EC1F2000E82F8C910BEF8084064
:10ACA0009EF90B0082F8CA70C821651901FB04F3F4
:10ACB00095FBF3FC03FB1C51BDE8F840FEF7BEBE5C
:10ACC000F8B54AF2E416C1F2000696F90B00FEF759
:10ACD000A9FE3468412225182254074671214D20CF
:10ACE0006970A870B37A83B103350024706800EBF3
:10ACF000C40E50F83410DEF804302846984796F811
:10AD00000AC00134A4450544F0DC4AF2E415C1F25E
:10AD100000052E892968B51E032D39443CDDCA780B
:10AD20000423AB4205F00100D4B21EDA48B111F899
:10AD300003C002EB0C00C2B205231419AB42E4B20B
:10AD400013DA11F803C0013302EB0C0011F803E031
:10AD50005FFA80FC0CEB0E020CEB0400D2B2013364
:10AD600052FA80F4AB42E4B2EBDB013E4AF2E41E5D
:10AD70004A55C1F2000E8C55BEF808209EF90B0012
:10AD8000C821D71901FB02F397FBF3F103FB117103
:10AD9000BDE8F840FEF752BE0024042603252246F3
:10ADA000E4E700BF2DE9F04F4AF2E414C1F20004D9
:10ADB000642305221846A3728BB008212281FFF775
:10ADC0006FFDA37A6060002B00F0CB8041F6B85590
:10ADD000C2F200054AF6FD37D5F83C842589CDF846
:10ADE000048008F1340308F138024AF6F136029380
:10ADF000039208F13C0308F10C02C0F60007C0F60C
:10AE000000064AF60D4C4AF6054B0493059208F1EC
:10AE1000100308F11402B646C0F6000C002140F2FF
:10AE2000646408F1300A0693079208F1040308F1FC
:10AE3000080208F14009C0F6000BB84608936646C0
:10AE40000992F4460B46C2F200045F46C64614F867
:10AE500013209B46632A67D8DFE812F04F024C02AA
:10AE600049024602430240023D023A0237023402DE
:10AE700031022E022B022802250222021F021C028E
:10AE800019021602130210020D020A02070204023E
:10AE90000102FE01FB01F801F501F201EF01EC01F5
:10AEA000E901E601E301E0017801750172016F013A
:10AEB0006C0169016601630160015D015A0157017E
:10AEC000540151014E014B014801450142013F012E
:10AED0003C0139013601330130012D012A012701DE
:10AEE000240121011E011B011801150112010F018E
:10AEF0000C010901060103010001FD00FA00F70041
:10AF0000F400F100EE00EB00E800E500E200DF00F5
:10AF1000DC00D900D600D300D000CD00CA00C700A5
:10AF2000C40064008B4A425004EB4B0898F801B00F
:10AF3000BBF1070F09D8DFE80BF032202020434394
:10AF40000404421801355660ADB24AF2E412C1F26F
:10AF50000002013392F80AB008319B453FF777AF02
:10AF600015814AF2E414C1F20004C8202189FFF7D8
:10AF700065FC20600BB0BDE8F08F00EB010B4AF2DE
:10AF8000E412C1F20002CBF804E092F80AB00133F7
:10AF9000043508319B45ADB23FF759AFE0E74218A1
:10AFA0000133C2F804C04AF2E412C1F200020835CB
:10AFB00092F80AB008319B45ADB23FF748AFCFE7F2
:10AFC00000EB01084AF2E412C1F20002C8F8047072
:10AFD00092F80AB00133023508319B45ADB23FF714
:10AFE00036AFBDE75C4A42509EE75C4A42509BE761
:10AFF0005B4A425098E75B4A425095E75A4A4250B2
:10B0000092E75A4A42508FE7594A42508CE7594AD0
:10B01000425089E7584A425086E7584A425083E7EF
:10B02000574A425080E7574A42507DE7564A4250BD
:10B030007AE7564A425077E7554A425074E7554AF4
:10B04000425071E7544A42506EE7544A42506BE70F
:10B05000534A425068E7534A425065E7524A4250C9
:10B0600062E7524A42505FE7514A42505CE7514A18
:10B07000425059E7504A425056E7504A425053E72F
:10B080004F4A425050E74F4A42504DE74E4A4250D5
:10B090004AE74E4A425047E74D4A425044E74D4A3C
:10B0A000425041E74C4A42503EE74C4A42503BE74F
:10B0B0004B4A425038E74B4A425035E74A4A4250E1
:10B0C00032E7099A42502FE7089A42502CE7019A3A
:10B0D000425029E740F8019026E740F8019023E725
:10B0E000079A425020E7069A42501DE7059A4250BF
:10B0F0001AE7049A425017E7039A425014E7029A5B
:10B10000425011E740F801A00EE7384A42500BE7E1
:10B11000374A425008E7374A425005E7364A42501C
:10B1200002E7364A4250FFE6354A4250FCE6354ACD
:10B130004250F9E6344A4250F6E6344A4250F3E6C9
:10B14000334A4250F0E6334A4250EDE6324A42502A
:10B15000EAE600BFF0A90010EEA90010ECA900106B
:10B16000EAA90010E8A90010E6A90010E4A900105F
:10B17000E2A90010E0A90010DEA90010DCA900106F
:10B18000DAA90010D8A90010D6A90010D4A900107F
:10B19000D2A90010D0A90010CEA90010CCA900108F
:10B1A000F4A9001088A2001084A2001080A2001050
:10B1B0008CA2001046A2001044A2001042A200106F
:10B1C00040A200103EA200103CA200103AA20010C3
:10B1D00038A2001036A2001034A2001032A20010D3
:10B1E00030A200102EA200102CA20010A802001005
:10B1F0002402001018020010140200102002001097
:10B20000300200102C020010D0100010C4100010EA
:10B21000C0100010BC10001004110010384A425039
:10B2200082E6384A42507FE6374A42507CE6374A47
:10B23000425079E6364A425076E6364A425073E644
:10B24000354A425070E6354A42506DE6344A425023
:10B250006AE6344A425067E6334A425064E6334A6B
:10B26000425061E6324A42505EE6324A42505BE664
:10B27000314A425058E6314A425055E6304A42502F
:10B2800052E6304A42504FE62F4A42504CE62F4A8F
:10B29000425049E62E4A425046E62E4A425043E684
:10B2A0002D4A425040E62D4A42503DE62C4A42503B
:10B2B0003AE62C4A425037E62B4A425034E62B4AB3
:10B2C000425031E62A4A42502EE62A4A42502BE6A4
:10B2D000294A425028E6294A425025E6284A425047
:10B2E00022E6284A42501FE6274A42501CE6274AD7
:10B2F000425019E6264A425016E6264A425013E6C4
:10B30000B8100010B4100010B0100010A8100010F9
:10B31000A01000100011001098100010EC10001088
:10B32000E8100010E4100010E0100010DC10001015
:10B33000D810001064020010600200105C020010BF
:10B340005802001054020010500200104C0200106D
:10B350004802001044020010100200100C020010FD
:10B36000080200100402001000020010FC0100108E
:10B37000F8010010F4010010F0010010EC010010C1
:10B38000E8010010E4010010E0010010DC010010F1
:10B39000D80100109802001010B54AF2E414C1F26E
:10B3A000000400210C22204612F0AAFFFFF7FAFC4D
:10B3B00041F6BC40C0F60200FEF772FA238921680C
:10B3C000E072C82202FB03F2FEF744FBBDE8104026
:10B3D000FFF720BC38B5FEF775FC05F015FC4FF4FF
:10B3E000A0600BF0C3FA0DF011F941F6C041C0F6B0
:10B3F00002014FF4C870FFF775FA40F68004054665
:10B4000000F5C663C2F2000442F22D6049F20C025C
:10B41000C0F201020C330021C0F6000025600EF0DE
:10B4200065F90DF03BF9002038BD00BFF0B54EF6D0
:10B43000FC54CEF200044FF480532568CEF2000392
:10B4400045F080712160186841F6B05440F0010267
:10B4500041F2040740F22C7683B01A600025C2F254
:10B460000004CEF20007C2F20006FFF787F9206859
:10B47000431C23603B68591B01910198326890423C
:10B4800001D2019D35601D46EFE700BF08B500F011
:10B4900071FAFEE710B54AF2F014C1F2000494F814
:10B4A000A430002B75D14AF2F014C1F2000494F8D4
:10B4B000A500002840F090804AF2F014C1F2000488
:10B4C00094F8A600002840F0AA804AF2F014C1F2D5
:10B4D000000494F8A700002840F0C5804AF2F01458
:10B4E000C1F2000494F8A800002840F0E0804AF27D
:10B4F000F014C1F2000494F8A900002840F0FB8089
:10B500004AF2F014C1F2000494F8AA00002840F0B6
:10B5100016814AF2F014C1F2000494F8AB0000283E
:10B5200040F031814AF2F014C1F2000494F8AC000A
:10B53000002840F04C814AF2F014C1F2000494F863
:10B54000AD00002840F067814AF2F014C1F2000417
:10B5500094F8AE00002840F082814AF2F014C1F263
:10B56000000494F8AF00002840F09D814AF2F014E6
:10B57000C1F2000494F8B000002840F0B8814AF20B
:10B58000F014C1F2000494F8B100002840F0D38117
:10B5900010BD40F2AC2CC1F2000CDCED3E0A9CED7B
:10B5A000400ABDEEE07AFDEEC07AB4F93C0017EE39
:10B5B000101A17EE902AFFF70FFA636882B2196823
:10B5C000A2874AF2F01410B2C1F20004086094F8A5
:10B5D000A50000283FF470AF40F2AC2EC1F2000E7F
:10B5E000DEED3E2ADEED401ABDEEE22ABDEEE11AA6
:10B5F000B4F93E0012EE101A11EE102AFFF7ECF922
:10B60000A36882B21968E28714B20C604AF2F0149F
:10B61000C1F2000494F8A60000283FF456AF40F2AF
:10B62000AC2CC1F2000CDCED3E4ADCED403ABDEE44
:10B63000E44ABDEEE33AB4F9400014EE101A13EEFA
:10B64000102AFFF7C9F9E36882B21968A4F840200C
:10B6500014B20C604AF2F014C1F2000494F8A7008E
:10B6600000283FF43BAF40F2AC2EC1F2000EDEEDFD
:10B670003E6ADEED405ABDEEE66ABDEEE55AB4F92B
:10B68000420016EE101A15EE102AFFF7A5F92369ED
:10B6900082B21968A4F8422014B20C604AF2F01485
:10B6A000C1F2000494F8A80000283FF420AF40F253
:10B6B000AC2CC1F2000CDCED3E0A9CED400ABDEE64
:10B6C000E07AFDEEC07AB4F9440017EE101A17EED6
:10B6D000902AFFF781F9636982B21968A4F84420BF
:10B6E00014B20C604AF2F014C1F2000494F8A900FC
:10B6F00000283FF405AF40F2AC2EC1F2000EDEEDA3
:10B700003E2ADEED401ABDEEE22ABDEEE11AB4F9A2
:10B71000460012EE101A11EE102AFFF75DF9A36928
:10B7200082B21968A4F8462014B20C604AF2F014F0
:10B73000C1F2000494F8AA0000283FF4EAAE40F2F7
:10B74000AC2CC1F2000CDCED3E4ADCED403ABDEE23
:10B75000E44ABDEEE33AB4F9480014EE101A13EED1
:10B76000102AFFF739F9E36982B21968A4F8482072
:10B7700014B20C604AF2F014C1F2000494F8AB0069
:10B7800000283FF4CFAE40F2AC2EC1F2000EDEED49
:10B790003E6ADEED405ABDEEE66ABDEEE55AB4F90A
:10B7A0004A0016EE101A15EE102AFFF715F9236A53
:10B7B00082B21968A4F84A2014B20C604AF2F0145C
:10B7C000C1F2000494F8AC0000283FF4B4AE40F29B
:10B7D000AC2CC1F2000CDCED3E0A9CED400ABDEE43
:10B7E000E07AFDEEC07AB4F94C0017EE101A17EEAD
:10B7F000902AFFF7F1F8636A82B21968A4F84C2026
:10B8000014B20C604AF2F014C1F2000494F8AD00D6
:10B8100000283FF499AE40F2AC2EC1F2000EDEEDEE
:10B820003E2ADEED401ABDEEE22ABDEEE11AB4F981
:10B830004E0012EE101A11EE102AFFF7CDF8A36A8F
:10B8400082B21968A4F84E2014B20C604AF2F014C7
:10B85000C1F2000494F8AE0000283FF47EAE40F23E
:10B86000AC2CC1F2000CDCED3E4ADCED403ABDEE02
:10B87000E44ABDEEE33AB4F9500014EE101A13EEA8
:10B88000102AFFF7A9F8E36A82B21968A4F85020D9
:10B8900014B20C604AF2F014C1F2000494F8AF0044
:10B8A00000283FF463AE40F2AC2EC1F2000EDEED94
:10B8B0003E6ADEED405ABDEEE66ABDEEE55AB4F9E9
:10B8C000520016EE101A15EE102AFFF785F8236BBA
:10B8D00082B21968A4F8522014B20C604AF2F01433
:10B8E000C1F2000494F8B00000283FF448AE40F2E2
:10B8F000AC2CC1F2000CDCED3E0A9CED400ABDEE22
:10B90000E07AFDEEC07AB4F9540017EE101A17EE83
:10B91000902AFFF761F8636B82B21968A4F854208B
:10B9200014B20C604AF2F014C1F2000494F8B100B1
:10B9300000283FF42DAE40F2AC2EC1F2000EDEED39
:10B940003E2ADEED401ABDEEE22ABDEEE11A12EE0D
:10B95000101A11EE102AB4F95600FFF73DF8A36B48
:10B960001FFA80FC1A68A4F856C00FFA8CF1116017
:10B9700010BD00BF40F2AC23C1F2000310B493ED40
:10B980003F0A4AF2F011C1F20001FDEEC07A91F8CF
:10B99000A44017EE900A034602B21CB14C68888797
:10B9A00021680A604AF2F011C1F2000191F8A50085
:10B9B00018B18868CB8701680A604AF2F011C1F2B9
:10B9C000000191F8A60020B1C868A1F840300168D4
:10B9D0000A604AF2F011C1F2000191F8A70020B10B
:10B9E0000869A1F8423001680A604AF2F011C1F218
:10B9F000000191F8A80020B14869A1F8443001681D
:10BA00000A604AF2F011C1F2000191F8A90020B1D8
:10BA10008869A1F8463001680A604AF2F011C1F263
:10BA2000000191F8AA0020B1C869A1F84830016866
:10BA30000A604AF2F011C1F2000191F8AB0020B1A6
:10BA4000086AA1F84A3001680A604AF2F011C1F2AE
:10BA5000000191F8AC0020B1486AA1F84C300168AF
:10BA60000A604AF2F011C1F2000191F8AD0020B174
:10BA7000886AA1F84E3001680A604AF2F011C1F2FA
:10BA8000000191F8AE0020B1C86AA1F850300168F9
:10BA90000A604AF2F011C1F2000191F8AF0020B142
:10BAA000086BA1F8523001680A604AF2F011C1F245
:10BAB000000191F8B00020B1486BA1F85430016842
:10BAC0000A604AF2F011C1F2000191F8B10020B110
:10BAD000886BA1F8563003681A604AF2F01CC1F274
:10BAE000000C0022CCF89C20CCF8A02010BC7047A1
:10BAF00038B54AF2F015C1F200052DED068BD5EDF3
:10BB0000283A9FEDEEAA40F2AC24C1F20004B0EE58
:10BB1000608AF0EE418AF0EE4A0A94ED401A30EE67
:10BB2000630AB0EE619AFEF75FFF94ED413AD4EDFF
:10BB3000422AF0EE409A33EE400AD4ED430A94EDE7
:10BB4000441A20EE220AFEF74FFF40F22013C1F202
:10BB5000000393ED422ADFEDDA1A93ED411A62EE0B
:10BB6000217A95F8A4202B6877EEC10AB7EE007A07
:10BB700080EEA76A08EE008A36EE076A48EE808AF1
:10BB800009EE009AD4ED3E6A94ED407AD5ED287A1C
:10BB900082B3D3ED005A9FEDCB1A69EEA53A93ED2F
:10BBA000013A03EE81AA68EE032A93ED020A02EE3F
:10BBB00081AA28EE802AD3ED031A02EE01AA69EECB
:10BBC000210AF0EE664A00EE81AA4AEE064ABDEE70
:10BBD000E44A14EE100A01B205EE101AF8EEC55A46
:10BBE000A887F4EE475AF1EE10FA04BFDFEDB65A1B
:10BBF00077EEA57A4AF2F012C1F2000292F8A5405F
:10BC0000A4B3D3ED044A9FEDAF0A29EEA44ADFEDB9
:10BC1000AB1A93ED055A44EE001A68EE055AD3EDBF
:10BC2000063A45EE801A28EEA33AD3ED072A43EEF2
:10BC3000001A29EE222AB0EE661A42EE001A01EE30
:10BC4000861AFDEEC14A14EE90CA0FFA8CFE04EE7D
:10BC500010EAB8EEC45AA2F83EC0B4EE475AF1EE6C
:10BC600010FA04BF9FED985A77EE857A4AF2F012E7
:10BC7000C1F2000292F8A60098B3D3ED081ADFEDE6
:10BC8000913A29EEA11ADFED8D2AD3ED090A41EE92
:10BC9000232A68EE204A93ED0A4A44EEA32A28EEAE
:10BCA000845AD3ED0B5A45EE232A29EE253AB0EEFD
:10BCB000660A43EE232A02EE860AFDEEC01A11EE52
:10BCC000901A0CB201EE104AF8EEC10AA2F8401028
:10BCD000F4EE470AF1EE10FA04BFDFED7B0A77EECF
:10BCE000A07A4AF2F012C1F2000292F8A700A0B3C3
:10BCF000D3ED0C2A9FED735A29EEA20ADFED6F5A9D
:10BD000093ED0D2A40EE055A68EE021A93ED0E1AD5
:10BD100041EE855A68EE810AD3ED0F4A40EE855A0E
:10BD200029EE244AF0EE663A44EE055A45EE863A8C
:10BD3000FDEEE32A12EE90CA0FFA8CF100EE101A13
:10BD4000B8EEC02AA2F842C0B4EE472AF1EE10FACB
:10BD500004BF9FED5D2A77EE827A4AF2F012C1F2BB
:10BD6000000292F8A840A4B3D3ED105A9FED551AE3
:10BD700069EEA53ADFED510A93ED113A43EE810ADF
:10BD800068EE032A93ED120A42EE810A28EE802A19
:10BD9000D3ED131A42EE010A69EE214AB0EE665A5B
:10BDA00044EE810A00EE865AFDEEC55A15EE90EA81
:10BDB0000FFA8EF003EE900AB8EEE33AA2F844E0F0
:10BDC000B4EE473AF1EE10FA04BF9FED3F3A77EE3A
:10BDD000837A4AF2F012C1F2000292F8A910A1B3DC
:10BDE000D3ED140A9FED370A29EEA04ADFED331A8E
:10BDF00093ED155A44EE001A68EE055AD3ED163A43
:10BE000045EE801A28EEA33AD3ED172A43EE001A26
:10BE100029EE222AB0EE661A42EE001A01EE861AC8
:10BE2000FDEEC10A10EE904A0FFA84FC05EE10CA2E
:10BE3000B8EEC54AA2F84640B4EE474AF1EE10FA11
:10BE400004BF9FED214A77EE847A4AF2F012C1F2E4
:10BE5000000292F8AA0000283FD0D3ED181ADFEDB7
:10BE6000193A29EEA11ADFED152AD3ED194A41EE50
:10BE7000232A68EE240A93ED1A4A40EEA32A28EEFC
:10BE8000845AD3ED1B5A45EE232A29EE253AB0EE0B
:10BE9000660A43EE232A02EE860AFDEEC01A11EE70
:10BEA00090EA0FFA8EF101EE101AF8EEC14AA2F8EC
:10BEB00048E0F4EE474AF1EE10FA09E00000000015
:10BEC000CDCC6C400AD7233C9A99993E00000000E3
:10BED00004BF5FED034A77EEA47A4AF2F012C1F292
:10BEE000000292F8AB40A4B3D3ED1C2A1FED0B5A0D
:10BEF00029EEA20A5FED0B5A93ED1D2A40EE055A7A
:10BF000068EE021A93ED1E1A41EE855A68EE814AD8
:10BF1000D3ED1F0A44EE855A29EE204AF0EE663A28
:10BF200044EE055A45EE863AFDEEE32A12EE90CA3B
:10BF30000FFA8CF000EE100AB8EEC02AA2F84AC040
:10BF4000B4EE472AF1EE10FA04BF1FED212A77EE76
:10BF5000827A4AF2F012C1F2000292F8AC10A1B358
:10BF6000D3ED205A1FED291A69EEA53A5FED290A93
:10BF700093ED213A43EE810A68EE032A93ED220AFB
:10BF800042EE810A28EE802AD3ED231A42EE010AFE
:10BF900069EE214AB0EE665A44EE810A00EE865AF6
:10BFA000FDEEC55A15EE904A0FFA84FE03EE90EAB4
:10BFB000B8EEE33AA2F84C40B4EE473AF1EE10FA8C
:10BFC00004BF1FED3F3A77EE837A4AF2F012C1F2D6
:10BFD000000292F8AD00A0B3D3ED240A1FED470A8A
:10BFE00029EEA04A5FED471A93ED255A44EE001A58
:10BFF00068EE055AD3ED263A45EE801A28EEA33AAC
:10C00000D3ED272A43EE001A29EE222AB0EE661A53
:10C0100042EE001A01EE861AFDEEC10A10EE90CA39
:10C020000FFA8CF105EE101AB8EEC54AA2F84EC010
:10C03000B4EE474AF1EE10FA04BF1FED5D4A77EE09
:10C04000847A4AF2F012C1F2000292F8AE40A4B330
:10C05000D3ED281A5FED653A29EEA11A5FED652A46
:10C06000D3ED294A41EE232A68EE240A93ED2A4AA9
:10C0700040EEA32A28EE845AD3ED2B5A45EE232A0C
:10C0800029EE253AB0EE660A43EE232A02EE860A2E
:10C09000FDEEC01A11EE90EA0FFA8EF001EE100AD2
:10C0A000F8EEC14AA2F850E0F4EE474AF1EE10FA79
:10C0B00004BF5FED7B4A77EEA47A4AF2F012C1F238
:10C0C000000292F8AF10A1B3D3ED2C2A1FED835AD2
:10C0D00029EEA20A5FED835A93ED2D2A40EE055A10
:10C0E00068EE021A93ED2E1A41EE855A68EE814AE7
:10C0F000D3ED2F0A44EE855A29EE204AF0EE663A37
:10C1000044EE055A45EE863AFDEEE32A12EE904AD9
:10C110000FFA84FC00EE10CAB8EEC02AA2F8524012
:10C12000B4EE472AF1EE10FA04BF1FED992A77EE1C
:10C13000827A4AF2F012C1F2000292F8B000A0B383
:10C14000D3ED305A1FEDA11A69EEA53A5FEDA10AB1
:10C1500093ED313A43EE810A68EE032A93ED320AF9
:10C1600042EE810A28EE802AD3ED331A42EE010A0C
:10C1700069EE214AB0EE665A44EE810A00EE865A14
:10C18000FDEEC55A15EE90EA0FFA8EF103EE901A05
:10C19000B8EEE33AA2F854E0B4EE473AF1EE10FA02
:10C1A00004BF1FEDB73A77EE837A4AF2F012C1F27C
:10C1B000000292F8B1408CB3D3ED343A1FEDBF5A70
:10C1C00029EEA33A5FEDBF0AD3ED352A43EE050A07
:10C1D00028EE220A93ED362A40EE050A68EE821A0E
:10C1E00093ED371A41EE850A69EE014A44EE850A5D
:10C1F00040EE866ABDEEE64A14EE103A18B206EE3C
:10C20000100AF8EEC66AA2F85630F4EE476AF1EE6C
:10C2100010FA04BF1FEDD47A77EE877A4AF2F01451
:10C22000C1F20004C4ED287AFFF734F940F2AC22E1
:10C23000C1F20002D4ED285A92ED407A5FEDDE6A39
:10C24000F6EE007A35EEE60A5FEDE00A27EE271AF1
:10C25000FEF7CAFB84ED248A84ED280AC4ED258A02
:10C2600084ED269AC4ED279ABDEC068B38BD00BF3D
:10C2700010B541F6C8402DED048BC0F60200F6F76C
:10C2800033FB4AF2F0100021B422C1F2000012F098
:10C2900037F840F2AC23C1F20003D3ED3D7A9FEDB5
:10C2A000E67AF4EEC77AF1EE10FA07DD9FEDE00AC8
:10C2B000F4EEC07AF1EE10FA00F1738440F2AC2390
:10C2C000C1F200039FEDDB8AD3ED457A4AF2F0120A
:10C2D000C1F20002F4EE487A03F58A71F1EE10FA29
:10C2E000116007D193ED462AB4EE482AF1EE10FA18
:10C2F00000F02C8440F2AC24C1F20004D4ED3E1ACC
:10C30000BCEEE11A002011EE102A40F6C4110346DB
:10C3100003F0CAFF4AF2F01CDFEDC60AC1F2000CBE
:10C32000D4ED468A94ED479A94ED488ACCF80400FF
:10C3300078EEA08A012039EE209A38EE208A8CF817
:10C34000A4004AF2F01EC1F2000EDFEDBA7ADEF868
:10C350000040D4ED043AF4EE673AF1EE10FA07D15A
:10C3600094ED056AB4EE676AF1EE10FA00F0DD8331
:10C3700040F2AC22C1F20002D2ED3E5ABCEEE55AC8
:10C3800040F6C411002315EE102A012003F08CFFA3
:10C390004AF2F013C1F20003012183F8A510D4ED95
:10C3A000056AD4ED064A94ED074A78EEA68A39EE7E
:10C3B000249A38EE048A98604AF2F010C1F2000024
:10C3C000DFED9C7A0468D4ED080AF4EE670AF1EE1A
:10C3D00010FA07D194ED093AB4EE673AF1EE10FA8B
:10C3E00000F0928340F2AC2EC1F2000EDEED3E2A48
:10C3F000BCEEE22A002312EE102A022040F6C411FD
:10C4000003F052FF4AF2F01CC1F2000C01238CF839
:10C41000A630D4ED091A94ED0A1AD4ED0B7A78EE11
:10C42000A18A39EE019A38EE278ACCF80C004AF23C
:10C43000F014C1F20004DFED7F7A2468D4ED0C4AD9
:10C44000F4EE674AF1EE10FA07D194ED0D0AB4EE5E
:10C45000670AF1EE10FA00F0468340F2AC20C1F218
:10C46000000090ED3E7ABCEEC76A40F6C41116EEAD
:10C47000102A0320002303F017FF4AF2F011C1F243
:10C480000001012281F8A720D4ED0D6AD4ED0E5AE7
:10C4900094ED0F5A78EEA68A39EE259A38EE058A81
:10C4A00008614AF2F01CC1F2000CDFED627ADCF8A0
:10C4B0000040D4ED101AF4EE671AF1EE10FA07D12D
:10C4C00094ED114AB4EE674AF1EE10FA00F0FA82E8
:10C4D00040F2AC2EC1F2000EDEED3E3ABCEEE33A85
:10C4E00040F6C411002313EE102A042003F0DCFEF2
:10C4F0004AF2F013C1F20003012183F8A810D4ED31
:10C50000112A94ED122AD4ED137A78EEA28A39EE2C
:10C51000029A38EE278A58614AF2F014C1F20004F8
:10C52000DFED447A2468D4ED145AF4EE675AF1EE44
:10C5300010FA07D194ED151AB4EE671AF1EE10FA5D
:10C5400000F0AF8240F2AC20C1F20000D0ED3E0A14
:10C55000BCEEE00A052010EE102A40F6C4110023BC
:10C5600003F0A2FE4AF2F01CC1F2000C01228CF88A
:10C57000A920D4ED156A94ED167A94ED176A78EE39
:10C58000A68A39EE079A38EE068ACCF818004AF2E5
:10C59000F013C1F20003DFED277A1C68D4ED182AEE
:10C5A000F4EE672AF1EE10FA07D194ED195AB4EEC1
:10C5B000675AF1EE10FA00F0638240F2AC2EC1F23D
:10C5C000000EDEED3E4ABCEEE44A40F6C41114EE25
:10C5D000102A0620002303F067FE4AF2F011C1F290
:10C5E0000001012281F8AA20D4ED193A94ED1A3AFB
:10C5F000D4ED1B7A78EEA38A39EE039A38EE278AB7
:10C60000C8614AF2F014C1F20004DFED0A7A24682E
:10C6100094ED1C7AB4EE677AF1EE10FA0ED194ED37
:10C620001D2AB4EE672AF1EE10FA00F0188205E038
:10C63000EC518040000000000AD7233C40F2AC20BF
:10C64000C1F20000D0ED3E1ABCEEE11A002311EE5B
:10C65000102A072040F6C41103F026FE4AF2F01C0F
:10C66000C1F2000C01238CF8AB30D4ED1D6AD4ED7F
:10C670001E0A94ED1F0A78EEA68A39EE209A38EE4B
:10C68000008ACCF820004AF2F011C1F200015FEDFF
:10C69000177A0C68D4ED203AF4EE673AF1EE10FA0E
:10C6A00007D194ED216AB4EE676AF1EE10FA00F05A
:10C6B000C58140F2AC2EC1F2000EDEED3E5ABCEE5A
:10C6C000E55A082015EE102A40F6C411002303F0A5
:10C6D000EBFD4AF2F01CC1F2000C01228CF8AC20F8
:10C6E000D4ED214A94ED224AD4ED237A78EEA48A3F
:10C6F00039EE049A38EE278ACCF824004AF2F01476
:10C70000C1F200045FED357A2468D4ED240AF4EE1A
:10C71000670AF1EE10FA07D194ED253AB4EE673AC4
:10C72000F1EE10FA00F0798140F2AC20C1F2000085
:10C73000D0ED3E2ABCEEE22A40F6C411002312EEF0
:10C74000102A092003F0B0FD4AF2F013C1F20003F1
:10C75000012183F8AD10D4ED256AD4ED261A94EDAD
:10C76000271A78EEA68A39EE219A38EE018A986265
:10C770004AF2F01CC1F2000C5FED527ADCF8004086
:10C78000D4ED284AF4EE674AF1EE10FA07D194EDA1
:10C79000290AB4EE670AF1EE10FA00F02D8140F29A
:10C7A000AC2EC1F2000E9EED3E7ABCEEC76A0023AD
:10C7B00016EE102A0A2040F6C41103F075FD4AF265
:10C7C000F013C1F20003012283F8AE20D4ED295A00
:10C7D00094ED2A5AD4ED2B7A78EEA58A39EE059A93
:10C7E00038EE278AD8624AF2F014C1F200045FEDF5
:10C7F0006F7A2468D4ED2C1AF4EE671AF1EE10FA71
:10C8000007D194ED2D4AB4EE674AF1EE10FA00F02C
:10C81000E28040F2AC20C1F20000D0ED3E3ABCEE26
:10C82000E33A40F6C411002313EE102A0B2003F064
:10C830003BFD4AF2F011C1F20001012381F8AF3053
:10C84000D4ED2D6AD4ED2E2A94ED2F2A78EEA68A07
:10C8500039EE229A38EE028A08634AF2F01CC1F2DD
:10C86000000C5FED8C7ADCF80040D4ED305AF4EE29
:10C87000675AF1EE10FA07D194ED311AB4EE671A47
:10C88000F1EE10FA00F0968040F2AC2EC1F2000EEC
:10C89000DEED3E0ABCEEE00A40F6C41110EE102AAE
:10C8A0000C20002303F000FD4AF2F01194ED317AE0
:10C8B00094ED326AD4ED337AC1F20001012278EEB0
:10C8C000878A39EE069A38EE278A486381F8B020C5
:10C8D0004AF2F014C1F200045FEDAA7A2468D4EDA4
:10C8E000342AF4EE672AF1EE10FA06D1D4ED356A57
:10C8F000F4EE676AF1EE10FA4DD040F2AC2CC1F2C2
:10C90000000CDCED3E7AFCEEE75A002315EE902A8F
:10C910000D2040F6C41103F0C7FC4AF2F013C1F237
:10C92000000394ED355AD4ED364A94ED374A9863B6
:10C9300078EE858A012039EE249A38EE048A83F84D
:10C94000B100B0EE680A11F069FA1FEDC56AB4EEE5
:10C95000C60AF1EE10FA00F31D81B0EE490A11F09B
:10C960005DFA1FEDCB7AB4EEC70AF1EE10FA00F3D0
:10C970000A81B0EE480A11F051FA5FEDD10AB4EE27
:10C98000E00AF1EE10FA00F3F780BDEC048BBDE88D
:10C990001040FEF7EFBF94ED363AB4EE673AF1EE91
:10C9A00010FAAAD1D4ED373AF4EE673AF1EE10FA64
:10C9B000C7D0A2E7D4ED321AF4EE671AF1EE10FAFE
:10C9C0007FF462AF94ED332AB4EE672AF1EE10FAE9
:10C9D0007FF45AAF7CE7D4ED2E4AF4EE674AF1EECD
:10C9E00010FA7FF416AF94ED2F5AB4EE675AF1EEB9
:10C9F00010FA7FF40EAF30E7D4ED2A0AF4EE670A9E
:10CA0000F1EE10FA7FF4CBAE94ED2B1AB4EE671A68
:10CA1000F1EE10FA7FF4C3AEE5E6D4ED263AF4EE7B
:10CA2000673AF1EE10FA7FF47FAE94ED274AB4EE48
:10CA3000674AF1EE10FA7FF477AE99E694ED227A28
:10CA4000B4EE677AF1EE10FA7FF433AE94ED230A78
:10CA5000B4EE670AF1EE10FA7FF42BAE4EE6D4ED99
:10CA60001E2AF4EE672AF1EE10FA7FF4E7AD94ED9A
:10CA70001F3AB4EE673AF1EE10FA7FF4DFAD02E64A
:10CA8000D4ED1A5AF4EE675AF1EE10FA7FF495AD30
:10CA900094ED1B6AB4EE676AF1EE10FA7FF48DAD87
:10CAA000AFE5D4ED161AF4EE671AF1EE10FA7FF442
:10CAB00049AD94ED172AB4EE672AF1EE10FA7FF42F
:10CAC00041AD64E5D4ED124AF4EE674AF1EE10FA96
:10CAD0007FF4FEAC94ED135AB4EE675AF1EE10FAFF
:10CAE0007FF4F6AC18E5D4ED0E0AF4EE670AF1EE29
:10CAF00010FA7FF4B2AC94ED0F1AB4EE671AF1EEAF
:10CB000010FA7FF4AAACCCE4D4ED0A3AF4EE673A1A
:10CB1000F1EE10FA7FF466AC94ED0B4AB4EE674A7E
:10CB2000F1EE10FA7FF45EAC81E494ED067AB4EE97
:10CB3000677AF1EE10FA7FF41BAC94ED070AB4EEBD
:10CB4000670AF1EE10FA7FF413AC35E4D3ED472A0F
:10CB5000F4EE482AF1EE10FA7FF4CCAB93ED483AAC
:10CB6000B4EE483AF1EE10FA7FF4C4ABB0EE489A56
:10CB7000F0EE488AFFF7E5BB41F66C50C0F60200C4
:10CB8000F5F7B2FE01E741F64450C0F60200F5F7B2
:10CB9000ABFEEEE641F61850C0F60200F5F7A4FE33
:10CBA000DBE641F6D840C0F60200BDEC048BBDE8E0
:10CBB0001040F5F799BE00BF4AF2A823C1F2000366
:10CBC000D3ED010A70EE807AC3ED017A704700BFA1
:10CBD00010B52DED028BB0EE408A0FF051FE40B93A
:10CBE0004AF2A823C1F2000383ED038ABDEC028B55
:10CBF00010BD4AF2A824C1F2000494ED040A38EEF4
:10CC0000000AFAF7E9FC84ED030AEFE72DE9F001E9
:10CC100041F2680241F6B855C2F20005C1F20002C5
:10CC20004AF2A823C1F2000392ED0E6B40F2AC274A
:10CC300003210026C1F20007D5F83C0483F82D1526
:10CC400083F82C6505F58064D7ED817A03F5A06C37
:10CC5000D0F84080D7F8FC6165688CED006B92EDF0
:10CC6000106B03F5A26103F5A464F5EE407A03F5B9
:10CC7000A167F1EE10FAC1F8008087ED006BCE607D
:10CC8000656007D090ED107A77EE877A03F5A86398
:10CC9000C3ED007ABDE8F001704700BF10B54AF25D
:10CCA000A824C1F2000404F5A06104F5A16091ED8F
:10CCB000000B90ED001B01F04FFA94F82C3504F5B1
:10CCC000A262D2ED007A002B39D094ED017A77EE92
:10CCD000877AC4ED017A4AF2A824C1F2000404F56F
:10CCE000A46E04F5A263DEF800C0DA68C4F81CC0C4
:10CCF0009EED010AA261FFF76BFF94ED060AB5EE07
:10CD0000400AF1EE10FA06D140F2AC21C1F2000166
:10CD1000D1F8FC01A0614AF2A823C1F20003D3EDCF
:10CD2000070AF5EE400AF1EE10FA07D140F2AC2204
:10CD3000C1F20002D2F854C2C3F81CC010BDC4ED49
:10CD4000017AC8E72DE9F84F4AF2A8232DED028BAE
:10CD5000C1F2000300EB400103EB0111044691F81E
:10CD60007D20551EEDB2042D63D891F87C0000287B
:10CD700056D1964ED1ED181A96ED001A71EEC10AF1
:10CD8000C3ED010A4AF2A825C1F2000504EB4403F1
:10CD900005EB031696ED1B8AD6ED1C8A012A85ED5C
:10CDA000068AC5ED078A48D0032A72D0042A00F00B
:10CDB0009380022A00F0D380052A00F0C280B5EEED
:10CDC000408AF1EE10FA0BD140F2AC22C1F200021F
:10CDD0004AF2A823D2F8FCC1C1F20003C3F818C07C
:10CDE000F5EE408AF1EE10FA0AD140F2AC2CC1F215
:10CDF000000C4AF2A820DCF85412C1F20000C16114
:10CE00004AF2A823C1F2000300222046C3F83025CD
:10CE100083F83A45BDEC028BBDE8F84FF5F718BE34
:10CE200093ED010A91ED187A77EE007AC3ED017A5D
:10CE3000A8E7BDEC028BBDE8F88F95F82C1505F539
:10CE4000A262D2ED007A002978D0D5ED012A37EE22
:10CE5000A22A85ED012A4AF2A825C1F2000505F5AE
:10CE6000A06105F5A16E91ED000B9EED001B01F098
:10CE700073F905F5A46C05F5A263DCF8040093EDE5
:10CE8000038ADCED008AA86085ED068AC5ED078A75
:10CE900095E7D6E914AB4FF000084FF00009504673
:10CEA000594642464B460FF0B7FC48B9D6E91667DB
:10CEB00042464B46304639460FF0AEFC002879D04A
:10CEC0004AF2A820C1F2000004EB440300EB031C6B
:10CED000DCF87420826072E7D6E914AB4FF00008EA
:10CEE0004FF000095046594642464B460FF094FC1D
:10CEF00080B9D6E9166742464B46304639460FF0B0
:10CF00008BFC38B94BEC10AB47EC116B01F024F9FA
:10CF1000D5ED078A4AF2A82EC1F2000E04EB4403B5
:10CF200040F2AC220EEB0310C1F20002416F92ED11
:10CF30007F8ACEF808108EED068A40E7C5ED017AAB
:10CF400089E7F5EE408AF1EE10FA7FF438AF4FF240
:10CF5000C350C3F6A860E86108EE900A2FE741F2DB
:10CF6000680EC1F2000E9EED0E0B9EED101B01F03F
:10CF7000F3F896ED1C3A1649B5EE403ADFED153A56
:10CF80004B68F1EE10FA08BFB0EE633AAB6085ED86
:10CF9000073AFFF73BFE686805F5A26205F5A46C49
:10CFA0004FF000411060CCF8041095ED068AD5EDE5
:10CFB000078A04E74BEC10AB47EC116B01F0CCF89F
:10CFC00095ED068AD5ED078A7AE700BFF8210020A3
:10CFD000B8210020C3F5A83E2DE9F84340F2201205
:10CFE0002DED028B41F26803C1F20003C1F2000291
:10CFF0009E6AD2F87841D3F898503068B6884AF2E1
:10D00000A82244F23F21671BC1F20002C0F20F01C7
:10D010008F4292F83A55468309D893ED137AF0EE91
:10D02000087AB4EEE77AF1EE10FA00F15B814AF289
:10D03000A823C1F2000393F83805012840F2CF83FA
:10D0400093F83975002F40F0518140F2AC26C1F2BF
:10D050000006D6ED072ABDEEE22A12EE102A4AF6A5
:10D06000BC1E0832C1F2000E3EF9122012F1F90383
:10D0700080F26D8141F6B8574AF2A82EC2F200073D
:10D08000C1F2000E0025D7F83C648EF838558EF8B2
:10D090003A55306CCEF804004AF2A823C1F20003DE
:10D0A00003F5A862D2ED007AF5EE407AF1EE10FABF
:10D0B0001DD041F6B85CC2F2000CDCF83C1491EDD6
:10D0C000107AF4EEC77AF1EE10FA40F1EA8293F8A2
:10D0D0003C05002840F0D1824FF4406EC4F2000EAF
:10D0E000012783F83C75DEF8246083F83E6540F242
:10D0F000AC21C1F2000191ED083AFDEEC32A4AF6D7
:10D10000BC1E12EE907AC1F2000E08373EF91730BD
:10D11000FA2B00F3E482FA33C0F25E8341F6B8568C
:10D12000C2F20006DFEDBA7AD6F83C34D3ED030A3A
:10D13000F4EE670AF1EE10FA93ED040A40F0EF8185
:10D14000B4EE670AF1EE10FA40F0E9814AF2A8263F
:10D15000C1F200064AF2A82E96F83835C1F2000E48
:10D16000042BCEED047ACEED057A00F00582032B78
:10D1700000F0B882042B00F0528241F6B857C2F298
:10D1800000074AF2A826C1F20006D7F83C14306C1A
:10D190009FED9F8AD1ED030AB0EE480A02F0C4FA6F
:10D1A000D7F83C74706C86ED080AD7ED040AB0EE2F
:10D1B000480A02F0B9FAF0EE407AC6ED097A96ED27
:10D1C000080AD6ED066A27EEA71A00EE001AB1EE9D
:10D1D000C17AF4EEC76AF1EE10FA0FD580EE070AB5
:10D1E0004AF2A82EC1F2000EC7EE877A26EE800A18
:10D1F00026EEA77A8EED080A8EED097A41F6B85729
:10D20000C2F200074AF2A826C1F20006D7F83C2471
:10D21000B06BD2ED000A02F087FAF1EE401AD7F8AF
:10D220003C34F06BC6ED0A1A96ED090AD3ED010AFB
:10D2300002F07AFA96F8383586ED0B0A002B00F0EA
:10D24000BA8140F2AC2EC1F2000E9EED023AFDEE24
:10D25000C32A4AF6BC1112EE907AC1F200010837D7
:10D260009EED177A31F917C0ACF52F7002EE100A57
:10D27000F8EEC27AB4EEE77AF1EE10FA40F1D2801D
:10D2800096F83D65002E40F0CD80F5EEC07A40F274
:10D29000AC22F1EE10FAC1F2000200F3B982D2ED35
:10D2A000800A37EE875ADFED5B4A25EE206A4AF2A4
:10D2B000A82226EE240AC1F2000282ED0D0A042BF8
:10D2C00000F0C98341F6B85EC2F2000E4AF2A82C03
:10D2D000DEF83C14C1F2000C0F6C9CED071ACCF880
:10D2E0000470D1E00123068382F8393540F2AC2284
:10D2F000C1F20002D2ED071ABDEEE11A4AF6BC1ED9
:10D3000011EE102AC1F2000E02F108033EF913607B
:10D31000FA2E7FF7A4AE4AF2A826C1F2000696F8CC
:10D32000380502287FF4B8AE182D3FF6B5AE05EBF0
:10D33000450706EB071C9CF87D1000293FF4ACAEB6
:10D340002846FFF7FFFC042386F83835A4E64AF2A6
:10D35000A826C1F2000696F83805002800F042839E
:10D360004AF2A826C1F2000696F8390500283FF4D3
:10D3700093AE96F83815022900F07D82032900F05B
:10D380007A8241F26803C1F2000393ED0E0B93ED34
:10D39000101B00F0E1FE4FF0000806F5A0634FF00F
:10D3A0000009D3E9000142464B460FF035FA002848
:10D3B00040F09C8306F5A166D6E9000142464B4643
:10D3C0000FF02AFA002840F091834AF2A826C1F211
:10D3D000000696F83875012F40F2268440F2AC2002
:10D3E000C1F200004AF2A82CC1F2000CD0F8FCE116
:10D3F000D0F85472CCF818E0022641F6AC50C0F6D2
:10D400000200CCF81C708CF83865F5F76DFA43E62D
:10D4100000000000E73EBB3A0AD7233C0000B442BC
:10D42000E02E6542F1EE473AF4EEE73AF1EE10FAFB
:10D430003FF72BAF042B0CD14AF2A823C1F2000313
:10D4400005EB450203EB021090F87D60052E00F01D
:10D450008E8341F6B85EC2F2000E4AF2A827C1F2EE
:10D460000007DEF83C14F86CD1ED100A97ED010AC4
:10D4700002F05AF940F2AC23C1F2000387ED0D0A25
:10D4800097ED071AD3ED800AF4EEC10AF1EE10FA17
:10D49000CCBFF1EE410AF1EE600A4AF2A826FDF790
:10D4A000A3FAC1F2000696ED0C1A1FED257A70EE74
:10D4B000417A96F8382507EE871A042A86ED0D0A78
:10D4C00086ED0C1A78D105EB450C06EB0C10D0ED6F
:10D4D0001E7AF5EE407AF1EE10FA6DD041F6B853AF
:10D4E000C2F2000396ED050AD3F83C2492ED104AEF
:10D4F00074EE673A23EEA33A00EE003AF1EEC32A47
:10D5000080EE220A0FF0C6FE96F838255FED3D1A30
:10D510001FED3D2A50EE021AC6ED001A52E0F1EE60
:10D52000600AB1EE400A0FF04FFF5FED434A20EE74
:10D53000240AFAF751F841F6B85CC2F2000C4AF23C
:10D54000A820C1F2000080ED040ADCF83C2492ED32
:10D55000046A92ED034A66EE063A44EE043AF1EEAE
:10D56000E35A4AF2A826C1F20006C0ED055A96F821
:10D570003835042B7FF4FBADD6F83035002B40F066
:10D580005A8105EB450706EB07112F4691F87D30D0
:10D59000032B00F06782012B00F06482042B00F063
:10D5A0001083022B00F0A5824AF2A82EC1F2000ED1
:10D5B0009EF83835DBE51A464AF2A827C1F2000783
:10D5C00000263E60042A00F0D98141F26805002659
:10D5D0000027C1F20005D5E90E0132463B460FF0A7
:10D5E0001BF990B9D5E9100132463B460FF014F90A
:10D5F00058B94AF2A823C1F2000393F8391500295B
:10D6000040F0B881022283F83B254AF2A82CC1F2EF
:10D61000000CCCF83445BDEC028BBDE8F8834AF22F
:10D62000A826C1F2000605EB450306EB031797F8A1
:10D630007D1004297FF4A1ADD6ED050A306C97ED7D
:10D64000190A02F071F8DF4A97ED1B5AD2ED014A30
:10D65000B1EE406AF1EE450AD2ED005A24EEA00A7E
:10D6600066EE247A15EE860A40EEA57A86ED080A63
:10D67000C6ED097AD6ED066AA5E54FF44062C4F21C
:10D68000000293F83E65506A811B02EE101ADFED2E
:10D69000CE1AB8EE421AB4EEE11AF1EE10FA00F327
:10D6A0000B824AF2A823C1F20003B3F83C65002EB6
:10D6B0003FF41DADF4EEC77AF1EE10FAFFF617ADA8
:10D6C00093F83D05002840F05F824AF2A82CC1F291
:10D6D000000C00228CF83C258CF83D2507E5FFF76F
:10D6E00095FA1BE540F2AC26C1F2000696ED044A1D
:10D6F000FDEEC46A4AF6BC1716EE900AC1F20007A6
:10D70000083096ED161A37F9103003EE903A4AF2C7
:10D71000A822F8EEE32AC1F2000240F2AC2CF4EEAB
:10D72000C12AD2ED066A9FEDA93AC1F2000CF1EED2
:10D7300010FA9CED032AC8BF72EEC15A26EE830A86
:10D74000F1EE417AF4EEE72AFDEEC21ACCBF65EEA7
:10D75000C05ADFEDA35AF1EE10FA48BF72EE812AEB
:10D7600011EE901A4AF6BC1E48BF62EEC05AC1F2D2
:10D77000000E0831934A3EF9117000EE907AB8EE2F
:10D78000E07A92ED015AB4EEC71AF1EE10FA48BFF2
:10D7900077EE410AF4EEC77A4CBF60EE800ADFED07
:10D7A000900AF1EE10FAC8BF31EE071AD2ED004A26
:10D7B000C8BF61EE000A65EE857A25EE200A14EEF8
:10D7C000A50A40EEA47A4AF2A820C1F2000080ED3A
:10D7D000080AC0ED097AF6E4FFF760FA9EE440F229
:10D7E000AC2CC1F2000CDCED070ABDEEE00A4AF6F3
:10D7F000BC1E10EE102AC1F2000E083200213EF9C4
:10D80000122083F8391512F1F903FFF633AC9EE5C7
:10D81000D2ED950A77EEC75ADFED6D6A25EEA04A84
:10D820004AF2A82024EE260AC1F2000080ED0D0A7B
:10D83000D2ED800A43E59C427FF6F1AE05EB45024E
:10D8400006EB021E9EF87D0005283FF4E8AE013588
:10D85000EDB2182D00F2418105EB450C06EB0C11E1
:10D8600091F87D70002F00F038812846FFF76AFAA2
:10D8700096F838357BE440F2AC23C1F2000393ED17
:10D88000045AFDEEC54A4AF6BC1214EE907AC1F273
:10D8900000020837D3ED167A32F9176006EE106AE7
:10D8A000B8EEC67AB4EEE77AF1EE10FA59DCF1EE92
:10D8B000676AB4EEE67AF1EE10FA52D4D3ED030AB9
:10D8C000BDEEE00A10EE103A083332F9132007EEED
:10D8D000102AB8EEC77AF4EEC77AF1EE10FA40D407
:10D8E000F4EEC76AF1EE10FA3BDC03297FF4D4AB07
:10D8F00041F6B85EC2F2000E9FED367ADEF83C3497
:10D90000D3ED007AF4EEC77AF1EE10FA40F14381DC
:10D91000DFED316AF4EEE67AF1EE10FA40F33B8186
:10D92000D3ED017AF4EEC77AF1EE10FA40F13381CB
:10D93000F4EEE67AF1EE10FA40F32D8141F2680C34
:10D94000C1F2000C9CED0E0B9CED101B00F004FCD2
:10D950004AF2A823C1F20003022183F83815FFF729
:10D960009BBB4AF2A82CC1F2000C03218CF838159D
:10D97000FFF792BB032083F83B0546E64AF2A82650
:10D98000C1F2000696ED020AFFF722F905EB450009
:10D9900006EB001191F87D50052D7FF416AE40F294
:10D9A000201EC1F2000EDFED0D5ADEF8382106EE22
:10D9B000902AF4EEE56AF1EE10FA7FF506AE07F074
:10D9C000CDFB02E6C82100208096984A6F12033BE7
:10D9D000E73EBB3ACDCCCC3DCDCCCCBD0F5C6BC1D2
:10D9E0000000000041F6B857C2F200074AF2F01EEC
:10D9F000D7F83C34B06C196C93ED024AC1F2000EBA
:10DA0000B1EE440ADEED270A716001F073FFD7F82A
:10DA10003C24F06C5FED0E0A92ED100A01F06AFFF3
:10DA2000D7F83C3440F2AC2CC1F2000CD3ED023AF2
:10DA3000DCF85472B1EE633A012141F69450C0F61D
:10DA4000020086ED0D3A86ED0C3AF76186F838153E
:10DA5000F4F74AFF84E44AF2A823C1F2000393EDED
:10DA6000071A11E54AF2A822C1F2000207EB4706A5
:10DA700002EB061892ED055A98ED197AB4EEC75AE2
:10DA8000F1EE10FA7FF58AAD41F6B850C2F200000F
:10DA900092ED010AD0F83C34D3ED106A30EE660AFC
:10DAA00010F0BCF9D8ED190AB4EEE00AF1EE10FA64
:10DAB00049D498F87D3071E5576A93F83D2583F88D
:10DAC0003E75002A00F0A9804AF2A823C1F20003A3
:10DAD000012183F83D15FFF70ABB4AF2A823C1F2E2
:10DAE0000003022683F83865FFF747BBFFF78EF87F
:10DAF0006BE44AF2A826C1F2000607EB470306EBE7
:10DB0000031808F1600896ED053AD8ED013AB4EE35
:10DB1000E33AF1EE10FA7FF5ABAE41F6B852C2F23D
:10DB2000000296ED014AD2F83C0490ED106A34EE02
:10DB3000460A10F073F9D8ED015AB4EEE50AF1EE99
:10DB400010FA7FF595AE4AF2A82607EB4703C1F21B
:10DB5000000606EB031C2846DCF868100F19C6F80F
:10DB60003075F4F7C9FE96F83835FFF700BB93ED32
:10DB7000071A40F2AC2CB1EE410AC1F2000C83ED61
:10DB80000D0ADCED800A7FE441F6E850C0F60200A1
:10DB9000F4F7AAFE99E540F2AC22C1F20002D2ED00
:10DBA000087AFDEEE76A4AF6BC1616EE907AC1F2E4
:10DBB0000006083736F9170010F1FA03BFF66CAA11
:10DBC000BCE64AF2A826C1F2000607EB470106EBC5
:10DBD000011896ED058AD8ED192A38EE620A10F080
:10DBE0001DF941F6B85CC2F2000CD6ED011ADCF862
:10DBF0003C2492ED102AB0EE408A31EEC20A10F0B9
:10DC00000DF938EE001AF0EE007AB4EEE71AF1EEF4
:10DC100010FA98D498F87D30C3E441F6C450C0F6A9
:10DC20000200F4F761FE4FE741F6B8571FED948A02
:10DC3000C2F2000786ED0A8AD7F83C34B06B86ED55
:10DC40000B8AF0EE480A93ED000A01F053FED7F874
:10DC50003C14F06B91ED010AF0EE480A01F04AFE27
:10DC6000D7F83C24306C92ED030AF0EE480A01F03C
:10DC700041FE706CD7F83C64F0EE480A96ED040A59
:10DC800001F038FEFFF7AABB2DE9F04F41F618600E
:10DC9000654E4AF2A82589B00024C1F20005C0F6FD
:10DCA0000200F4F721FE371D21464FF4A9622846F1
:10DCB00010F026FB06F1080906F10C0A06F1100B1C
:10DCC00039462246234630468DE800060294CDF8B8
:10DCD0000CB0049405940694079401F007FD3946AE
:10DCE0008646224623463046C5F838E08DE80006D1
:10DCF0000294CDF80CB0049405940694079401F0B6
:10DD0000F5FC06F1200806F11C07844606F118010F
:10DD10008DE880012246234606F114000837C5F835
:10DD20003CC003970294049405940694079401F070
:10DD3000DDFC083F814606F118018DE8800122468E
:10DD4000234606F114000837C5F840900397029463
:10DD5000049405940694079401F0C8FC06F1380772
:10DD600006F1300C06F1340E804606F12C0106F166
:10DD70002800224623468DE80050C5F844800397CA
:10DD80000294049405940694079401F0AFFC06F104
:10DD9000480906F1440C864606F14001234606F187
:10DDA0003C00224641F6B8574C36CDF800C0C2F2CE
:10DDB0000007C5F848E0CDF8049002940396049457
:10DDC00005940694079401F091FC05F5A86107F508
:10DDD00080624FF0000892ED010AC1F80080E8640B
:10DDE00085F83C4585F83D4585F83845FEF7F0FE59
:10DDF000D7F83C344CF6CD4C0120C3F6CC5C1A6C01
:10DE000085F87D00C5F864C0196C6A604FF07E50DB
:10DE10000523A967C5F89C00C5F8A880AC6685F8FD
:10DE2000AD3009B0BDE8F08FB40400104AF2A82369
:10DE3000C1F20003002093F87D2082B1012030332D
:10DE400007E093F8AD200130603332B1013019287A
:10DE500004D093F87D100029F3D1704770477047C4
:10DE60004AF2A823C1F2000393F83825042A10D0FF
:10DE7000002203F5966083F87D20303303F13001F2
:10DE800083F87D206033834281F87D20F6D1012024
:10DE900070470020704700BF4AF2A823C1F2000378
:10DEA00000EB400003EB0010503070470048704713
:10DEB000A8A7001090ED001AFDEEC10A92ED007ABD
:10DEC00010EE90CA01EB8C0090ED090A77EE407AD3
:10DED000C3ED007A704700BF91ED107A92ED000A11
:10DEE00077EE007AC3ED007A704700BFD1ED101ACB
:10DEF00092ED001A71EE810AC3ED000A91ED057AE8
:10DF000092ED010A77EE007AC3ED017A704700BF07
:10DF100091ED033AD2ED002A33EE222A83ED002A56
:10DF2000D1ED041A92ED011A71EE810AC3ED010AD6
:10DF300091ED057A92ED020A77EE007AC3ED027A4E
:10DF4000704700BF91ED003AD2ED002A33EE222A4D
:10DF500083ED002AD1ED011A92ED011A71EE810ACA
:10DF6000C3ED010A91ED027A92ED020A77EE007A92
:10DF7000C3ED027A704700BF9FED081A08B5DFEDC8
:10DF8000080A80EE010A0FF023FDF7EE007A37EE63
:10DF9000C00A9FED047A20EE070A08BD80E6C54757
:10DFA0005C8F423E2B2A2D4741F6B850C2F200004A
:10DFB00000F58862D0F83C34D3ED100A70EE607A38
:10DFC000C2ED007A704700BF2DE9D0432EA3D3E9FC
:10DFD00000232DED048B51EC100B0EF02BFA41ECCD
:10DFE000100B41EC190B0FF0EFFD51EC100B02463A
:10DFF0000B460EF01FFA26A3D3E900230EF01AFAFF
:10E000000B4600210246C3F6F07100200EF0CCF85A
:10E010009FED1B1B41EC100B41EC180B0FF0DCFBD0
:10E020001DA1D1E9000153EC102B0EF0B9FAB0EEAE
:10E03000480AF0EE680A41F6B854C2F20004C4E996
:10E040000C010FF0B5FE57EC106BB0EE490AF0EE84
:10E05000690A0FF01DFA59EC108B32463B4610A1AD
:10E06000D1E900010EF09CFA42464B460EF0E2F96F
:10E07000C4E90E01BDEC048BBDE8D083AFF3008092
:10E08000000000000000F83F000000A046DF913FC4
:10E0900000000000916B7B3F2CF52966E4FEFA40FE
:10E0A00080D6C1D6772DFB4041F6B853C2F20003AB
:10E0B00070B403F1400103F1E002F0EE407A03F5A1
:10E0C000C073002691ED006A76EE275A0D46E5EC06
:10E0D000015A92ED005A75EE204A1446E4EC014ACA
:10E0E00093ED004A74EE013A1846E0EC013A91EDE6
:10E0F000013A73EE272A0236C1ED012A92ED012A78
:10E1000072EE201A291DC2ED011A93ED010A30EEBC
:10E11000017A221D83ED017A031D282ED2D141F60A
:10E12000B852C2F20002B0EE410AD2F83C14D1ED6E
:10E13000031AD1ED046A91ED057A71EEA77A76EEB5
:10E14000A00A37EE011AC1ED037AC1ED040A81ED90
:10E15000051A70BCFEF730BD2DE9D04F41F6B8541A
:10E16000C2F200042DED028B57EC106BD4E90CAB1E
:10E1700082B0D4E908233046394659EC118B0EF0B1
:10E1800013F852465B460EF055F90DF0D1FF94EDB1
:10E190000E7BD4E90A2308EE100A494640468DED6D
:10E1A000007B0EF001F8DDE900230EF043F90DF0DD
:10E1B000BFFF324608EE900A3B4630463946C4E976
:10E1C0000867C4E90A890DF0EFFF02460B46504686
:10E1D00059460EF02FF90DF0ABFF07EE900A4246BC
:10E1E0004B464046494637EEC88A0DF0DDFF0246F1
:10E1F0000B46DDE900010EF01DF90DF099FF00EE70
:10E20000900A9FED061A70EEE80AB0EE480A02B0D6
:10E21000BDEC028BBDE8D04FFFF746BF0000000009
:10E22000D1ED014A91ED003A64EEA43A43EE033A8F
:10E2300091ED024A44EE043AD1ED036A46EEA63A65
:10E24000B1EEE30AC3EE002AC0ED002A91ED012AE7
:10E25000C2EE001AC0ED011A91ED021AC1EE000AD9
:10E26000C0ED020A91ED037AC7EE007AC0ED037AA1
:10E27000704700BF92ED026A92ED005A76EE067A80
:10E28000D2ED035A91ED023A67EE856AD1ED004A6C
:10E2900025EE054A75EEA52A26EE837A04EE247A49
:10E2A00091ED012A62EE853AD2ED016A03EEC27A5F
:10E2B00066EEA63A66EEA70A04EEA37A02EE207A8C
:10E2C00066EEA21A25EEA52A03EE217A04EEC27AA2
:10E2D00026EE063A76EEA61A04EEC37A21EE861AE8
:10E2E00080ED007AD1ED014AD1ED000A23EE247AC7
:10E2F00001EE207A26EE220A91ED021A75EE052A29
:10E3000000EE017A22EEA50A25EE215A00EE807A6F
:10E3100002EE647A04EE247A01EE457A03EEE47AA2
:10E3200025EEA70A80ED017A91ED015AD1ED004A60
:10E3300065EEA15A60EE057A45EEA47A91ED027A77
:10E3400042EE077A26EE226A66EEA26A44EEC67AAA
:10E3500043EE477A45EE267A43EEC77A44EE077AD3
:10E36000C0ED027A704700BF00B592ED011AD2ED00
:10E37000020A92ED030A85B01368F1EE416AB1EE2C
:10E38000607AF1EE407A6A460093CDED016A8DED38
:10E39000027ACDED037AFFF76DFF05B000BD00BF37
:10E3A00038B51C4601F13003154620460E491A4681
:10E3B000FFF7DAFFD5ED002A94ED003A33EE222A7A
:10E3C000D4ED011A84ED002A95ED011A71EE810A4F
:10E3D00094ED027AC4ED010A95ED020A77EE007A17
:10E3E000C4ED027A38BD00BFC81D002038B51C46F8
:10E3F00001F13003154620460E491A46FFF7B4FFD7
:10E40000D5ED002A94ED003A33EE222AD4ED011A1C
:10E4100084ED002A95ED011A71EE810A94ED027ADD
:10E42000C4ED010A95ED020A77EE007AC4ED027A96
:10E4300038BD00BFBC1D0020D2ED010A91ED010ADC
:10E44000D2ED006A91ED007A20EE805A06EE875AEE
:10E45000D1ED027AD2ED025A05EEA75A80ED005AAC
:10E46000D2ED044A91ED014A92ED033AD1ED003A22
:10E4700064EE841A43EE231A92ED052AD1ED022AA6
:10E4800042EE221AC0ED011A92ED076A91ED011ACF
:10E4900092ED060AD1ED000A66EE017A40EE207A8E
:10E4A000D2ED086A91ED027A46EE877AC0ED027AE3
:10E4B000704700BFD2ED030A91ED010AD2ED006A68
:10E4C00091ED007A20EE805A06EE875AD1ED027A5D
:10E4D000D2ED065A05EEA75A80ED005AD2ED044A55
:10E4E00091ED014A92ED013AD1ED003A64EE841AC1
:10E4F00043EE231A92ED072AD1ED022A42EE221AA8
:10E50000C0ED011A92ED056A91ED011A92ED020A31
:10E51000D1ED000A66EE017A40EE207AD2ED086A6B
:10E5200091ED027A46EE877AC0ED027A704700BF1D
:10E5300091ED007AD1ED015A91ED026AD1ED036AB5
:10E5400027EE077A65EEA55A26EE066A66EEA66AFB
:10E55000002A7ED075EE860AB7EE005A30EEA60A83
:10E5600070EE077AC5EE277AF1EE652A35EEC62AF7
:10E5700076EE651A32EEC61A72EE660A31EEE60AD9
:10E5800071EE266A30EE875A70EE075A36EE877AB9
:10E5900025EE276A65EEA74A27EE274A80ED006A36
:10E5A000C0ED044A80ED084AD1ED013A91ED023AFE
:10E5B00091ED032AD1ED002A63EE831A22EE221A8E
:10E5C00071EE810A31EEC10A30EEA05A70EE005AA7
:10E5D00065EE276A25EEA76AC0ED036A80ED016A41
:10E5E00091ED017AD1ED034AD1ED023A91ED004A65
:10E5F00027EE243A63EE842A33EE622A73EE221A5F
:10E6000032EE021A71EEA10A21EE270A20EEA75A75
:10E6100080ED060A80ED025AD1ED025A91ED036AAF
:10E6200091ED017AD1ED006A65EE864A27EE264A21
:10E6300074EE843A34EEC43A73EEA32A33EE032A1E
:10E6400062EEA71A22EE271AC0ED071A80ED051A0E
:10E650007047F7EE007A87E770B52DED088BD0EDA7
:10E66000039AD0ED008A90ED018A90ED029A28EE8F
:10E67000A8AA69EEA9AA28EEA91A08EE091A7AEE44
:10E680006A1A29EE09BA68EE08BA71EECB0A31EEC1
:10E69000010A70EEAB0A0C4615461E460EF094FEBB
:10E6A00069EE287A58EE297A84ED000AB8EE000A5D
:10E6B00027EE800A0EF0EEFD28EE288A09EE298A60
:10E6C0003AEE2AAA38EE088A3AEE4BBA85ED000AED
:10E6D0003BEE6BBA88EE0B0A0EF0E0FD86ED000A09
:10E6E000BDEC088B70BD00BFD2ED016A70B592ED34
:10E6F000005A26EEA66A05EE056AD2ED025A2DED05
:10E70000048B1446054605EEA56A0E46B0EE409A07
:10E71000F1EEC68AB6EE008A68EE888AB0EE680A24
:10E720000FF032FB20EE087AD4ED007AC7EE280A0B
:10E73000D4ED014A94ED024AF1EE603A27EEA33A95
:10E7400064EEA32A24EE232A84ED003AC4ED012AC4
:10E7500084ED022A96ED018AD6ED001A28EE088A89
:10E7600001EEA18A96ED021A01EE018A96ED030AE6
:10E7700000EE008AB0EE680A0EF06EFFF7EE006A57
:10E7800048EE486A96ED011A26EE895AD4ED005AF1
:10E7900005EE090A96ED005A61EE250A40EE050ADB
:10E7A000D6ED025A94ED016A45EE860A94ED027A9E
:10E7B00096ED036A46EE070A60EE013AC5ED000ADF
:10E7C000D4ED007A47EEC53AD4ED024A45EEE43A7C
:10E7D00094ED014A46EE043AC5ED013A94ED023A51
:10E7E000D4ED012A61EE031A42EEC51A40EE251A55
:10E7F00094ED002A46EE421AC5ED021AD4ED016AE4
:10E80000D4ED020A61EE267A50EEC57A94ED007AD4
:10E8100045EE877A40EE067AC5ED037ABDEC048BAF
:10E8200070BD00BF91ED002AD0ED060A2DE9F04140
:10E8300040EE020A2DED028BC2ED060AD1ED015A1F
:10E8400090ED074A00EE254A0E4682ED074AD1EDCB
:10E85000023AD0ED087A40EE237A92B0C2ED087AFF
:10E8600091ED033AD0ED096A40EE036A02F13008F7
:10E87000C2ED096AD6ED042A90ED0A1A00EE221ABA
:10E88000044682ED0A1AD6ED051AD0ED0B4A40EE89
:10E89000214A1546C2ED0B4A93ED035A93ED047AD3
:10E8A00093ED056A76EE850A74EE867A31EE074AB4
:10E8B00096ED062AD6ED075AD6ED083A74EE252ACB
:10E8C00077EEA31A30EE823A22EE807A63EE006A87
:10E8D00021EE801A00F130010FAA4046B0EE408AC6
:10E8E0001F46CDED0F6A8DED107A8DED111AFFF7F1
:10E8F000FBFE684641460122FFF71AFE97ED005ADB
:10E90000D5ED064A97ED012AD5ED070A97ED026A83
:10E9100095ED084A75EE243A72EE205A36EE043A26
:10E920000CA809A96A46CDED093ACDED0A5A8DED3C
:10E930000B3AFFF781FDD4ED007ADDED0C2A48EEAD
:10E94000227AD6ED0A1A37EEA14A9DED0D1A85ED11
:10E95000004AD4ED016A48EE016A96ED0B0A36EEE4
:10E96000801A9FED2C7A85ED011A9DED0E5A94EDDB
:10E97000022A75EE074AD6ED0C0A08EE242A32EE7A
:10E98000202AF6EE000A85ED022AD4ED003A74EE54
:10E99000235AD4ED032A25EEA06A96ED0D3A46EEF1
:10E9A000082A72EE831AC5ED031AD4ED017A71EECE
:10E9B000276A94ED045A26EEA00A96ED0E7A00EE30
:10E9C000085A75EE074AC5ED044A94ED024A72EE04
:10E9D000043A94ED053A63EEA05A96ED0F6A05EEFF
:10E9E000C83A73EE062AC5ED052AD4ED021A32EEB6
:10E9F000211A94ED100A61EE207AD6ED096A07EE2D
:10EA0000C80A30EE267A85ED107A12B0BDEC028B82
:10EA1000BDE8F0810AE81C4170B541F6B854C2F275
:10EA200000042DED028BD4F83C0430300146FFF792
:10EA3000F7FBD4F83C0404F5806504F581663030BA
:10EA4000291D05F10C033246FFF706FE9FED168ADD
:10EA500095ED011A21EE080AF8F7BEFDD5ED036A1F
:10EA6000F0EE400A96ED000ADFED108A20EE087AFB
:10EA700026EE888A20EEA80AC5ED010A86ED007A06
:10EA800085ED038A0EF0E8FDD5ED017A04F5826488
:10EA900084ED000A27EEA80A0FF076F984ED010A4A
:10EAA000BDEC028B70BD00BFE02E654235FA8E3C96
:10EAB000F0B540F22013C1F2000341F6B854D3F888
:10EAC00030C1D3F83411D3F83871D3F82461D3F8B6
:10EAD0002851D3F82C21C2F2000487B08E4620685A
:10EAE000CDF800C0694693ED610A0396049505923E
:10EAF000CDF804E0029705F0F7FAD4F83C24D4F8F6
:10EB00000034D66804EB83010E641569C1F8E05047
:10EB10005069C1F88001D2F800C0C1F820C256681F
:10EB20000D4646F26760591CC6F26660C5F8C062C1
:10EB300080FB015CCE17C6EB2C10956804EB8303B9
:10EB400000EB8002A1EBC201C3F86053C4F80014CB
:10EB500007B0F0BD00B507EE100A89B0F8EEC77A2D
:10EB600005AA08A941F6B85C61ED017AC2F2000C71
:10EB700001924CF2AC534DF6B562C3F22773C0F666
:10EB80000002059302920123DCF80000009306AA1C
:10EB90008DED060A05F096FC09B000BD00B51B49D5
:10EBA00089B0086804900590FFF7E6F941F6B8537C
:10EBB000C2F2000303F58862D2ED007AF5EE407AE6
:10EBC000F1EE10FA8DED060A8DED070A18680ED1E8
:10EBD0004DF6ED6204A9C0F60002022301910292F3
:10EBE000002106AA009305F06DFC09B000BD4DF6AA
:10EBF000D96204A9C0F6000201230191029200210A
:10EC000006AA009305F05EFCEFE700BF14070010B2
:10EC100041F6B85CC2F2000C10B5DCF83C2492ED71
:10EC2000074AD2ED063A30EE842A70EE232A92ED9E
:10EC3000086A22EE023A2DED028B02EEA23A71EE44
:10EC4000060A8AB000EEA03AF1EEC36AC2EEA61A36
:10EC500040F2AC24C1F2000404F58C6104F58E642A
:10EC600082EE267A80EEA61A9FED1E0A30EE660A24
:10EC700091ED038ACDED071A8DED087A8DED091A15
:10EC80000FF0CCF8D4ED007A4AF61440C1F200003F
:10EC900000EE278A90F8BC315B078DED048A05D41D
:10ECA000DFED114A28EE248A8DED048A41F6B85E24
:10ECB000C2F2000E4EF2ED3104AAC0F60001DEF8F9
:10ECC000000001920323029107AA00218DED058A1D
:10ECD0008DED068A009305F0F5FB0AB0BDEC028BC2
:10ECE00010BD00BF0AE81C416F12833A00B54AF616
:10ECF0001440C1F20000204A90F8BC31D2ED017AF4
:10ED00008BB05A07CDED047A05D49FED1C7A67EEDF
:10ED1000877ACDED047A60EEA02A40EE002ACDED90
:10ED2000057ACDED067A41EE012AB1EEE22AF7EE40
:10ED3000007AC7EE821A41F6B85CC2F2000C4EF2BD
:10ED4000A13104AAC0F60001032301920291DCF86C
:10ED500000000093002107AA20EE210A60EEA10A1C
:10ED600021EE211A8DED070ACDED080A8DED091A65
:10ED700005F0A8FB0BB000BD1C0700106F12833A12
:10ED8000F0B5F1EE007A2DED088BB0EE40AAF0EE72
:10ED900060AAB0EE41BAF0EE61BAF4EEE72AF1EE05
:10EDA00010FA8BB0B0EE628A0546F0EE428AB0EE01
:10EDB000439A40F1F98041F26803C1F2000393EDF8
:10EDC0001F0AB5EE400AF1EE10FA00F0ED8041F6B0
:10EDD000B854C2F20004D4E908670022304639462C
:10EDE00000230DF019FD002840F0158132463B4606
:10EDF00051EC1A0B0DF0D8F9D4E90C230DF01AFBE5
:10EE00000DF096F9D4E90A23064651EC1B0B049643
:10EE10000DF0CAF9D4E90E230DF00CFB0DF088F9C2
:10EE20004FF44062CDED068AC4F2000240F2201396
:10EE30000590C1F20003D3ED616A05EE105A536AE2
:10EE40008749D4F800249FED877AD1ED007AB8EE97
:10EE5000456A05EE903A26EE877A76EE277AF8EE46
:10EE6000656ABDEEC77A76EEE77AB8EEC77A41F604
:10EE7000B854C7EE877AC2F20004FDEEE77A17EEC7
:10EE8000903AD31A48BF2833272B88BF002304EBBE
:10EE90008301D4F83C24D1ED106A03F138016033CA
:10EEA00004EB830304EB8101D1ED005A93ED006A7A
:10EEB000D2ED038AC2ED036A0968D2ED049A1161AA
:10EEC000196841F2680392ED05AAC1F2000351618D
:10EED000D3ED1F7A40F2AC2267EEA77A93ED207A49
:10EEE000C1F2000202F5896179EEE59AF0EE675A07
:10EEF00078EEE68A3AEE46AAD1ED006A47EE075A66
:10EF0000F1EEE55A02F5886191ED036A68EE255A43
:10EF1000B0EE665A05EE865A93ED217AF0EE455A28
:10EF2000B0EE675ACDED075A07EE075AB1EEC57A33
:10EF300028EE078A93ED1E7A46EE086A47EE077AB6
:10EF4000CDED086AF1EEE77A02F58A6292ED017A78
:10EF500027EE899AD2ED007A032549EE077A2B46EF
:10EF6000009507AD01954DF611752068002104AAA2
:10EF7000C0F60005CDED097A029505F0A3FAD4F8A4
:10EF80003C34D3ED036A93ED047AD3ED057A76EE43
:10EF9000A88A77EE299A37EE8AAAC3ED038AC3EDD1
:10EFA000049A83ED05AA2EE041F6B85EC2F2000E87
:10EFB0004AF6144CDEF83C34C1F2000C196C9CF893
:10EFC000BC01069100224107049205921FD44BF622
:10EFD0009573C3F2D63341F6B85007930893C2F243
:10EFE000000000234DF61171C4F2C82307AAC0F631
:10EFF00000010068099301920323029104AA0021F1
:10F00000009305F05FFA0BB0BDEC088BF0BD002358
:10F01000C4F22013DFE7B0EE4A0AF0EE6A0A84ED8C
:10F0200008AB84ED0ABBFEF7CFFFB0EE4A0AF0EE64
:10F030006A0AB0EE4B1AF0EE6B1AFFF78DF8D4F8AF
:10F040003C3493ED030AD3ED040A93ED051AB1EEB7
:10F05000400AF1EE600A38EEC11AFFF725F8D2E750
:10F06000240700100024744930B5F0EE007A2DED2D
:10F07000048BF4EEE71AF1EE10FA8BB040F1D88071
:10F0800041F26803C1F2000393ED1F2AB5EE402A56
:10F09000F1EE10FA00F0CC804FF4406C8DED040AD4
:10F0A000CDED050A8DED061AC4F2000C40F2201ECB
:10F0B000C1F2000EDCF824307849DEED616A08EE1A
:10F0C000900A9FED771AD1ED030A26EE810AB8EE79
:10F0D000689A07EE103A79EE207AB8EE472ABDEE2C
:10F0E000C05A32EE676AF8EEC54A41F6B852C6EE2B
:10F0F000245AC2F20002D2F80054BDEEE54A14EEE2
:10F10000104A2B1B48BF283341F6B854C2F2000402
:10F11000272B88BF002304EB8300D4F83C54D0EDA8
:10F12000883A03F1B001D83304EB810E04EB83027B
:10F1300095ED008ADEED002A92ED001AC5ED003A49
:10F14000DEF800C0D5ED018AC5F804C0106841F2B0
:10F15000680E95ED029AC1F2000EA8609EED1F3A6E
:10F1600040F2AC2C23EE033ADEED200AC1F2000C93
:10F170000CF58B63F0EE436A38EE638A78EEE28A30
:10F18000D3ED003A39EE419A40EEA06AB1EEE67A4C
:10F190000CF58A6191ED036A21EE870AB0EE635A9D
:10F1A00000EE065A9EED212AF0EE437A8DED075AC5
:10F1B00042EE027AF1EEE74A61EEA45A9EED1E4A53
:10F1C00046EE253A04EE043ACDED083AF1EEC32AB4
:10F1D0000CF58C6292ED011AD2ED000A61EEA21AD2
:10F1E000032541EE810A206800952B4607AD019565
:10F1F0004DF64575002104AAC0F60005CDED090ABB
:10F20000029505F05FF9D4F83C04D0ED006A90ED6A
:10F21000017A90ED020A36EE888A77EE288A30EE7F
:10F22000099A80ED008AC0ED018A80ED029A28E0FB
:10F230004AF61442C1F20002002392F8BC01049382
:10F2400040070593069320D44BF6957CC3F2D63C39
:10F25000CDF81CC0CDF820C0CDF824C041F6B85E72
:10F26000C2F2000E4DF6457207A9C0F60002DEF8A4
:10F270000000019103230292002104AA009305F0EB
:10F2800021F90BB0BDEC048B30BD0020C4F2A0000E
:10F290004FF08041079008900991DFE71C070010AC
:10F2A000002474492DE9F04F41F6B856C2F2000629
:10F2B0002DED068BD6F83C84002740F22014C8F8C8
:10F2C0000070C8F80470C8F80870C8F80C70C8F866
:10F2D0001070C1F20004ADF50F7D94ED450AFEF704
:10F2E0004BFED6F83C544FF07E5388ED050AAF61D3
:10F2F000EF612F626F62AF62EF622B636F63AF6388
:10F30000EF6394ED450AFEF737FE282085ED100ADD
:10F31000FBF760F900273D4606F10408D4F8782190
:10F32000D4F878019042FBD0D4F824B1D4F828A1C5
:10F33000D4F82C91D4F83CE1D4F84001D4F844112D
:10F34000D4F83031D4F83421D4F838C10AEE902AF8
:10F3500046F267620AEE103AC6F266627B1C06EE5F
:10F36000909A05EE10AA82FB03924FEAE37A6AEEC6
:10F37000AA7ABF0004EE90BA4AEE0A7ACAEB2212C9
:10F380000DF1A40A03EE10CA0DF104090AEB070CF3
:10F390000DF50E7AB944F1EE645A5744B1EE456A60
:10F3A000B1EE667A02EB820207ED3D7AC9ED005AB2
:10F3B0008CED006AA3EBC20708EE90EA09EE100A92
:10F3C00008EE101A43EE037AF1EEE79A69EE092A85
:10F3D00048EEA82A8AEE29AACAEEA9AA48EE082A67
:10F3E000C3EE299AB1EEE22AD6F83C14012230315C
:10F3F00079A8C8EE828A89EE029A88EE028AFFF71F
:10F4000097F882A8414679AAFFF754F806F110014F
:10F4100085A879AAFFF74EF8DDED861A9DED871ACB
:10F42000DDED850A9DED820ADDED833A9DED844A8E
:10F4300061EE094A20EE885A61EEA85A51EE884AD8
:10F4400064EE2A6A11EE285A20EE297A50EE895A83
:10F4500063EE8A7A53EEA96A14EE0A7A50EE2A7A9B
:10F46000B6EE006AD6F83C0454EEC66A15EE467A4B
:10F4700055EEC67A3030014688AA9FED2F0ACDEDB1
:10F48000886A8DED897ACDED8A7AFFF72DF9272DDF
:10F4900042DCD4ED613AF7EE000A80EEA34A013572
:10F4A000BDEEC40A10EE100A00EB80018D4214DAA2
:10F4B000C82D7FF733AFDDED8C7A9DED8B3ADDED16
:10F4C0008D2A33EE272ADFED1D1A32EE221AB4EE12
:10F4D000E11AF1EE10FA3FF721AF41F6B854C2F24B
:10F4E000000401A8D4F83C24282124320AF0B6FCF8
:10F4F000D4F83C242821283229A80AF0AFFCD4F8FB
:10F500003C2451A82C3228210AF0A8FC0DF50F7DCF
:10F51000BDEC068BBDE8F08F01A828218BAA0AF06C
:10F5200021FD28218CAA29A80AF01CFD51A8282118
:10F530008DAA0AF017FDACE7CDCCCC3D6F12833B12
:10F540002DE9F04F2DED068B41F6B855C2F20005BE
:10F5500040F2AC24A5B0C1F2000400214FF48A624D
:10F5600028460EF0CDFEDFED5F8AD4EDE82A9FED50
:10F570005E9A002022EEA80ACBF68070E86085ED46
:10F58000019A85ED029A0EF067F894EDE82AF0EE04
:10F59000409A22EE280A0EF0F7FBD4EDE91AB0EEFD
:10F5A00040AA21EEA80A0EF057F8D4EDE97A29EE28
:10F5B000808A27EEA80A0EF0E7FB00EE498A94ED58
:10F5C000E91A21EE280A85ED048A0EF045F8D4EDFB
:10F5D000E90AB0EE408A20EEA80A0EF0D5FB29EE2B
:10F5E000800A08EE090A03214EF6250610220B4672
:10F5F000B1EE4AAA1120C0F6000685ED050A009674
:10F6000085ED06AA04F074FB0146296004F58168C3
:10F6100004F0E8FA04F5806A04F5826C04F584626B
:10F6200004F5836B04F58569DBF800E0DCF80C7009
:10F63000D9F80060DAF80CB0D8F80090DCF804A033
:10F64000DCF80080D2F804C01368D168CDF84CC053
:10F6500004F5866204F5886C04F58764C5F83C04FB
:10F66000CDF824E0CDF828E0CDF82CE00C970D97EC
:10F670000E970F9310931193129314961596169656
:10F6800017911891CDF80C90CDF81090CDF814B0DA
:10F69000CDF81880CDF81C80CDF820A01991116804
:10F6A000D668D2F804E0DCF800202468DCF80470A6
:10F6B00028681A9100231B911C91239203A914AA74
:10F6C000CDF874E000931E961F9620972194229403
:10F6D00004F08AFAFFF7E6FD25B0BDEC068BBDE825
:10F6E000F08F00BF35FA8E3C00000000F8B50546EB
:10F6F0000C460120582116461F46FBF7D1F8069903
:10F70000079B089AC161036209990A9B4262816260
:10F71000C3620B9A0C990D9B0561C46046618761B9
:10F72000026341638363F8BD0169C2684369F0EE17
:10F73000407A91ED006A92ED007A002B00F0CD80C6
:10F74000D3ED005A8369002B00F0CD80D3ED006A21
:10F75000C36A5BB1B3F9003001EE103AB8EEC10AEA
:10F760009FED625A60EE064A04EE856A036B5BB158
:10F77000B3F9002003EE102AF8EEC32A9FED5B2AAE
:10F7800062EE871A01EE827A436B5BB1B3F9001027
:10F7900005EE101AF8EEC54A9FED544A65EEA43AFC
:10F7A00043EE845A836B5BB1B3F900C002EE10CA1A
:10F7B000F8EEC21A9FED4D1A26EEA10A40EE016A3C
:10F7C00037EEE05AC36926EE056A80ED126AD3ED82
:10F7D000004AB4EEE46AF1EE10FA6EDCF1EE644A2F
:10F7E000B4EEE46AF1EE10FA67D490ED026A75EEB9
:10F7F000062A026A27EE226AC0ED022A80ED136A09
:10F8000092ED005AB4EEC56AF1EE10FA47DCB1EEA3
:10F81000455AB4EEC56AF1EE10FA40D441690029A8
:10F8200046D090ED013AB1EE604A74EE433A65EE8F
:10F83000A65A06EEA33A25EEA37A80ED013A80EDB2
:10F84000147A436AD3ED006AB4EEE67AF1EE10FA68
:10F8500036DDC0ED146AB0EE667AD0ED124A90ED56
:10F86000135A74EE856AC0ED0F0A37EE260AC0ED12
:10F87000157A80ED110A816AD1ED007AB4EEE70ABB
:10F88000F1EE10FA24DCF1EE677AB4EEE70AF1EE5D
:10F8900010FA44BFC0ED117AB0EE670A704785EEEA
:10F8A000077A416980ED135A80ED027A0029B8D1B8
:10F8B0000022026507EE102ACFE7C0ED124A94E756
:10F8C000F1EE666AB4EEE67AF1EE10FAC5D5C0E75D
:10F8D000C0ED117AB0EE670A70478369DFED045A14
:10F8E000002B7FF433AFF7EE006A31E76F12033B72
:10F8F00000000000C16891ED001AB5EE401AF1EE6B
:10F9000010FA18BF80EE811AF1EE407A18BF80ED30
:10F91000021A0023C0ED017A80ED150A436480EDE0
:10F920000F0A80ED100A704710B54AF2F074C1F268
:10F93000000440F68C22A1684AF2F074431A9BB28C
:10F94000C1F200049342A06016D9A37B227B23BBA3
:10F95000FF200C2A20743BD94AF2F070C1F200005B
:10F960000021C1734AF2F073C1F2000300205A7300
:10F97000012218735A7410BD617C69B1227B0B2A75
:10F980002FD8A3F53A70811F1FFA81FC40F2DC509A
:10F99000844538D90023237410BD934224D04AF6FD
:10F9A000BC1CC1F2000C4AF2F073DCF83440C1F226
:10F9B00000034AF2F071601CC1F20001FF24CCF890
:10F9C00034005A73002001220C7418735A7410BD4D
:10F9D00094F80DC09445BFD1E37B132B1AD9A273C1
:10F9E000C0E70022627410BD637C002BD7D01822C0
:10F9F00004F1120004F12A010EF064FC01222271CC
:10FA00002274227BAEE704EB420C0132ACF82A30C0
:10FA1000227310BD0133E373A4E700BF10B54AF2AF
:10FA2000F074C1F200040021442220460EF068FC6C
:10FA30004FF62913C0F600030D2001214FF4803248
:10FA400000F040FD206010BD10B44AF2F073C1F226
:10FA50000003187900286BD040F2AC24C1F20004F6
:10FA600094ED022AFDEEC27A94ED0F1A17EE901A69
:10FA700003EB410CF1EE040ABCF9120006EE100A89
:10FA8000F8EEC61AD4ED0E7A31EEC10ADFEDDA6A6D
:10FA900020EE207A002287EE277A1A71B4EEE67AF9
:10FAA000F1EE10FA46D54FF6AE6440F2AC23C1F247
:10FAB000000393ED030ABDEEC07A4AF2F07C17EE24
:10FAC000100AC1F2000C0CEB400293ED107AB2F96F
:10FAD00012C006EE90CAF8EEE65AB1EE045A75EE80
:10FAE000C74ADFEDC73A24EE854A4AF6BC12C4EE97
:10FAF000276A0831C1F2000222F81140F4EEE36AED
:10FB0000F1EE10FA21D4DFEDBF0AF4EEE06AF1EE77
:10FB100010FA40F3978240F2FF3218E04FF47C4134
:10FB20004AF6BC13C1F200030832012023F8121078
:10FB300010BC7047DFEDB12AB4EEE27AF1EE10FAB4
:10FB400040F3868240F2AD64AFE74FF47C4240F26E
:10FB5000AC21C1F20001D1ED044ABDEEE44A4AF203
:10FB6000F07C14EE101AC1F2000C0CEB4103F1EE24
:10FB7000042AB3F912C003EE90CAB8EEE33ADFEDFF
:10FB8000A01A33EE472A4AF6BC1322EE226A083046
:10FB9000C6EE276AC1F2000323F81020F4EEE16AF2
:10FBA000F1EE10FA0AD49FED975AF4EEC56AF1EE21
:10FBB00010FA40F3418240F2FF3001E04FF47C4004
:10FBC00040F2AC22C1F20002D2ED052ABDEEE22ADB
:10FBD0004AF2F07C12EE102AC1F2000C0CEB420348
:10FBE000B1EE041AB3F912C006EE10CAF8EEC61A46
:10FBF0009FED830A71EEC70A4AF6BC1360EE816A74
:10FC00000831C6EEA76AC1F2000323F81100F4EE32
:10FC1000C06AF1EE10FA0AD49FED7A3AF4EEC36AA4
:10FC2000F1EE10FA40F3028240F2FF3001E04FF4AF
:10FC30007C4040F2AC21C1F2000191ED061AFDEECC
:10FC4000C10A4AF2F07C10EE901AC1F2000C0CEBE3
:10FC50004103F1EE045AB3F912C006EE90CAB8EEB1
:10FC6000E60A9FED674A30EE475A4AF6BC1365EE46
:10FC7000254A0832C4EEA76AC1F2000323F8120035
:10FC8000F4EEC46AF1EE10FA0AD4DFED5E1AF4EE77
:10FC9000E16AF1EE10FA40F3C38140F2FF3001E077
:10FCA0004FF47C4040F2AC22C1F20002D2ED075A80
:10FCB000BDEEE55A4AF2F07C15EE102AC1F2000CB6
:10FCC0000CEB4203F1EE043AB3F912C004EE90CA11
:10FCD000B8EEE44A9FED4A2A34EE473A4AF6BC139E
:10FCE00063EE232A0831C2EEA76AC1F2000323F8AB
:10FCF0001100F4EEC26AF1EE10FA0AD49FED410A47
:10FD0000F4EEC06AF1EE10FA40F3848140F2FF3065
:10FD100001E04FF47C4040F2AC21C1F20001D1ED92
:10FD2000083ABDEEE33A4AF2F07C13EE101AC1F243
:10FD3000000C0CEB4103B1EE046AB3F912C002EE01
:10FD400090CAB8EEE22ADFED2E0A72EE471A4AF6A2
:10FD5000BC1321EE861A0832C1EE276AC1F20003F5
:10FD600023F81200F4EEE06AF1EE10FA0AD49FEDE7
:10FD7000254AF4EEC46AF1EE10FA40F3458140F2F0
:10FD8000FF3001E04FF47C4040F2AC22C1F20002AF
:10FD900092ED096AFDEEC61A4AF2F07C11EE902A45
:10FDA000C1F2000C0CEB4203F1EE046AB3F912C08D
:10FDB00001EE10CAF8EEC10A9FED115A30EEC70AE3
:10FDC0004AF6BC1360EE265A0831C5EEA76AC1F2A6
:10FDD000000323F81100F4EEC56AF1EE10FA13D413
:10FDE0009FED082AF4EEC26AF1EE10FA40F30681A4
:10FDF00040F2FF300AE000BF0000A9C300A0D544D4
:10FE0000000080C400C07F444FF47C4040F2AC212D
:10FE1000C1F20001D1ED0A6ABDEEE60A4AF2F07CB9
:10FE200010EE101AC1F2000C0CEB4103F1EE044A83
:10FE3000B3F912C005EE90CAB8EEE55A1FED103ABC
:10FE400035EE474A4AF6BC1364EE243A0832C3EE54
:10FE5000A76AC1F2000323F81200F4EEC36AF1EEC0
:10FE600010FA0AD45FED190AF4EEE06AF1EE10FA26
:10FE700040F3BE8040F2FF3001E04FF47C4040F29E
:10FE8000AC22C1F20002D2ED0B4ABDEEE44A4AF2C6
:10FE9000F07C14EE102AC1F2000C0CEB4203F1EEE0
:10FEA000042AB3F912C003EE90CAB8EEE33A5FED4C
:10FEB0002C1A33EE472A4AF6BC1322EE226A083186
:10FEC000C6EE276AC1F2000323F81100F4EEE16ADE
:10FED000F1EE10FA09D41FED355AF4EEC56AF1EED1
:10FEE00010FA7FDD40F2FF3001E04FF47C4040F239
:10FEF000AC21C1F20001D1ED0C2ABDEEE22A4AF29A
:10FF0000F07C12EE101AC1F2000C0CEB4103B1EEC2
:10FF1000041AB3F912C006EE10CAF8EEC61A1FEDA5
:10FF2000480A71EEC70A4AF6BC1360EE816A0832CD
:10FF3000C6EEA76AC1F2000323F81200F4EEC06A0D
:10FF4000F1EE10FA09D41FED513AF4EEC36AF1EE66
:10FF500010FA41DD40F2FF3001E04FF47C4040F206
:10FF6000AC22C1F20002D2ED0D0AFDEEE06A4AF2C7
:10FF7000F07C16EE902AC1F2000C0CEB4203B1EEBD
:10FF8000045AB3F912C000EE10CAF8EEC05A4AF68D
:10FF9000BC1375EEC74A1FED667A24EE854A083118
:10FFA000C4EE277AC1F2000323F81100F4EEC77AF9
:10FFB000F1EE10FA3FF5B2AD1FED6E1AF4EEC17A14
:10FFC000F1EE10FA02DD40F2FF31A9E5FDEEE77A2D
:10FFD00017EE901A89B2A3E5FDEEE63A13EE900A09
:10FFE00080B2BCE7FDEEE65A15EE901A88B27EE7C5
:10FFF000BDEEE61A11EE100A80B240E7FDEEE62AE9
:020000040801F1
:1000000012EE901A88B201E7FDEEE64A14EE900A6D
:1000100080B2B9E6FDEEE66A16EE901A88B27AE68C
:10002000BDEEE66A16EE100A80B23BE6FDEEE63A59
:1000300013EE901A88B2FCE5FDEEE65A15EE900A32
:1000400080B2BDE5BDEEE61A11EE101A8AB27EE569
:10005000BDEEC73A13EE103A9CB226E54AF2F073B1
:10006000C1F2000393F91000704700BF70B584B06F
:100070000C461646054601A807F03EFE013C00234B
:10008000013E284601A90294ADF80460ADF80C3099
:10009000ADF8063007F0D4FD04B070BD70B586B081
:1000A000044601A815460E4607F06EFF00236020A7
:1000B0000122ADF80400ADF80620ADF81030ADF81F
:1000C000083003950C2E0CD8DFE806F0170B0B0B4D
:1000D000120B0B0B0D0B0B0B0700204601A907F0B1
:1000E00019FF06B070BD204601A907F0C3FEF8E76E
:1000F000204601A907F06EFEF3E7204601A907F0AC
:100100001DFEEEE770B584B0044601A80D46164604
:1001100008F03CF800230122204601A9ADF8045064
:10012000ADF80660ADF80820ADF80A30ADF80C3037
:1001300007F060FF04B070BD10B584B00446684697
:1001400008F04EF800214FF48040ADF80410ADF8EF
:100150000C004FF4806320466946ADF8023008F089
:1001600025F804B010BD00BF70B582B004466846E3
:100170000D46164607F0B6F80023022220466946CF
:1001800000958DF804608DF805208DF806308DF807
:10019000073006F0EBFF02B070BD00BF0D2810B5B0
:1001A00019D84AF63403C1F20003C0EBC00003EBD8
:1001B000800393F91040B4B959B1DB68DBB19942BF
:1001C00007D041F6B060C0F60200F2F78DFB204682
:1001D00010BD012010BD41F66060C0F60200F2F7CC
:1001E00083FB002010BD41F68860C0F60200F2F7E4
:1001F0007BFB002010BD012010BD00BF10B540F2F8
:100200003074C2F2000400212068012207F07EFD54
:1002100060680021012207F079FDA0680021012219
:1002200007F074FDE0680021012207F06FFD2069EE
:100230000021012207F06AFD60690021012207F018
:1002400065FDA0690021012207F060FDE069002141
:10025000012207F05BFD206A0021012207F056FD14
:10026000606A0021012207F051FDA06A01220021ED
:1002700007F04CFD0021E06A012207F047FD206BEA
:100280000021012207F042FD606B00210122BDE840
:10029000104007F03BBD00BF40F23073C2F20003D4
:1002A00053F8200007F038BD2DE9F84304460D4609
:1002B00016469846FFF772FF002800F09D8041F631
:1002C000D86EC0F6020E4AF6340C5EF82410C1F265
:1002D000000C40F230704DF68369C4EBC4070CEBA0
:1002E0008707C2F20000C4F21B39A9FB01320123C7
:1002F000920C50F824003B742946FFF7B7FEB8F182
:10030000000F56DB41F62072C0F6020240F268731D
:1003100052F82490C2F200031FFA89F153F8240026
:100320005FFA88F2F8F7FCFE40F26875C2F2000549
:10033000494655F824000222FFF716FF41F62462D1
:1003400041F64063C0F60203C0F6020241F610789F
:10035000C0F6020855F8240032F814101A5D40F275
:10036000307506F0CFFFC2F2000518F8048055F88A
:10037000240041463246FFF791FE41F6506CC0F62C
:10038000020C1CF8041091BB40F23070C2F2000065
:10039000012150F8240007F0C3FCB8F10C0F1BD862
:1003A000DFE808F0481A1A1A3B1A1A1A2E1A1A1AF3
:1003B0000E0041F62075C0F6020555F82490B3E70B
:1003C00040F2307EC2F2000E5EF8240000F14001DF
:1003D0003960082107F002FE40F2307CC2F2000CC6
:1003E00038465CF8243024337B60BDE8F88355F848
:1003F0002400FFF7A1FEC7E707463846BDE8F883AB
:1004000040F23070C2F20000082150F8240000F1E0
:100410003C023A6007F0D8FDDEE740F2307CC2F2E1
:10042000000C08215CF8240000F138033B6007F061
:10043000BFFDD1E740F2307EC2F2000E5EF824002C
:1004400000F134013960082107F0A8FDC4E700BFBE
:1004500038B500210546FFF7A1FEE8B141F620714D
:1004600040F26872C2F20002C0F602014AF6340499
:1004700052F8250051F82510C1F20004C5EBC5055E
:1004800004EB85048BB201226061227423834383D1
:10049000FFF76AFE204638BD0446204638BD00BF3F
:1004A00000B583B001238DF80400022201A88DF865
:1004B00005208DF806308DF8073006F061FA03B09C
:1004C00000BD00BF2DE9F8430D46002104469146CA
:1004D0001E46FFF763FE002800F0A580002E00F006
:1004E000A68041F6D86EC0F6020E4AF6340C5EF8CD
:1004F0002410C1F2000C40F230704DF68368C4EB5A
:10050000C4070CEB8707C4F21B38C2F20000A8FB3B
:1005100001324FF00208920C50F82400BE604946A8
:1005200087F81080FFF7A2FD40F2687641F620714F
:10053000C2F20006C0F6020156F8240051F8241059
:100540004246FFF711FE41F6246241F64063C0F6D1
:100550000202C0F6020332F8141056F824001A5DA5
:1005600006F0D0FE002D32DD002241F61076C0F6F6
:10057000020640F23075365DC2F20005314655F88C
:100580002400FFF7BFFD55F82400012107F0C8FB48
:1005900041F65873C0F60203185DFFF781FF0C2E79
:1005A00012D8DFE806F024111111311111110711D1
:1005B0001111170040F2307CC2F2000C08215CF8E7
:1005C0002400012207F016FE3846BDE8F88328D142
:1005D0000A22CAE740F23070C2F20000102150F83F
:1005E0002400012207F006FE3846BDE8F88340F2F9
:1005F0003072C2F20002022152F82400012207F0F8
:10060000F9FD3846BDE8F88340F23071C2F20001CE
:10061000012251F82400042107F0ECFD3846BDE822
:10062000F8834246A1E707463846BDE8F8833746D7
:10063000CAE700BF38B50024C4F2010402212046F5
:1006400007F0E2FD012820462BD0042107F0DCFD55
:10065000012820463ED0082107F0D6FD012820467B
:1006600051D0102107F0D0FD012800D038BD102155
:10067000204607F0D5FD4AF63401C1F200012046BC
:10068000CC6D07F091FD40F26873C2F2000305469D
:100690004FF48041D86806F02FFE01462846A04757
:1006A00038BD022107F0BCFD4AF63401C1F2000159
:1006B00020468C6807F072FD40F26873C2F20003B6
:1006C00005464FF40071186806F016FE01462846EC
:1006D000A04738BD042107F0A3FD4AF63402C1F259
:1006E00000022046546A07F05BFD054640F2687040
:1006F000C2F200004FF40061406806F0FDFD0146C3
:100700002846A04738BD4AF634050821C1F2000545
:1007100007F086FD20462C6C07F044FD40F2687C13
:10072000C2F2000C05464FF40051DCF8080006F058
:10073000E3FD01462846A04738BD00BF38B54FF459
:100740000064C4F200040221204607F05DFD012888
:1007500020462CD0042107F057FD012820463FD029
:10076000082107F051FD0128204653D0102107F041
:100770004BFD012800D038BD1021204607F050FD68
:100780004AF63401C1F200012046D1F8CC4007F00E
:100790000BFD40F26873C2F2000305464FF40041BE
:1007A000D86906F0A9FD01462846A04738BD0221B8
:1007B00007F036FD4AF63401C1F2000120468C6F85
:1007C00007F0ECFC40F26873C2F2000305464FF4F8
:1007D0008051186906F090FD01462846A04738BDB3
:1007E000042107F01DFD4AF63402C1F20002204642
:1007F000D2F8944007F0D4FC054640F26870C2F28B
:1008000000004FF40051406906F076FD014628468D
:10081000A04738BD4AF634050821C1F2000507F0AB
:10082000FFFC2046D5F8B04007F0BCFC40F2687CE5
:10083000C2F2000C05464FF48041DCF8180006F0C7
:100840005BFD01462846A04738BD00BF38B54FF4D0
:100850008044C4F201040221204607F0D5FC01289F
:10086000204605D0042107F0CFFC012819D038BD5F
:10087000022107F0D5FC4AF63401C1F200012046FE
:10088000D1F8E84007F08AFC40F26873C2F2000336
:1008900005462021186A06F02FFD01462846A0478C
:1008A00038BD0421204607F0BBFC4AF63402C1F2F1
:1008B00000022046D2F8044107F072FC054640F2DF
:1008C0006870C2F200004021406A06F015FD014642
:1008D0002846A04738BD00BF082138B54FF08040FA
:1008E00007F092FC012807D010214FF0804007F05C
:1008F0008BFC01281DD038BD08214FF0804007F047
:100900008FFC4AF63401C1F200014FF08040D1F86B
:10091000204107F047FC40F26873C2F2000305462D
:100920004FF48061986A06F0E7FC01462846A0472C
:1009300038BD10214FF0804007F072FC4AF63402B7
:10094000C1F200024FF08040D2F83C4107F02CFC8D
:10095000054640F26870C2F200004FF40061C06AC0
:1009600006F0CAFC01462846A04738BD38B54FF40A
:100970008844C4F201040221204607F045FC012806
:1009800000D038BD0221204607F04AFC4AF6340167
:10099000C1F200012046D1F8584107F0FFFB40F2B8
:1009A0006873C2F2000305464FF48071186B06F0BD
:1009B000A3FC01462846A04738BD00BF38B54FF418
:1009C0009044C4F201040221204607F01DFC0128D6
:1009D00000D038BD0221204607F022FC4AF634013F
:1009E000C1F200012046D1F8744107F0D7FB40F274
:1009F0006873C2F2000305464FF40071586B06F0AD
:100A00007BFC01462846A04738BD00BF02EE100A15
:100A100010B5B8EEC21A4AF6BC14C1F20004F7EEE3
:100A2000001A04F1080031EE210AFAF7D3F8F6EEC5
:100A3000000A20EE200A9FED037A60EE077AC4EDEB
:100A40000E7A10BD0000C84270B53B4D3B486C6843
:100A5000F1F74AFF4FF44066C4F20006022008F0A6
:100A600069FF95F93C30042B1CD8DFE803F0080837
:100A700045543100706A28640120FFF7C7FF204603
:100A800002F000FE0146204661B102F009FE02F0CC
:100A900035FF0028EED1204602F0F4FD0146204645
:100AA0000029F2D12B6C706A4EF6602CC21A624596
:100AB0003DD895F93CE0BEF1030FCFD1FFF7CEFA58
:100AC000FFF7A4FFCAE7706A28640120FFF79EFFC2
:100AD000204602F0D7FD014620460029E2D002F070
:100AE000DFFDC0B205F0D4FB0028F1D0EBE7726A5D
:100AF00001202A64FFF78AFF204602F0C3FD034667
:100B00002046002BCED002F0CBFDC0B2F9F7D2F9CF
:100B10000028F1D0EBE7FEF797FF0028C2D0736AF8
:100B20002B64706A4EF6602CC21A6245C1D94FF030
:100B3000FF30FFF76BFF91E7BCA90010681F0208A8
:100B400038B541F67C704AF6BC14C1F20004C0F618
:100B50000200F1F7C9FE4422002120460DF0D0FB2F
:100B600004F108009FED260AF6EE080A9FED251A0B
:100B7000F9F7F8FF40F2AC20C1F2000090ED010A55
:100B8000FDEEC07A17EE902A53B284F83C20042B75
:100B90002DD8DFE803F029292623030005F0C0FB48
:100BA00041F6A871C0F602014020F9F79BFE42F21F
:100BB0000824C2F20004054640F649200021C0F690
:100BC000010005F1FC0344F21902256008F08EFDD6
:100BD0004AF6BC11C1F20001087038BDFEF71EFFD5
:100BE000DEE7F9F78FF9DBE702F0F0FED8E741F630
:100BF0008870C0F60200BDE83840F1F775BE00BF4E
:100C00000AD7A33C0000000000B5012183B01F20DB
:100C100006F022FC684606F065FB4FF48060032274
:100C20004FF6FF736946C4F202008DF8042000936A
:100C300006F09CFA4FF400606946C4F2020006F028
:100C400095FA4FF440606946C4F2020006F08EFA4D
:100C50004FF480506946C4F2020006F087FA002083
:100C600049F6FF736946C4F20200009306F07EFA6B
:100C700001214FF4C00006F0EFFB01214FF480404A
:100C800006F006FC0720012106F0F4FB01200121FB
:100C9000C0F2070006F0FCFB012006F0E1FE06F0C2
:100CA0003FFC42F20C20C2F2000006F04FFBFFF7BF
:100CB000A5FA03B000BD00BF2DE9F0474FF4205462
:100CC000C4F2000484B0E66816F0400600F04B81E0
:100CD0003030C0B2C9B200F5FA6A48F21F55022995
:100CE000CCBF5446AAF10104C5F2EB1541F6DC79FC
:100CF00085FB046EC0F60209E61701F1FF35A6EB8D
:100D00006E1704EBA40404EB070859F82550C6EB52
:100D1000EE1708EB070C0CEB0506D2B2941942F261
:100D20009347013CC9F2492787FB046909EB040892
:100D3000E517C5EBA806C6EBC607E41B651C09282A
:100D400089469046EDB240F219810A384CF6CD46FC
:100D5000C0B2CCF6CC46A6FB006701240928C7F335
:100D6000C0060DD926B10A38C0B20224092807D915
:100D7000143800F0FF000234092804F0FF04F7D80B
:100D80002701FCB220430004092940F2F9800A3906
:100D90004CF6CD46C9B2CCF6CC46A6FB016C01247C
:100DA0000929CCF3C0060DD926B10A39C9B20224EB
:100DB000092907D9143901F0FF010234092904F087
:100DC000FF04F7D82701FCB221430902092A40F2A7
:100DD000D9800A3A4CF6CD46D2B2CCF6CC46A6FB28
:100DE000026E0124092ACEF3C0060DD926B10A3AB3
:100DF000D2B20224092A07D9143A02F0FF020234BF
:100E0000092A04F0FF04F7D82701FCB240EA453C68
:100E100044EA02064CEA010747EA060121F07F4551
:100E20004FF4205025F0C002C4F20000DDB2092DBD
:100E300042609DF830609DF8347040F2A580A5F1C5
:100E40000A034CF6CD40DBB2CCF6CC40A0FB030449
:100E50000122092BC4F3C0010DD921B10A3BDBB239
:100E60000222092B07D9143B03F0FF030232092B9E
:100E700002F0FF02F7D81101CAB242EA03042304C8
:100E8000092E40F28480A6F10A0C4CF6CD405FFAA0
:100E90008CF2CCF6CC40A0FB020E0121092ACEF345
:100EA000C0000DD920B10A3AD2B20221092A07D9CD
:100EB000143A02F0FF020231092A01F0FF01F7D8CB
:100EC0000C01E1B20A43092F43EA022253D9A7F1E8
:100ED0000A0E4CF6CD405FFA8EF1CCF6CC40A0FB6A
:100EE000010301200929C3F3C0030DD923B10A3935
:100EF000C9B20220092907D9143901F0FF01841C65
:100F0000092904F0FF00F7D80301D8B240EA010430
:100F10004FF4205C47F67F702243C4F2000CC0F20D
:100F20007F0002EA0001CCF8001006F05FFB42F2FD
:100F30001C24012006F0FEFAC2F2000441F6B07152
:100F4000C0F6020152464B462046CDF8008001957E
:100F5000029603970DF05EF92046F1F7C5FC0120DB
:100F600004B0BDE8F087304606F0E4FA4FF0FF33F6
:100F7000E3603046F4E739460020C7E7002401E784
:100F8000002421E7002441E72B46002275E7324682
:100F9000002197E730B583B0002001A906F0A4FB3B
:100FA0000020694606F072FB9DF805309DF806505A
:100FB0009DF800409DF801109DF802209DF8070063
:100FC0005B0543EA054343EAC42C4CEA411141EA7C
:100FD0005203143043EA406003B030BDF0B54AF626
:100FE00000208BB018220021C1F200000DF088F91A
:100FF00001214FF0805006F03DFA012006F09AF9E9
:10100000012006F09DF96124204606F06BFA0028C5
:10101000FAD04FF4007006F0F7F9012006F016FA46
:1010200006F0EEFA4FF480000124002505F0ECFFF5
:10103000082707A84FF4800607968DF821708DF8D1
:1010400022408DF8205005F09BFF032109A88DF860
:1010500024108DF825408DF827408DF8265005F096
:101060008FFC284606F08CFB042006F06BFB28461C
:1010700006F07AFB204606F083FB4FF4804006F032
:10108000F7FB4FF4406621464FF48040C4F200065F
:1010900006F0A6FB3846214606F0ECF93046402122
:1010A00007F0C2F822463046294606F02FFE0C22F1
:1010B00004A93046ADF81020ADF81620ADF8144064
:1010C000ADF81250ADF8185006F094FF322309A87D
:1010D0008DF824308DF827408DF825508DF8265056
:1010E00005F04EFC2146304606F01AFE22463582B7
:1010F0003046102107F07EF84AF600242F46C1F250
:10110000000460690128FCDD4FF44060C4F2000077
:1011100006F0ACFC42F20C2CC2F2000C4DF68365DA
:10112000DCF80820E06821695300C4F21B35A5FBF8
:10113000035244F65F03950C091AC0F20F031FFA1D
:1011400081FC03FB05F0B0FBFCF24CF6CD45D10071
:10115000CCF6CC45A5FB01230AA89B08013B042241
:10116000002584E80E0040F8245D0292039306F007
:1011700013FA012006F06CFA284606F0DBF906F0B7
:10118000E7F90BB0F0BD00BF08B54FF4804006F0A2
:1011900055FB00B908BD4FF4804006F069FB4FF4E1
:1011A0008000BDE8084005F02FBF00BF2DE9F04FDB
:1011B0002DED068B42F20C008BB0C0F60200F1F769
:1011C00093FB46F2676741F210134CF6CD494AF69D
:1011D000182440F22016C1F20003C6F26667CCF66E
:1011E000CC49C1F2000400250493C1F20006059722
:1011F000CDF8009039E0009FEB1DA7FB03710A09B1
:1012000002EB8200B3EB800F00F05A81DDF800B0F2
:1012100005F10E0AABFB0A92130903EB8300BAEB4C
:10122000800F40F0F3809FEDD95A20EE050A66EE5C
:10123000850A27EE051AFDF759FDFDF7EDFBFBF7D3
:10124000CBFE48F21F50C5F2EB10A0FB0513990925
:10125000C82707FB1152002A00F0D580F9F730FDAE
:101260000135F8F743FFF1F79FFCDDF810900021FE
:1012700099F8010007F002FCFDF71AFCD6F830B12E
:10128000D4F84031D6F834A1D6F83891D6F83C716C
:10129000D6F84011D6F8442101970291039203EE4B
:1012A00010BA03F10208DDF814B003F10C0E03F1DB
:1012B000160003F1200C03F12A0703F1340103F1B6
:1012C0003E0204EB8808013304EB8E0E04EB800031
:1012D00004EB8C0C04EB870704EB810104EB820226
:1012E000D8ED010ADEED017A90ED010ADCED016A2C
:1012F00097ED017A91ED012A05EE109A04EE10AAFD
:1013000094ED49AA8BFB039AD4ED4A9ADDF800B01C
:1013100094ED4B9AD4ED4C8A94ED4D8A94ED4E1A8F
:10132000D4ED4F1AD2ED01AA4FEAE379DDED013A8F
:10133000DDED035A96ED456ADDED024A7AEE602A4C
:10134000C9EBAA0A79EEE70AABFB05B979EE407A58
:1013500038EEE60A78EE476A31EE427A31EEEA2A52
:101360000AEB8A0A4FEA191BA3EB4A0372EE832A9F
:1013700070EE840A77EE857A30EE230A76EEA46A60
:1013800037EE257A32EE062A0BEB8B0AB5EB8A0F85
:1013900088ED013ACCED013A8EED014AC7ED014AE4
:1013A00080ED015AC4ED492AC4ED4A0AC4ED4B7AD6
:1013B000C1ED015A84ED4C0AC4ED4D6A84ED4E7ABC
:1013C00082ED016A84ED4F2AC4F840317FF413AFF7
:1013D0009FED6E6A22EE860A60EE860A27EE861A76
:1013E000FDF716FCFDF718FBFBF7F6FD48F21F5062
:1013F000C5F2EB10A0FB05139909C82707FB115292
:10140000002A7FF42BAFF9F705FC27E741F26807C4
:10141000C1F20007B87807F005FB002857D1D4EDDA
:10142000017AB7EE007AF4EEC77AF1EE10FAD7ED52
:10143000132A15DDF1EE044AF4EEE42AF1EE10FA77
:101440000ED59FED534A77EEC47AF4EEC77AF1EEEB
:1014500010FAC4ED017A44BF84ED017AF0EE477AC8
:1014600041F26807C1F2000797ED143A62EEA72A2D
:1014700027EE833AD7F8980097ED0E0B97ED101BE7
:1014800097ED122AFDF77CFCB87807F099FBD7EDB1
:10149000137AD4ED023AF4EEE37AF1EE10FA7FF526
:1014A000CCAEF0EE082AF4EEE27AF1EE10FA7FF517
:1014B000C4AE97ED120AFCF777FDF96CA160BCE6AB
:1014C000DFED325A22EE250AFDF768FBB5E67878A3
:1014D00007F0A8FA002845D04AF6144CC1F2000CD7
:1014E0009CF8BC717B073FF5A8AE0A21294807AAE2
:1014F00008F038FD0A2104F1340008AA08F032FD92
:101500000A2104F15C0009AA08F02CFDDDED088A2F
:10151000DDED076A9DED098A36EEA87A9FED1B1A6C
:1015200037EE082AB4EEC12AF1EE10FA7FF585AE47
:1015300042F2402EC2F2000E4AF6AB20DEF8002046
:10154000D6F82C71CAF6AA20A0FB02B3590801EB09
:101550004100531C00EE107A101ACEF80030FDF74F
:10156000F9FA6AE6D7ED1AAAD4ED011AD7F89C0069
:1015700097ED150AD7ED160A97ED171A6AEEA11A1C
:10158000FDF772FD787807F01BFB56E6CDCCCC3D1D
:101590000AD7A33C24AA0010F8B54AF61824C1F2D1
:1015A00000044FF4A272002120460CF0A9FE42F282
:1015B0002001C0F60201FA20F9F794F942F244251D
:1015C000C2F20005064641F2AD1006F579732E60B1
:1015D00000214FF61E22C0F6010008F087F840F205
:1015E000201CC1F2000CDCED457ADCF83071DCF82F
:1015F0003461DCF83851DCF83C11DCF84021DCF8CF
:101600004431207006EE101A07EE103A04EE907A7C
:1016100005EE106A05EE905A06EE902A94ED492ADE
:10162000D4ED4A2A94ED4B3AD4ED4C3A94ED4D4A20
:10163000D4ED4E0A94ED4F0A32EE241A72EE851A5A
:1016400035EE832A76EE232A36EE843A77EE203A78
:1016500037EE804A74EE810A35EE210A35EE822A91
:1016600076EE222A36EE833A77EE233A37EE844A34
:1016700034EEA01A75EE001A75EE820A36EE220AD2
:1016800036EE833A77EE233A37EE844A35EEA02AD7
:1016900076EE002A76EE830A37EE230A37EE844A86
:1016A00034EE811A75EE211A34EE811A36EEA03A24
:1016B00077EE003A77EE840A75EE211A35EE822A2B
:1016C00076EE222A34EE810A75EE211A35EE822A50
:1016D00037EEA04A76EE222A36EE833A77EE233AA8
:1016E00034EE801A75EE210A35EE820A76EE222A51
:1016F00036EE833A77EE233A37EE844A75EE201AB7
:1017000035EE802A76EE220A36EE830A77EE233A09
:1017100037EE844A34EE811A76EE202A36EE803A8D
:1017200034EE811A75EE211A35EE822A77EE230AFD
:1017300037EE840AC4F88410C4F8D430C4F8881092
:10174000C4F8D830C4F88C1034EE811A75EE211A22
:1017500035EE822A76EE222A36EE833A77EE203A6A
:1017600037EE804AE7606663E565C4F8AC20C4EDF7
:101770003F7A2761A6632566C4F8B020C4ED407A9D
:101780006761E6636566C4F8B420C4F8DC30C4F869
:101790009010C4F8E030C4F89410C4F8E430C4F8F1
:1017A0009810C4F8E830C4F89C10C4F8EC30C4EDCC
:1017B000417AA7612664A566C4F8B820C4ED427AD0
:1017C000E7616664E566C4F8BC20C4ED437A27622D
:1017D000A6642567C4F8C020C4ED447A6762E66455
:1017E0006567C4F8C420C4ED457AA7622665A5677D
:1017F000C4F8A010C4F8A410C4F8A8104CF6CD4149
:10180000C4F8F030C4F8F430C4F8F830C4F2C7219A
:101810004FF07E500023C4F8C820C4ED467AE7623A
:101820006665E567C4F8CC20C4ED477A2763A665F2
:10183000C4F88050C4F8D020C4ED487A84ED491A29
:10184000C4ED4A1A84ED4B2AC4ED4C2A84ED4D3A7E
:10185000C4ED4E3A84ED4F4AA1606060C4F8403157
:10186000F8BD00BF10B54FF43053C4F201035C6BF8
:1018700014F0450FFBD063070DD414F0010405D11B
:1018800040F2FF5006F0B6F8204610BD012006F0E9
:10189000B1F8012010BD042006F0ACF8032010BD03
:1018A0004FF43052C4F20102536B13F0450F07D1CD
:1018B00000BF00BF00BF00BF506B10F0450FF7D056
:1018C0004FF4305CC4F2010C40F2FF53CCF83830D6
:1018D000DCF8142002F00801C8B270472DE9F0418D
:1018E000044692B0002006F037F810F0007304D0E0
:1018F0000E23184612B0BDE8F08110220BA808276D
:1019000040264FF4806510930C920E930B970D9622
:101910000F9505F0FFFFFFF7C3FF024603460028BF
:10192000E7D14AF65C38C1F200080BA8D8F830308D
:101930000E92190437230C930B910D960F9505F019
:10194000E9FFFFF7ADFF804603460028D1D14FF0F5
:10195000FF330121302268468DE88800022303937B
:1019600005910292CDF8108006F004F833220BA8FE
:101970000C92CDF82C800D96CDF838800F9505F09F
:10198000C9FFFFF78DFF03460028B2D14FF4305551
:101990000DEB0608C4F2010540F22A664FF4001769
:1019A000686B304209D1384606F01AF80028F7D0A3
:1019B00005F0FAFF48F8040BF2E7082006F010F8EB
:1019C00020B1082006F016F8042392E7022006F062
:1019D00007F820B1022006F00DF8022389E7202045
:1019E00005F0FEFF20B1202006F004F8062380E772
:1019F0004FF4007005F0F4FF054628B14FF4007075
:101A000005F0F8FF072374E740F2FF5005F0F2FFFE
:101A10001099012C0BBA29D0DA0301D4252368E7E9
:101A20004AF65C3EC1F2000E3723DEF8300009951D
:101A30000204402506A84FF4806407930692089597
:101A40000A9405F067FFFFF72BFF034600287FF499
:101A500050AF06A8069309930621079108950A94AA
:101A600005F058FFFFF71CFF034642E75903D5D5A1
:101A70004AF65C3CC1F2000C3723DCF83040099593
:101A8000220406A840254FF4806407930692089527
:101A90000A9405F03FFFFFF703FF034600287FF499
:101AA00028AF022106A809930691D5E700B54FF4A7
:101AB000006083B00123C4F202004FF400518DF89E
:101AC000073005F019FC10B100208DF807009DF8D3
:101AD000070003B000BD00BF10B44AF65C33C1F28A
:101AE000000383B05A6801218DF80710AAB14FF4A2
:101AF0004064C4F2000448F2A060646A61F31F40CD
:101B0000A21A824209D998680168B0F804C000227C
:101B1000A1F81AC08DF807201A709DF8070003B0CD
:101B200010BC70472DE9F0418CB00024B22168460A
:101B30008DF814108DF82F400094019402940394B2
:101B4000049405F0B3FE032005F0D6FE012005F055
:101B5000CDFE4FF4806306A8069407940894099478
:101B60000A934FF4803505F0D5FE802406E005F099
:101B700037FF013D48B9013D00F0CF80204605F018
:101B80002FFF02462046002AF1D040F2FF5005F018
:101B900031FF00238DF82F309DF82F3023B19DF8B1
:101BA0002F000CB0BDE8F08108214FF4D57240241D
:101BB00006A84FF4806706920791089409930A9744
:101BC00005F0A8FE4FF43051C4F201014A6B12F047
:101BD000450F0ED14FF4803305E04A6B013B12F004
:101BE000450F05D143B14A6B013B12F0450FF4D0CC
:101BF00013B112F004046FD0042005F0FBFE03249F
